:020000040800F2
:1000000000000110F1FC060811230008ED48020869
:1000100091FD060891FD060891FD0608000000000C
:10002000000000000000000000000000B1470008D0
:10003000B547000800000000B947000831D00008AB
:1000400091FD060891FD060891FD060891FD060840
:1000500091FD060891FD0608F9A00008FDA0000822
:1000600091FD060801A1000805A10008C9280008A3
:10007000DD280008F12800080529000819290008D2
:100080002D2900084129000891FD060891FD060868
:1000900091FD060891FD060891FD060809A10008DA
:1000A000752700089D270008C5270008612700085C
:1000B000ED270008012800081528000891FD060812
:1000C00091FD060891FD060891FD060891FD0608C0
:1000D00091FD060815230008212300082D230008A0
:1000E0000DA1000891FD0608BD4700085128000831
:1000F00079280008A12800083D2800085529000893
:1001000091FD060891FD06082928000891FD0608C2
:10011000392300084523000891FD060891FD0608D3
:10012000692900087D29000891290008A5290008EF
:10013000B929000891FD060891FD060891FD060801
:1001400091FD060891FD060891FD0608114800087A
:10015000C9290008D9290008E92900085123000805
:1001600091FD060891FD060891FD060891FD06081F
:1001700091FD060891FD060891FD060891FD06080F
:0801800091FD060891FD06083F
:10019000D0E907239A422FBFD01AC0688018C01A2E
:1001A000704700BFD0E9092300699A4238BF12188E
:1001B000D31A0138C01A7047D0E90902101AB0FAF0
:1001C00080F04009704700BF0246036A4069D16869
:1001D000C05C01338B4228BF00231362704700BF0D
:1001E000436A8269D154436A0169426B01338B428D
:1001F00028BF00234362D36843F08003D360704775
:10020000436B188810F0100002D01A889B880120D8
:10021000704700BF436B99891A88890610B5044658
:100220000AD592B2900607D5E26A002A29D09888AA
:10023000216B80B29047636B99891A88090692B244
:100240000FD510060DD5D4E909128A4214D0A16940
:100250002069895C99800132B2FBF0F100FB112228
:10026000A262998A1A88C90592B204D5D20744BFFE
:100270004FF6F7721A8010BDDA6822F08002DA6059
:10028000EFE79B88E2696169DBB28B54E269E16860
:10029000636B0132B2FBF1F001FB1022E261CBE7AC
:1002A000036942681F2B10B40AD95468A3F1200CCB
:1002B000202101FA0CF1214207D15DF8044B70476F
:1002C0001468202199402142F7D081690024C86830
:1002D0000C7480684C68016821F00101016020689D
:1002E00094F805C00C4C818934F81C4089B221EA8D
:1002F00004011F2B818107D9A3F1200120238B400A
:100300005DF8044BD3607047202101FA03F35DF8D8
:10031000044B9360704700BFE464070882B0092271
:10032000274B8DF80720DA68D00319D4DA68D10694
:1003300040D4DA68D20541D4DA6812F0E00F3BD13C
:10034000DB6813F0020F14BF082309238DF8073070
:100350009DF80730012B0AD09DF8070002B07047C6
:1003600001238DF807309DF80730012BF4D1144A92
:1003700012E0D368DB0519D4D36813F0E00F17D16E
:10038000D36813F0020F14BF082309238DF8073038
:100390009DF80730012BDFD1D168C8034FF001036E
:1003A000F4D4D368D906E4D50623EFE70223EDE7BA
:1003B0000723EBE70623D4E70723D2E70223D0E79E
:1003C000003C0240704700BF704700BF01207047EB
:1003D000034BD3E90003C01AC0F30A00704700BF03
:1003E00038220020054AD2E900138B42FDD0D118F3
:1003F0000133C3F30A03087A5360704738220020A0
:10040000064BD3F8080800B97047D3F80808A0F1E4
:100410000500B0FA80F04009704700BF3822002084
:10042000012380F849307047044BD3E90003C01A18
:10043000C0F30A00C0F50060704700BF38220020FA
:1004400010B5D0F8E83504461B699847032384F8B3
:100450001231002010BD00BF08B5042290F812111F
:10046000D0F8E83580F8131180F81221DB6898473E
:10047000002008BD08B5D0F8E435DB6903B1984722
:10048000002008BD08B5D0F8E4351B6A9847002065
:1004900008BD00BF08B5D0F8E4355B6A9847002076
:1004A00008BD00BF037830B403B30446C0F1010CAB
:1004B00004EB0C0314F8015FDBB2002DF8D101331B
:1004C0005B00DCB2138003230C704B7004785CB1CA
:1004D000022300255A1CD2B2CC548D5410F8014F7F
:1004E0000233DBB2002CF5D130BC70470224234626
:1004F000E8E700BF10B5074C2068FF2808D0064980
:10050000D1F80C2801F5016100F080F8FF23236089
:10051000002010BD000000203822002043230148A5
:100520000B80704704000020122301480B807047A5
:1005300048000020042301480B8070475C00002025
:1005400008B5044B04480A461946FFF7ABFF0846B6
:1005500008BD00BF502A00200813080808B5044B46
:1005600004480A461946FFF79DFF084608BD00BF2C
:10057000502A00201413080808B5044B04480A4602
:100580001946FFF78FFF084608BD00BF502A00201C
:100590001C13080808B5044B04480A461946FFF71F
:1005A00081FF084608BD00BF502A00202813080814
:1005B00008B5044B04480A461946FFF773FF08467E
:1005C00008BD00BF502A002034130808704700BF40
:1005D000704700BF704700BF704700BF704700BF43
:1005E000704700BF044B00200522C3F80828C3F859
:1005F0001809C3F81C09704738220020024B00205C
:10060000C3F80808704700BF38220020212838B5F9
:100610000C4605D022282DD0202813D0002038BD2C
:100620000029FBD0072AF9D1194BD3F8200993F8F8
:10063000241993F8252993F82639206021716271D5
:10064000A371EBE70029E9D0072AE7D1104DD5F8CF
:100650001C3913B109680020984720682179627914
:10066000A379C5F8200985F8241985F8252985F886
:100670002639D3E70029D1D0022ACFD1044BD3F8B1
:100680001839002BCAD0098800209847C6E700BF58
:100690003822002010B4124CD4E900329A1AC2F366
:1006A0000A020A44B2F5006F13D8B1B101444A1EE0
:1006B000013810F801CFE118824203F1010381F8FB
:1006C00008C0C3F30A03F4D1236000205DF8044B93
:1006D000704702205DF8044B70470846F6E700BFFC
:1006E0003822002010B5812104466DF015FB20460C
:1006F00001216DF011FB204682216DF00DFBFFF70B
:100700007DFF002010BD00BFC169026910B4002345
:1007100040F20114A0F844410B60D169846D21F0CE
:1007200002014FF0010CD161A0F89CC32360D16994
:10073000044821F4003180F827395DF8044BD16179
:100740001846704738220020202301480B8070474C
:1007500060000020122301480B80704780000020B9
:10076000042301480B807047940000200A4608B516
:10077000054920B90548FFF795FE034808BD044820
:10078000FFF790FE004808BD602B002044130808C6
:100790005C13080808B5044B04480A461946FFF7DD
:1007A00081FE084608BD00BF602B002074130808B6
:1007B0002048D0F8E837D0F8EC2730B59B184FF038
:1007C0001A040C8001D11C4830BD1B4AD0F8EA172E
:1007D0004FF0000E10467546B3F1204F4FEA137CE0
:1007E0000CF130040EF1020E2ABF0CF1370C8470AC
:1007F00080F802C0BEF1100FC5704FEA031300F17C
:100800000200E9D100200446B1F1204F4FEA1173F4
:1008100003F1300C00F102002ABF373382F812C016
:1008200093740828D4744FEA011102F10202EBD14B
:10083000014830BD00F0FF1F9800002008B5044BB0
:1008400004480A461946FFF72DFE084608BD00BFBA
:10085000602B00208813080808B5044B04480A469A
:100860001946FFF71FFE084608BD00BF602B002099
:1008700094130808034BD3F85C2CB3F8603C138343
:1008800000207047382200204FF40070034B1060A6
:10089000D3F8803C0B600020704700BF3822002056
:1008A00000207047012070470120704700207047EA
:1008B00010B51C6994420DD396468A188C46944212
:1008C000996938BFA4EB0E0C71446246BDE8104034
:1008D00072F048BC10BD00BF704700BF704700BF3A
:1008E000D0ED007AD0ED036A30EE677AE6EE877AD3
:1008F000B0EE670AC0ED007A704700BFD0ED017A14
:10090000F5EE407AF1EE10FA09D1DFED0E7A60EEE5
:10091000A70AB7EE007AC7EE207AC0ED017A31EE71
:10092000277AD0ED007A80ED021AC1EE076A30EE28
:10093000677AC0ED036AE6EE877AB0EE670AC0ED2B
:10094000007A7047DB0FC94090ED017AD0ED036A61
:10095000D0ED027A30EE470AA6EE807A90ED000ADA
:1009600080ED017A37EE676AE6EE867A37EEC07A76
:10097000C0ED027AA6EE870A80ED000A704700BF3C
:10098000D0ED056AD0ED017A90ED007A90ED066A1F
:10099000D0ED025A90ED035A80ED050A66EEA77A73
:1009A000C0ED066AE7EE007A90ED077AE5EE867A0A
:1009B00090ED086AD0ED045A80ED087AE5EE477AAA
:1009C000E5EEC67AB0EE670AC0ED077A704700BF61
:1009D000D0ED057A90ED006A90ED037AD0ED025AE1
:1009E000E6EE007AF0EE406AB0EE670A90ED016A3A
:1009F000D0ED047A27EE407A67EEC07AA6EE267A2A
:100A0000E5EEA67A90ED066AC0ED067A36EE077A34
:100A100080ED057A704700BF03685A1C02601970A8
:100A2000704700BF03685A1C02601970704700BF0E
:100A3000024BD3F8B00C03681B681847382200201B
:100A4000007970470079C0F3401070470079400981
:100A5000704700BF90F83C20034602F0FF0012B13F
:100A6000002283F83C2070472DE9F84346697EB99F
:100A7000D0F80080C8F30D0904460F46B9F1000F05
:100A800026D03F68FFF74AFC092804D06FF0010622
:100A90003046BDE8F8834A4D2B6923F440732B613F
:100AA0002B6943F400732B612B6943F001032B6125
:100AB000C8F80070FFF732FC2B69092823F0010306
:100AC0002B61E3D12368043323603046BDE8F8830B
:100AD0003C4B98452AD303F58043984524D303F52E
:100AE0008043984554D3384B984554D903F5803307
:100AF000984553D903F50033984552D903F500338F
:100B0000984551D903F5003398453ED903F5003394
:100B100098454CD903F5802398454BD9B8F1016F1E
:100B20004BD305200DF050F94FF00809FFF7F6FB05
:100B3000092804D04FF0FF363046BDE8F883204D39
:100B40002B6923F440732B612B6943F400732B61F1
:100B50002B6923F0F8032B612B6943EA090343F067
:100B600002032B612B6943F480332B61FFF7D6FB23
:100B70002B6923F002032B612B69092823F0F8036A
:100B80002B61D7D1D4F800807BE74FF03809CDE74F
:100B90004FF01009CAE74FF01809C7E74FF02009D6
:100BA000C4E74FF02809C1E74FF03009BEE74FF026
:100BB0004009BBE74FF04809B8E74FF05809B5E7DF
:100BC000003C024000400008FFFF00082DE9F04112
:100BD0000446D0E90030134483421DD88E188E425B
:100BE00017D00D4604F10C08002701E0AE4210D0EA
:100BF00023695A1C2261234415F8010B1873042A37
:100C0000F4D141462046FFF72FFFAE42C4E90470FD
:100C1000EED16069BDE8F0814FF0FF30FAE700BF28
:100C20002DE9F0411E4E96F8B43C002BFBD199B350
:100C3000014400F1FF384F1ED6F8B83CD6F8BC2C62
:100C40000133C3F30A039A4216D10CF03DFA04466D
:100C50000D460CF039FA031B61EB0501B3F57A7F01
:100C600071F10003F5D3D6F8B83CD6F8BC2C0133AB
:100C7000C3F30A039342E8D0D6F8B82CD6F8B83CB0
:100C800018F8011F32440133C3F30A03B84582F850
:100C9000C01CC6F8B83CCFD10020BDE8F08100BF31
:100CA000382200200A4B10B5D3F8084804B910BD0B
:100CB000D3F80838052BFAD1064C002A0846D4F898
:100CC000C8331146F3DDFFF7ABFFD4F8C83310BDCE
:100CD000382200203033002090F84820531C024472
:100CE000DBB280F8483082F8341090F849200AB11D
:100CF000132B03D9002280F8482003B970470A4A11
:100D0000D2F808180029F9D0D2F80828052AF5D118
:100D100010B5064C19463430D4F8C833FFF780FFBD
:100D2000D4F8C83310BD00BF382200203033002073
:100D300090F848100023A0F8483001B97047094BDB
:100D4000D3F80828002AF9D0D3F80838052BF5D1B4
:100D500010B5054C3430D4F8C833FFF761FFD4F830
:100D6000C83310BD38220020303300202DE9F04771
:100D70005D4E1F4606EB80039C68002C00F0AD80A2
:100D800004F13E03A36104F59F73E3614FF48073A4
:100D9000C4E904332836236866600546E16094F8A8
:100DA0003D00A363904609F037FA814694F8440267
:100DB00094F83CA0261D00284FD194F8450268BB4A
:100DC000D4F8403283BB390734D418F0020F60D115
:100DD00018F0010F44D194F9472294F84712D4F83F
:100DE0004832002A10DB41481B018418DBB284F82A
:100DF00000335209012301F01F0103FA01F140F809
:100E000022103046BDE8F087394A01F00F010A444C
:100E10001B01DBB213763046BDE8F0876AF072FF43
:100E2000D4F84032002BCED0324A116B0B43390735
:100E30001363CAD50135EDB2B9F1000FCBD040F242
:100E40000673FA0689F80850A9F8063036D4BB06AE
:100E500094F8462245D4322133E06AF053FFACE7E0
:100E6000504609F0D9F90135EDB20028B3D040F26F
:100E700006620572C28094F84622022109F0B0FB96
:100E800094F9472294F84712D4F84832002AAADA93
:100E9000BAE76B1CDBB2B9F1000F99D089F80830C2
:100EA00040F20653A9F8063094F84622484602213B
:100EB00009F096FB18F0010F8DD0D1E794F8462287
:100EC0000221484609F08CFB94F9472294F8471216
:100ED000D4F84832002A86DA96E726463046BDE83E
:100EE000F0871221EDE700BFE464070800E100E0AD
:100EF000FCEC00E0003802402DE9F047038A8489C9
:100F0000A4B21C4082B045D0814688464FF00045CF
:100F100001F14C0701F13406B4FA84F325FA03F227
:100F2000D24391B2A9F8101014401B3BB8F1000F46
:100F30005DD0042B2CD8DFE803F050463B30030093
:100F4000D8F80C30D9F82CA033B19B6823B11FFA24
:100F50008AF108F104009847D8F8243033B19B682F
:100F600023B11FFA8AF108F11C009847D8F83C30E9
:100F70002BB19B681BB11FFA8AF130469847D8F80D
:100F800054302BB19B681BB11FFA8AF13846984741
:100F9000002CC1D102B0BDE8F087D8F80C30D9F8E8
:100FA00034105B6808F104009847002CB4D1F1E7D5
:100FB000D8F82430D9F838105B6808F11C0098473D
:100FC000002CA9D1E6E7D8F83C30D9F83C105B6892
:100FD00030469847002C9FD1DCE7D8F85430D9F838
:100FE00040105B6838469847002C95D1D2E7042B17
:100FF00007D8DFE803F00319140F0A00D9F84030CE
:101000000193019B002C87D1C4E7D9F82C300193C0
:10101000019BF7E7D9F834300193019BF2E7D9F847
:1010200038300193019BEDE7D9F83C300193019BE7
:10103000E8E700BF70B5254C94F8B42C012A0346AC
:1010400003D0022A09D0002070BD214ED6F8CC531F
:101050008DB984F8B45C002070BD002540F2011207
:10106000C0E95455C0E95655A0F8442100F5A271D5
:101070006CF062FFEDE7402D22D823D0D4F8BC1CE1
:10108000144AC3F858510A44C3E954220022C3F851
:101090005C2140F2011203F5A271A3F84421184625
:1010A0006CF04AFFD4F8BC3CD6F8CC232B44C3F3F5
:1010B0000A03521BC4F8BC3CC6F8CC23002070BD08
:1010C0004025DBE7022284F8B42CD7E73822002041
:1010D00030330020F82E002001EB810138B500EB01
:1010E000C1010E4DB1F88C1304462846FFF7D2FA21
:1010F000E378C4F8A85340210022C4E9EC1201228D
:1011000093422046A4F89C2304F5677108BFC4F8F5
:10111000AC536CF011FF002038BD00BF0037002039
:1011200070B52B4CD4F810340F2B04D05A1CC4F8D3
:101130001024002070BD274D95F8B43C0022C4F85F
:101140001024002BF5D1D5F8BC2CD5F8B83C9A4228
:10115000EFD0D5F8BC2CD5F8B83C9A422CD8D5F8AD
:10116000B86CD5F8BC3CF61A402EC4F8CC6328D92C
:10117000012385F8B43C4026D5F8BC2C164BC0F8AA
:1011800058611344C0E954330023C0F85C3140F285
:101190000113A0F8443100F5A2716CF0CDFED5F832
:1011A000BC3CD4F8CC233344C3F30A03921BC5F8E8
:1011B000BC3CC4F8CC23BCE7D5F8BC6CC6F50066D3
:1011C000D2E70CBF0223012385F8B43CD4E700BF6B
:1011D0003033002038220020F82E002038B5224D70
:1011E000D5F81C3495F834C4044623B195F820345E
:1011F0005CEA030331D00123E06984F8463140F210
:101200000112A4F8442102681849002AA8BFC2F3B9
:1012100080739B0301EA124143F020030B4363F305
:101220001F42BCF1020F026000D038BDE278104BC3
:10123000C4F8A8331F200021C4E9EC01012A4FF0B3
:101240000101A4F89C1308BFC4F8AC3304F567711E
:101250002046BDE838406CF06FBE01216AF02AFBE1
:1012600095F834C4C7E700BF30330020DFBFFFFF6D
:101270004437002070B590F8CF2590F8D13590F81C
:10128000CE5590F8D0C590F8CC1590F8CD6505EB0B
:1012900002250CEB032C90F8D32590F8D23503EB04
:1012A0000223012284B080F8112101F01F029BB2B9
:1012B000ADB21FFA8CFC012A04468DF80810ADF877
:1012C0000A50ADF80CC0ADF80E30C0F840318DF8C2
:1012D00009600AD0022A57D0002A3CD001F08001D0
:1012E0006AF0E8FA002004B070BD90F81231032BC8
:1012F0002BD15FFA8CFCBCF1010F26D8D0F8E43575
:1013000002A99B689847BDF80E30002BEAD1C4E9CA
:101310004A33C4E94C3304214FF4807284F811112C
:10132000A4F81C2104F58E7120466CF097FD636DC6
:10133000C44A1A61E278012AD4D104F2CC545C6127
:101340004FF0802219681A60CCE720466AF07AFADA
:10135000002004B070BD092EF7D801A252F826F083
:101360000B1400081B1500084B1300085515000846
:101370004B130008831500082F1400084B130008B6
:1013800099140008C914000801F0600120295FFACF
:101390008CF334D0012E00F06181032E00F0958192
:1013A000002E9FD190F81221022A00F01B81032AFF
:1013B000CBD11CF0800F40F0A48103EB830300EB42
:1013C000C30393F87633002B00F0A6819E4B0122D5
:1013D000C3F844249D4A0223C4E94E334FF480707D
:1013E000002184F81131A4F81C01C4E94C31C4E98E
:1013F0004A2204F58E7120466CF030FD72E7D0F879
:10140000E43502A99B6898476CE790F81231023BDB
:10141000012B9AD88C4BD0F818210021C3F83C142A
:1014200012B10222C3F83C24894A0223D4E72E0ACF
:10143000022EADF8063000F0CD81032E00F0918130
:10144000012E82D1D0F8EC3580781B680DF10601B1
:101450009847BDF80630002B3FF444AFBDF80E208E
:10146000002A3FF43FAF934228BF13464FF48072E7
:101470000221A4F81C210022C4E94A0084F81111B9
:10148000C4E94E33C4E94C3204F58E712046ADF800
:1014900006306CF0E3FC25E7012B7FF456AF90F8A3
:1014A0001221022A00F04981032A7FF44EAF4FF443
:1014B000807100F588720220A4F81C11C4E94E3333
:1014C00084F81101002190E7EDB25F4E012D86F8FE
:1014D00035543FF63AAF90F81231022B00F02181DB
:1014E000032B7FF432AF002D00F07F8190F81011B4
:1014F000012910D0D0F8E4355B68984796F8351488
:10150000D4F8E43584F810111B6820469847D4F8C5
:10151000E8359B6898470023F9E690F81231023BC2
:10152000012B3FF612AF012D7FF4DCAED0F8E4358D
:1015300000259B68C0F8185102A9984704224FF46F
:101540008073C4E94A55C4E94C5584F81121A4F8C4
:101550001C31E7E6012D00F0CC80022D7FF4C2AEF5
:101560005FFA8CF3002B7FF4BDAE02694FEA1C23B7
:10157000023B5268032B00F25681DFE803F05B4226
:101580006B5F5CEA03037FF4E0AE90F81221032A5C
:101590003FF4DBAE016905F07F0680F8146108684E
:1015A0001A4665F30A1202430A604FF4807204215E
:1015B000C4E94A33C4E94C3384F81111A4F81C215E
:1015C00004F58E7120466CF049FC636D1D4A1A616A
:1015D000E278012A0DD0002E00F01281022384F857
:1015E00012317FE65A063FF47DAE19466AF062F981
:1015F00078E604F2CC525A614FF0802219681A60E2
:10160000E9E7032363F3061201210F4D84F8161155
:101610000421002384F811114FF48071A4F81C11E7
:10162000C4E94A33C4E94C3304F58E712046C5F849
:1016300040247AE6022363F30612E5E7052363F309
:101640000612E1E7180008603033002074370020EC
:101650006C370020042363F30612D5E790F81221BB
:10166000022ABFD0032A7FF470AE002D7FF43AAE79
:1016700013F07F023FF44FAF1CF0800F40F0C480A6
:1016800003EB830100EBC10181F8742381F87653E9
:1016900081F87553282101FB030300EB820293F8C4
:1016A0007713506D03688A1E012A6FF35553D4F8DF
:1016B000E4258CBFC3F30071012161F31C739268B0
:1016C000036002A92046904725E790F81221022ADC
:1016D00088D0032A7FF439AE25B9590602D01946BD
:1016E0006AF0E8F8D4F8E43502A99B6820469847E8
:1016F00011E7D0F8E43502A99B68C0F81851984763
:1017000009E703F07F0303EB830300EBC30393F8C4
:101710001E31002B7FF45AAE454B0022C3F84424FF
:1017200058E6002D3FF40AAF01210322D0F8E4353A
:1017300080F8101180F81221E6E63E4984F8112164
:101740004FF480700022C4E94A11A4F81C01C4E9D6
:101750004E33C4E94C3204F58E7120466CF07EFBAA
:10176000C0E5EDB2052D3FF6F0ADDFE805F02B2327
:101770001B130B03D0F8EC3580789B690DF1060143
:10178000984766E6D0F8EC3580785B690DF1060184
:1017900098475EE6D0F8EC3580781B690DF10601BC
:1017A000984756E6D0F8EC358078DB680DF10601F5
:1017B00098474EE6D0F8EC3580789B680DF106012D
:1017C000984746E6D0F8EC3580785B680DF1060165
:1017D00098473EE6D0F8E43580789B6A0DF1060123
:1017E00098474670C4F8F00533E60222D0F8E43595
:1017F00080F8122180F810515B68294698479DE6D1
:10180000012384F812316DE5282303FB020181F8DE
:101810001C2100EB820281F81E5181F81D61906944
:1018200091F81F113EE7012363F30612ECE600BFB7
:10183000303300206837002010B5044629B990F8ED
:101840001121032A0DD0002010BDD0F8E4359B698A
:10185000002BF8D090F81221032AF4D198470020E9
:1018600010BDD0F890230B46D0F87C138A4213D9D0
:10187000C078521A0128C4F8902336D08A4228BF73
:101880000A4692B2C4E9E22304F55D71A4F8743308
:1018900020466CF0E3FAD6E7D0F8E4351B691BB1BB
:1018A00090F81221032A1ED000234FF480720421E5
:1018B000C4E94A33C4E94C3384F81111A4F81C215B
:1018C00004F58E7120466CF0C9FA636D104A1A61F6
:1018D000E278012AB7D104F2CC545C614FF0802247
:1018E00019681A60AFE79847DEE78A42D4F88003A8
:1018F000A4F8743328BF0A46084492B2C4E9E2232C
:1019000004F55D71C4F88003C4F88403C0E700BF28
:101910001800086038B5044649B990F81131022B17
:1019200011D094F81631012B40D0002038BDD0F8EA
:10193000E4355B69002BF8D090F81221032AF4D12A
:101940009847002038BDD0F83831D0F82421934290
:1019500036D9C178012908BFD0F82811A3EB0203BA
:1019600018BFD0F82821C0F8383108BF52189BB2F0
:101970004FF480710025C0E94C35A0F81C11C0E976
:101980004A2200F58E716CF069FAE378C4F880534E
:10199000012BC4E9E255A4F8745308BFC4F884537A
:1019A00004F55D7120466CF059FABAE72A4B2269BA
:1019B000D3F840145160002384F81631002038BD5C
:1019C000D0F83C31B3FBF2F502FB1535ADB99A42C4
:1019D00013D8D0F8402193420FD24FF48073A0F86F
:1019E0001C31C0E94A55C0E94C5500F58E716CF0C8
:1019F00035FAE378C4F84051C8E7D4F8E435DB6839
:101A00001BB194F81221032A23D0E2780023012A83
:101A10004FF0050108BFC4F88433C4E9E23384F809
:101A20001111C4F88033A4F8743304F55D712046B5
:101A30006CF014FA636D094A1A61E278012A7FF4A6
:101A400070AF04F2CC525A614FF0802219681A60CC
:101A500067E720469847D8E7303300201800086031
:101A6000F8B50B7813F060060D46044620D0202E02
:101A700025D1CE884EB31B0649D5384F68783246FB
:101A80003946FEF7C3FDEB880222002684F81121B7
:101A90004FF48072C4E94E33C4E94A77C4E94C3646
:101AA000A4F81C2104F58E7120466CF0D7F90AE0E9
:101AB0004B780A2B17D00B2B0ED0062B03D12046C8
:101AC00069F0C0FE02263046F8BD02224878114473
:101AD000FEF79CFD3046F8BD8B78002B3AD1204BA9
:101AE000C3F84864EFE7022280F811214FF48072B6
:101AF000A0F81C211B4A0123C0E94E33C0E94A2249
:101B0000C0E94C3600F58E716CF0A8F9DBE7164B96
:101B1000164A4978116003F501620321C0E9E466C1
:101B200080F81111C0F88863C0F88023C078C3F82A
:101B30000C6801284FF00003C4F88C33A4F8743308
:101B400004F55D7108BFC4F8842320466CF086F963
:101B50000026B8E769F076FEB5E700BF482A002006
:101B60003033002078370020382200200000002089
:101B7000002310B51946044640226CF0FFF880217E
:101B80002046002340226CF0F9F8D4F8E835A0781C
:101B9000012284F812215B689847002010BD00BF25
:101BA00010B502230446402281216CF0E7F820465C
:101BB0000223402201216CF0E1F820460323082291
:101BC00082216CF0DBF80E4B0222A3F84C20FEF7CA
:101BD00009FDE2780B4BC4F8A83340200021C4E98A
:101BE000EC01012A4FF00101A4F89C13204604F5F2
:101BF000677108BFC4F8AC336CF09EF9002010BDCB
:101C0000000000200037002070B5812182B004461A
:101C1000314E6CF081F8012120466CF07DF80025F2
:101C2000022340228121204686F827596CF0A6F82D
:101C300001210223402220466CF0A0F8274B86F8B1
:101C40002759D3F84C2483F8345412682846904717
:101C50000095009BE16843F010030093009B0B612B
:101C60000A691F4B009203E00A690092013B02D00F
:101C7000009AD006F8D400230193019B43F020037F
:101C80000193019A164B012060F38A120192019A86
:101C90000A610A69019203E00A690192013B02D0DC
:101CA000019A9206F8D4E2780E4BC4F8A8330021CA
:101CB0001F20C4E9EC01012A4FF00101A4F89C1394
:101CC00004F5677105D020466CF036F9002002B0AB
:101CD00070BDC4F8AC33F6E7382200203033002062
:101CE000400D0300443700202DE9F047089F884647
:101CF00015460021202204461E4673F0D3FB4FB147
:101D00003B68E3811B0C23827B687A89E3821B0C8E
:101D10006282238340466CF0DDFFEB0619D4431E3C
:101D2000B8B108EB000701E0013B12D317F801CD71
:101D3000BCF12E0FF8D1C01A421E032AA8BF0322FD
:101D4000082B03F1010AA8BF08239146C2441A4692
:101D500006E008280246C246A8BF08224FF0000944
:101D60004FF0203341462360636004F108072046AA
:101D700071F0F8F9174B23815146BB704A4638463B
:101D800071F0F0F9611EE31D11F801CFACF1610EA5
:101D9000BEF1190F9CBFACF1200C81F800C08B4242
:101DA000F2D1384604F10B0110F8013BA3F16102B6
:101DB000192A9CBF203B00F8013C8842F4D118232B
:101DC0002373330CA382E572099B6683E361BDE84C
:101DD000F08700BF202020002DE9F04FDFF8949419
:101DE000D9F85C0CB9F8604C448387B0002B00F044
:101DF000DE8001F5FE781344DFF87CB403931646C9
:101E000001F12007C24621E0002E64D0D9F88C3CB5
:101E1000B34200F0D180D9F8883CB34200F004818D
:101E2000D9F8903CD9F8941CB3424BD8B14200F297
:101E30009E81711A204669F08BFC039B01369E42FD
:101E400007F500770AF5007A00F0AD80D9F8985CC4
:101E5000B542A7F12004D7D8751BD9F8A88C05F096
:101E60000702EB080492D8F830200233934203D3E0
:101E7000D8F8382093420BD941461846059369F0AB
:101E800037FC059B8046002800F09181C9F8A80C1A
:101E900098F80420002A40F03981D8F82850002D05
:101EA00000F07E81D8F830209B1A049A02EBC3031D
:101EB000D8F80C20204602EB43224FF40071434631
:101EC000A847BAE7B142B4D920464FF400720021C6
:101ED00073F0E8FAB1E74FF400723146204673F030
:101EE000E1FA802387F89E310C2387F8A231D9F8D4
:101EF000883CD74AD9F8801CC4F8C6319342C4F84C
:101F0000CA1100F33981D34AD34C82FB03021A442D
:101F1000D817C0EB621284FB0254D04D85FB03C579
:101F2000C0EB2530C2EB821587F8A1015B1B801046
:101F300020F03F0001330343144487F8A031D31746
:101F4000C3EBE4142244C24B87F89F214A1E9A42F5
:101F500000F31E81BF4BC04883FB02311144D317ED
:101F6000C3EB611180FB0140BC4C84FB0254C3EB0A
:101F70002433C1EB811487F8A531121B9B1023F089
:101F80003F0301321343084487F8A431CB17C3EB56
:101F9000E010014487F8A311552387F8DE31AA2306
:101FA00087F8DF3149E7D9F85C0CB9F8604C048355
:101FB000002007B0BDE8F08F4FF0FF3384F8EC311C
:101FC00084F8ED3184F8EE3184F8EF31D9F8A03C93
:101FD000C4F8E8315223237063706123A37084F83E
:101FE000E73141230025E37084F8E631722384F859
:101FF000E43184F8E5314FF4F0722946A7F11C0072
:1020000073F050FA5523C7F8D051C7F8D451C7F828
:10201000D85184F8FE316FF0550384F8FC5184F8F0
:10202000FD5184F8FF3108E700214FF4007220468B
:1020300073F038FA8A4A03CA47F81D0CEB2007F8F8
:10204000200C582007F81F0C902047F8191C07F89F
:102050001E0C002302220821F820E372227307F8E5
:10206000131CA273E37307F8102C07F80B0CD9F8B4
:10207000880C84F82C20D9F8802C6376121A2262FE
:10208000D9F8900CD9F8942CE376121A3F202076D8
:102090004FF0FF30A0763E20207701206377A377B2
:1020A000E37784F82D3084F82E3084F82F30626284
:1020B00084F8300084F8313087F82610802187F8C2
:1020C0002010292187F82210942187F823100E214F
:1020D00087F824100D21634A87F82510552187F8C9
:1020E000DE11AA2187F8DF1103CA5F4BC7F827006A
:1020F000C7F82B1003CB1388A7F82F309378C7F8B5
:102100003200C7F8361087F8313096E64FF4007287
:102110000021204673F0C6F9049B002B4ED1D8F85D
:102120004030002B00F0AA80049AD8F830304F4994
:10213000CDE9002220461122FFF7D6FDD8F8403025
:102140001A6C002A00F0AD80049A1B6BCDE90022C6
:10215000474911223846FFF7C7FDD8F8448007F1F8
:1021600020044FF4E075B8F1000F3FD165E6F11A95
:10217000204669F0EDFA60E6FF2387F89F3187F883
:10218000A13187F8A031324B4A1E9A427FF7E2AE66
:10219000FF2387F8A33187F8A53187F8A431FBE640
:1021A000294620464FF4007273F07CF945E6A7F10A
:1021B000240343F804BF9A45FBD13EE6D8F84030EB
:1021C000049AD8F84480002B0CBF01230223C3EBF0
:1021D00002154346002B3FF430AE013D9B6CF9D114
:1021E00098464FF40075002B3FF427AE2544203469
:1021F000234620354446049698460EE05CF81C1BA6
:10220000236BCDF800C000260196FFF76DFDA46C8E
:1022100008F12008CCB1454517D02379A44604F134
:102220001C0E1122A8F12000002BE7D1627926694B
:10223000236B216842F02102CDE900E6FFF754FD4F
:10224000A46C08F12008002CE5D1049EF5E500BF40
:10225000FF03FB00832008828180808097554541E1
:10226000A4130808B0130808BC130808841A080847
:102270009C1B080838220020DEADBEEF049BD9F875
:10228000841CCDE9003320460822FFF72DFDD8F845
:102290004480B8F1000F3FF4D0AD3C464FF4F075E8
:1022A000A4E7049BCDE9003352E700BF8C461346F8
:1022B00001466246184648F041BE00BF1049114B26
:1022C000D1F8882042F4700210B4C1F888201A684E
:1022D0000D4C002042F001021A6098601A6822F04A
:1022E000847222F480321A605C601A68074C22F40F
:1022F00080221A60D8608C605DF8044B704700BF84
:1023000000ED00E00038024010300024000000081A
:10231000704700BF0148FDF77DBF00BFB800002037
:102320000148FDF777BF00BF040300200148FDF717
:1023300071BF00BF500500200148FDF76BBF00BF13
:102340009C0700200148FDF765BF00BFE809002099
:102350000148FDF75FBF00BF340C0020704700BF8D
:10236000704700BF38B5D0E9004307EE902A1B68DC
:10237000354A20680139934204688DB216D002F5BF
:102380008062934212D002F5705293420ED002F551
:10239000806293420AD002F58062934206D02B4BB2
:1023A000D3F87C3E5B0807EE103A04E0274B03F6B7
:1023B0007C6393ED007ADFED266AB8EE477AF8EE9B
:1023C000677A87EE270A30EE260A6EF0B5F81E4AC5
:1023D00023880138944280B29BB212D002F5806209
:1023E00094420ED0B4F1804F0BD0A2F580329442CB
:1023F00007D002F58062944203D002F580629442D5
:1024000002D123F070039BB2124A944212D002F51B
:10241000806294420ED023F4407302F56C429BB26A
:1024200094422380E56220850AD10023238601237C
:10243000A38238BD2380E56220850123A38238BDB5
:10244000054B9C42F1D0F8E700000140000000205D
:102450000AD7233C001000400004014070B54068DA
:10246000837903F0020213F0040300F0C9804FF0F7
:10247000000E134604247246754690F805C0BCF160
:10248000030F30D8DFE80CF08E5F30020368188C41
:1024900020F480500004000C1884188C9C8820F4D0
:1024A000005000042A43000C40EA0232988B6C4D25
:1024B00020F4E6400004000CAB42A4B240F4C0405B
:1024C00000F0B08005F58065AB4200F0AB809C80E9
:1024D000988319641A849A8B22F400621204120CF5
:1024E00042F400629A8370BD2A4305685C4E288CD2
:1024F00020F480700004000C2884288CB5F804C0F7
:1025000020F400700004000C40EA0222A88B20F0A6
:1025100073000004000CB5421FFA8CFC40F0600010
:1025200073D006F58066B5426FD0A5F804C0A883C5
:10253000E9632A84AB8B23F008031B041B0C43F0D4
:102540000803AB8370BD2A430568454E288C20F0F4
:1025500010000004000C2884288CB5F804C020F07A
:1025600020000004000C40EA0212288B20F4E64010
:102570000004000CB5421FFA8CFC40F4C04061D04E
:1025800006F58066B5425DD0A5F804C02883A9632E
:102590002A842B8B23F400631B041B0C43F400637D
:1025A0002B8370BD00682E4E2A43058C25F0010553
:1025B0002D042D0C0584058CB0F804C025F002050F
:1025C0002D042D0C2A43058B25F073052D042D0CAD
:1025D000B0421FFA8CFC45F0600528D006F58066F5
:1025E000B04224D0A0F804C0058341630284038B69
:1025F00023F008031B041B0C43F00803038370BD86
:102600004FF4807E1C46012537E722F4006242EA3F
:10261000032222F480622CF4405C42EA04224CEA59
:102620000E1C82E724F4804444EA8E144FE74FF6F0
:10263000F37616402CF4407C46EA03024EEA0C0C7A
:102640002243CFE722F0800242EA031222F0400246
:102650002CF4406C42EA04124CEA8E0C94E700BF62
:102660000000014042685379032B0FD8DFE803F0E4
:102670000B08050210684030704710683C30704706
:102680001068383070471068343070470020704749
:1026900070B4EFF31182102383F31288C468466884
:1026A000A5682B6823F001032B603568114B767900
:1026B00033F81660AB899BB223EA0603AB8123692A
:1026C00065681F2B11D9203B202404FA03F3EB602B
:1026D000D3B283F31188C3689B6859601A680124D8
:1026E00022431A60047470BC7047202404FA03F378
:1026F000AB60EDE7E464070803681A7D012A04BFB4
:1027000002221A7593F82C100CBF4FF400720022AD
:10271000012904D1022183F82C1042F4806293F83D
:102720004410012905D093F85C1001290AD072B930
:102730007047022183F8441093F85C10012942F499
:10274000006204D1022183F85C1042F48052416897
:10275000096800234B628B899BB21A438A817047B8
:10276000024B0348D3F85014FEF7C6BB30330020A9
:102770000000014010B5064C0648D4F85014FEF78E
:10278000BBFBD4F870140448BDE81040FEF7B4BB9E
:1027900030330020000001400040014010B5064CDD
:1027A0000648D4F85014FEF7A7FBD4F87414044874
:1027B000BDE81040FEF7A0BB303300200000014010
:1027C0000044014010B5064C0648D4F85014FEF7FA
:1027D00093FBD4F878140448BDE81040FEF78CBB96
:1027E000303300200000014000480140034B4FF00F
:1027F0008040D3F85414FEF77FBB00BF3033002075
:10280000024B0348D3F85814FEF776BB3033002050
:1028100000040040024B0348D3F85C14FEF76CBB85
:102820003033002000080040024B0348D3F8601406
:10283000FEF762BB30330020000C0040024B03481F
:10284000D3F86C14FEF758BB30330020000401406D
:1028500010B5064C0648D4F86C14FEF74DFBD4F8BE
:102860007C140448BDE81040FEF746BB303300201E
:10287000000401400018004010B5064C0648D4F88A
:102880006C14FEF739FBD4F880140448BDE81040FE
:10289000FEF732BB3033002000040140001C004032
:1028A00010B5064C0648D4F86C14FEF725FBD4F896
:1028B00084140448BDE81040FEF71EBB30330020EE
:1028C00000040140002000400348D0F88C3E13B1C2
:1028D00000F5686018477047000000200348D0F8F2
:1028E000AC3E13B100F56A60184770470000002045
:1028F0000348D0F8CC3E13B100F56C601847704720
:10290000000000200348D0F8EC3E13B100F56E60E3
:1029100018477047000000200348D0F80C3F13B15F
:1029200000F5706018477047000000200348D0F899
:102930002C3F13B100F5726018477047000000206B
:102940000348D0F84C3F13B100F574601847704746
:10295000000000200348D0F86C3F13B100F576600A
:1029600018477047000000200348D0F88C3F13B18F
:1029700000F5786018477047000000200348D0F841
:10298000AC3F13B100F57A60184770470000002093
:102990000348D0F8CC3F13B100F57C60184770476E
:1029A000000000200348D0F8EC3F13B100F57E6032
:1029B00018477047000000200248C36803B1184759
:1029C000704700BF001000200248C36A0BB12030DE
:1029D00018477047001000200248C36C0BB140300C
:1029E00018477047001000200248C36E0BB16030DA
:1029F000184770470010002002683649002310B4C1
:102A000022F0010221248842026003604360836057
:102A1000C3600361446138D02F4B98422ED02F4BB6
:102A200098423CD02E4B984240D02E4B984232D008
:102A30002D4B984241D02D4B984246D02C4B98427A
:102A400017D02C4B98423CD02B4B984216D02B4B96
:102A5000984224D02A4B984228D02A4B98421AD028
:102A6000294B984229D0294B98422ED0284B984286
:102A700008D14FF03D5243F8AC2C03E04FF47462A0
:102A800043F8202C5DF8044B7047224B5DF8044B53
:102A90003D229A607047204A43F8642CF2E74FF4D5
:102AA00074125DF8044B43F8382C70474FF0746291
:102AB0005DF8044B43F8502C7047184A43F87C2CBF
:102AC000E0E73D2243F8082CDCE7154A43F8942C54
:102AD000D8E700BF1060024028600240406002401A
:102AE000586002407060024088600240A06002406E
:102AF000B860024010640240286402404064024012
:102B0000586402407064024088640240A06402403D
:102B1000B8640240006002403D000020400F0020E9
:102B200000003D2000222DE9F04713460D684FF0CC
:102B3000010E032604E00133102B02F1020239D00A
:102B40000EFA03FC3CEA0504F5D1076806FA02F424
:102B500027EA040707600F79D0F800A007FA02F906
:102B6000013F49EA0A09012FA046C0F800906FEA28
:102B7000040411D887683C4084604C79876894408D
:102B80003C438460446824EA0C0444608C794768C0
:102B90009C40A4B23C434460C46824EA0804C46076
:102BA000CC79C768944001333C43102BC46002F1D8
:102BB0000202C5D1BDE8F0872DE9F0412348244F3A
:102BC000244E254C82B03822002172F06BFC002587
:102BD00057F825103246002301E054F83320914283
:102BE0002ED001330E2BF8D10020053569F08AF87C
:102BF0002D2DEDD1DFF85880184F08F1B4054FF0B6
:102C0000007698F8040007F007FB08F11408044662
:102C100088B1036803F13F4303F57E0307EB932379
:102C200093F8C80069F06EF8A388019620680093B5
:102C30006946FFF777FFA845E3D102B0BDE8F08110
:102C4000064A02EBC30393F85C00CEE7803700200E
:102C500080100020000001403C650708E46407087C
:102C6000224A936803F00C03042B10B421D0082BE4
:102C700022D01F4B03601D4C1E4AA168C1F30311F3
:102C8000114491F83C10CB404360A168C1F382210C
:102C9000114491F83C1023FA01F18160A1685DF8BC
:102CA000044BC1F342310A4492F83C20D340C36044
:102CB0007047114B0360DEE75368516813F4800FCF
:102CC00001F03F01536814BF0B4A094AB2FBF1F10E
:102CD000064A5268C2F30142C3F38813013201FB72
:102CE00003F35200B3FBF2F30360C4E70038024081
:102CF0000024F400F810002000127A0070B5446B34
:102D00008668A38923F400531B041B0CA3818279DA
:102D10000546407912F0040F14BF4FF4805C4FF069
:102D2000000C110310F0010F4FEA02220CBF002328
:102D3000042302F48062800748BF43F0080342EA9C
:102D40000C021343228A92B201F4005122F4405241
:102D50000A432282A28922F4B05222F00C02120409
:102D6000120C1A43A281A38A23F440731B041B0C88
:102D700084B0A3826846FFF773FF2F4B9C4205D0B7
:102D800003F580639C4201D0029A00E0039AA38974
:102D90002A491B0402EB82024CBF7300B30002EB12
:102DA0008202B2FBF3F3A1FB0302A089520964265D
:102DB000000406FB12334FEA021228D41B013233FF
:102DC000A1FB0313C3F3431313439BB223816A791B
:102DD0006B6BA879960702F00101194A48BF41F0D0
:102DE000020193421BD001079A8A0AD592B242F09F
:102DF00008029A829A8992B242F400529A8104B0EF
:102E000070BD22F008021204120C9A82F2E7DB0075
:102E10003233A1FB0313C3F342131343D5E7CD07AA
:102E2000E1D5084AD2F8A81BB2F8AC2BC4074CBFB6
:102E30000A834A83D7E700BF001001401F85EB518A
:102E400000440040382200202DE9F843394C9DF819
:102E500020509DF82490A0420F4690461E4649D02F
:102E6000354B98424ED0354B984253D0344B984214
:102E70002BD0344B984255D0334B984221D14B46FE
:102E80002A4631460520FDF771FF04460023C4E9B8
:102E90000B78C4E90733C4E909336571A66084F887
:102EA00006902046FFF72AFFEA07616B1AD4AB07AA
:102EB00013D48B899BB243F400538B812046BDE829
:102EC000F88300242046BDE8F8834B462A46314665
:102ED0000320FDF74BFF0446D8E7CB6843F080039F
:102EE000CB60E6E74FF6DF730B80CB6843F020033F
:102EF000CB60DCE74B462A4631460020FDF736FF23
:102F00000446C3E74B462A4631460120FDF72EFF13
:102F10000446BBE74B462A4631460220FDF726FF12
:102F20000446B3E74B462A4631460420FDF71EFF10
:102F30000446ABE700100140004400400048004058
:102F4000004C004000500040001401408160D5E674
:102F50004171D3E62DE9F043DFF8108208EBC00998
:102F600085B00546C70099F8500007F055F90446AA
:102F700099F8510007F050F9064699F8520068F0A8
:102F8000C1FE6B1CDBB2002C00F0AC8040F60C12D2
:102F90002372E280002E00F0C280337240F60C23D0
:102FA0002046F38004223A2107F01AFB042230461F
:102FB0003A2107F015FB08EB0703614ADC6C9442E9
:102FC00000F098805F4B9C4200F09E805E4B9C42DC
:102FD00000F0AB80474497F85320022A5CD0032AC4
:102FE0007ED05A4B5A4E012A18BF1E46A788684603
:102FF000FFF736FE27F03F07029B564AB3FBF6F673
:103000003F04A2FB03233F0C47EA9347A780228893
:1030100022F001021204120C2280B2B2C6F30B0697
:103020009B0C002E59D04FF4967101FB03F34A49D3
:10303000A1FB03139B0901339BB242F4004223849A
:10304000A2832388454A9BB243F00103238023884F
:1030500023F4816323F002031B041B0C4FF4804113
:1030600043F4806323802181238823F080031B04A1
:103070001B0C238023889BB202EB451243F0010313
:1030800023800121002382F8885482F8891482F871
:103090008A3405B0BDE8F083A6886846FFF7E0FDF6
:1030A00026F03F06029A2B4B3604A3FB0213360C84
:1030B00046EA9346A680218821F001010904090C03
:1030C00021809B0C2649013392092384A1FB023203
:1030D0009209042A38BF0422B2E742F00102A2E7B3
:1030E000204E83E7002E3FF466AF337240F60C2388
:1030F000F3805BE71C4B1A6A42F400121A621A6AE8
:1031000022F400121A6265E703F5F0331A6A42F4FA
:1031100080021A621A6A22F480021A625AE70422B2
:1031200020463A2107F05CFA45E703F5EE331A6AC8
:1031300042F400021A621A6A22F400021A6249E793
:103140000054004000580040005C0040804F1200D6
:10315000009F240083DE1B43D34D621030330020D8
:10316000632D3E05C027090000380240F8100020FA
:103170002DE9F047954D90F900108046807805EBD9
:10318000C1060138CC0090B0F16C14282ED8DFE8CD
:1031900010F054012701150057006100A200AA0099
:1031A000CC01BE017D00870046020E02E101C50090
:1031B000D50030003800AB019D015C01888A0C8B82
:1031C00081B2834841EA044130EA010100F02781DD
:1031D000D8E90210521A42F2107163EB00038A42DE
:1031E00073F1000302D3152388F8023010B0BDE854
:1031F000F08798F813000882C8E90223122088F8A3
:103200000200888A0C8B80B240EA0440714C34EA98
:10321000000000F0B68000200E900F9001200F916A
:103220000E900E99002900F01F820F9914310F9112
:103230000F9909684905CBD5142388F80230D5E7E2
:1032400098F8110000F0FE000882C8E9022305206A
:1032500088F80200888A0C8B80B240EA04405E4CF9
:1032600034EA000000F0A4800020009001900120CA
:10327000019100900099002900F002820199143117
:103280000191019909684F05D6D4A1E798F811007A
:1032900040F001000882C8E902230B2088F80200F0
:1032A000888A0C8B80B240EA04404C4C34EA00001F
:1032B0006FD000200490059001200591049004999E
:1032C000002900F0D7810599143105910599096805
:1032D0004D05B1D47CE798F813000882C8E90223B1
:1032E000072088F80200888A0C8B80B240EA0440EC
:1032F000384C34EA00005FD0002002900390012097
:10330000039102900299002900F0C68103991431BB
:103310000391039909684E058ED459E7088820F473
:1033200080600004000C088098F8110000F0FE0096
:103330000882C8E90223102088F80200888A0C8BD2
:1033400080B240EA0440244C34EA000012D000204D
:103350000C900D9001200D910C900C99002900F01B
:1033600095810D9914310D910D99096848053FF526
:1033700063AF2DE798F81330FF2B06D198F8103083
:103380001BB1132388F8023030E7112388F802308C
:103390002CE7D8F81400012800F09481022800F0EE
:1033A0004A820E20098B88F80200C8E902231DE733
:1033B000062388F8023019E7D8F81400002800F036
:1033C0007181082388F8023010E700BFF810002050
:1033D00001000300840007008200070002000300D0
:1033E000088820F400600004000C0880088880B27F
:1033F00040F480600880088880B240F480700880C3
:10340000032088F80200888A0C8B81B2AB4841EA1D
:103410000441C8E9022330EA01037FF4E7AE98F8DB
:103420001230002B40F0D38198F81330FF2B00F0BE
:103430004682042388F80230D8E6098889053FF5DA
:10344000C7AE002388F80230D0E62C4494F8500030
:1034500006F0E2FE064694F8510006F0DDFE984ABA
:10346000B2F8E83401339BB28246A2F8E83416B1D0
:103470003368B2881A83BAF1000F04D0DAF800304A
:10348000BAF804201A831121304604F0B3FF112149
:10349000504604F0AFFF4FF0090965272EB133689D
:1034A000B28819690A4240F02881013F00F0228168
:1034B00009F00AFE04460D4609F006FE001B61EB0A
:1034C0000501052871F10003F6D3E7E7088880B20B
:1034D00040F4007008804FF6FF3088820121C8E96F
:1034E000022388F8021081E6D8F81400002800F0C2
:1034F0007281D8F8184014F8016B0E820138122539
:10350000C8E90504C8E9022388F802506EE6888AF3
:103510000C8B81B2694841EA044130EA01017FF431
:1035200057AE0A2388F8023060E6088880B240F47B
:1035300080700880092088F80200888A0C8B81B28C
:103540005E4841EA0441C8E9022330EA01037FF4FE
:103550004DAEE6E7002401250A940B940B910A95E1
:103560000A98002800F04A810B9814300B900B98B1
:10357000006846077FF52CAED8F81400032800F049
:103580007281022800F24681088820F480600004DD
:10359000000C0880088880B240F400700880098A16
:1035A00088F81C40C8E9022388F802501EE6002073
:1035B000012408900990099108940898002800F0C7
:1035C00017810998143009900998006847077FF51A
:1035D000FFADEFF31185102080F31288088880B2C8
:1035E00040F400700880D8F818000E8A471CC8F80C
:1035F0001870EDB2067085F311880D8AD8F818108E
:103600006FF001004E1CC8F818600D70C8E9022365
:10361000C8F8140088F81C4088F80240E6E500204D
:1036200006900790012007910690069C002C00F060
:10363000EB80079C14340794079C246864067FF58C
:10364000C7AD0C8AD8F818104D1CC8F818500C706B
:10365000D8F8141088F81C000139C8E90223C8F80A
:10366000141088F80200C1E50F9918310F910F99D5
:103670000968ADE505991831059105990968A7E52F
:1036800001991831019101990968A1E50D99183145
:103690000D910D9909689BE50399183103910399E0
:1036A000096895E5088880B240F40070088001211F
:1036B000C8E9022388F8021098E500BF0100030062
:1036C00030330020088820F480600004000C08805B
:1036D000EFF31184102080F31288088B088880B2E1
:1036E00040F40070E4B2088084F311880C2188F85B
:1036F00002105AE616B13368B2885A8309F0E4FC26
:1037000004460D4609F0E0FC031B61EB0501052BA7
:1037100071F10003F6D316B13368B2881A8309F049
:10372000D3FC04460D4609F0CFFC031B61EB0501F9
:10373000052B71F10003F6D3B9F101097FF4ADAEA9
:1037400016B13368B2885A8309F0BEFC04460D46B0
:1037500009F0BAFC031B61EB0501052B71F10003B5
:10376000F6D3BAF1000F04D0DAF80030BAF804202A
:103770005A8309F0A9FC04460D4609F0A5FC031B79
:1037800061EB0501052B71F10003F6D316B1336827
:10379000B2881A8309F098FC04460D4609F094FC9F
:1037A000031B61EB0502052B72F10003F6D3BAF19E
:1037B000000F04D0DAF80030BAF804201A8398F920
:1037C0000000441C3FF43DAEFFF7C4FB39E60F2375
:1037D00088F802300AE5088880B240F4007008805A
:1037E0000121C8E9022388F81C1088F80210FDE4C2
:1037F00009991831099109990968E9E40B99183177
:103800000B910B990968E3E407991831079107991F
:103810000968DDE4D8F81800098A441CC8F8184083
:103820000170D8F81410C8F808200139C8F814102D
:10383000C8F80C30DAE4088880B240F400600880F0
:10384000EFF31184102080F31288088B088820F48D
:1038500080600004000CE4B2088084F311880D211C
:1038600088F80210A1E5088820F480600004000CAC
:103870000880EFF31184102080F31288D8F8180024
:103880000D8A461CC8F818600570088880B240F49C
:103890000070E4B2088084F31188D8F81800098A0F
:1038A000441CC8F818400170D8F814100C200239D4
:1038B000C8E90223C8F8141088F8020096E498F8C2
:1038C0001030002B3FF4B5AD2BE600BF38B5184DD6
:1038D0009DF814E005EB40144FEA401C94F889046D
:1038E00000B938BD490084F89B24C4F89C3484F89E
:1038F00099140023049984F898E4022205F591654F
:1039000084F89A34C4F8A01484F8A43484F88A247F
:10391000654409F0D9FB02460B462846FFF728FC10
:1039200094F88A34002BF4D194F8A40438BD00BF75
:1039300030330020F0B5044683B00D461746061D0F
:1039400020680379012B18D0022B13D18368DB0781
:1039500032464FF0FF015CBF3246FF2105F064FDA7
:1039600030B115B12379DB07EAD40FB123793B706D
:1039700003B0F0BD002003B0F0BD8268417C90F937
:10398000100002F00102CDE90062FF22FFF79EFF66
:10399000E6E700BF30B5044683B0051D2068037913
:1039A000012B14D0022B0FD18368DB072A464FF07E
:1039B000FF015CBF2A46FF2105F036FD10B12379D7
:1039C000DB07EBD403B030BD002003B030BD82680C
:1039D000417C90F9100002F00102CDE90052FF2273
:1039E000FFF774FFEAE700BF30B50246044652F81D
:1039F000040B0379012B83B00ED0022B09D1FF21D8
:103A000005F012FD18B12079C04300F0010003B0A9
:103A100030BD002003B030BD8568417C90F91000B6
:103A2000009205F001050195FF22FFF74FFFE9E73E
:103A300030B5B42283B00446FF21006804F0D0FD05
:103A400010B9002003B030BD20680379012B04F1C8
:103A5000040514D0022BF4D18368DB072A464FF00B
:103A6000FF015CBF2A46FF2105F0DEFC0028E8D0FC
:103A70002379DB07E6D520680379012BEAD1826838
:103A8000417C90F9100002F00102CDE90052FF22C2
:103A9000FFF71CFFEAE700BF30B50A4683B00446D3
:103AA000A521006804F09CFD10B9002003B030BDD2
:103AB00020680379012B04F1040514D0022BF4D102
:103AC0008368DB072A464FF0FF015CBF2A46FF21CF
:103AD00005F0AAFC0028E8D02379DB07E6D52068AA
:103AE0000379012BEAD18268417C90F9100002F041
:103AF0000102CDE90052FF22FFF7E8FEEAE700BF2E
:103B000070B582B0CDE900230446FFF791FF10B9EC
:103B1000002002B070BD20685522A52104F060FD90
:103B20000028F5D0251D20682A46FF2105F0D2FC8B
:103B30000028EDD02379DB07F5D40DF1FF350DF129
:103B4000070615F8011F2046FFF7A6FF0028DFD063
:103B5000B542F6D1DDE700BF002A37D0F0B5013A13
:103B600083B004464E1E51FA82F7051D16F8012F48
:103B70002068A52104F034FD90B9002003B0F0BD09
:103B80008268417C90F9100002F00102CDE90052F8
:103B9000FF22FFF79BFE0028EFD02379DB0710D52B
:103BA00020680379012BEBD0022BE6D18368DB0779
:103BB0002A464FF0FF015CBF2A46FF2105F034FC86
:103BC000E9E7B742D2D1012003B0F0BD0120704730
:103BD00070B5962282B004460E460068FF2104F0BC
:103BE000FFFC10B9002002B070BD251D20680379CC
:103BF000012B1FD0022BF5D18368DB072A464FF03B
:103C0000FF015CBF2A46FF2105F00EFC0028E9D029
:103C10002379DB07EAD4E1222068114604F0E0FCB6
:103C20000028DFD020683246FF2102B0BDE8704096
:103C300005F050BC8268417C90F9100002F001024E
:103C4000CDE90052FF22FFF741FEDFE7002A46D010
:103C5000F0B5013A4F1C83B004460E4657FA82F77E
:103C6000051D20689622FF2104F0BAFC90B90020BF
:103C700003B0F0BD8268417C90F9100002F00102AF
:103C8000CDE90052FF22FFF721FE0028EFD0237973
:103C9000DB0710D520680379012BEBD0022BE6D18E
:103CA0008368DB072A464FF0FF015CBF2A46FF21ED
:103CB00005F0BAFBE9E7E1222068114604F090FC28
:103CC0000028D4D020683246FF2105F003FC0028EC
:103CD000CDD00136BE42C4D1012003B0F0BD0120D9
:103CE000704700BF70B505460B460446164655F8AA
:103CF000040B82B087211A4604F072FC2068037915
:103D0000012B18D0022B13D18368DB072A464FF012
:103D1000FF015CBF2A46FF2105F086FB30B1237905
:103D2000DA07EBD416B1C3F34013337002B070BDA1
:103D3000002002B070BD8268417C90F9100002F052
:103D40000102CDE90052FF22FFF7C0FDE6E700BF08
:103D500070B5782182B0044616460068002204F04F
:103D60003FFC10B9002002B070BD251D206803790A
:103D7000012B14D0022BF5D18368DB072A464FF0C4
:103D8000FF015CBF2A46FF2105F04EFB0028E9D069
:103D90002379DA07EAD45B09337002B070BD826818
:103DA000417C90F9100002F00102CDE90052FF229F
:103DB000FFF78CFDEAE700BF30B5CC2283B00446A4
:103DC000A521006804F00CFC10B9002003B030BD40
:103DD00020680379012B04F1040514D0022BF4D1DF
:103DE0008368DB072A464FF0FF015CBF2A46FF21AC
:103DF00005F01AFB0028E8D02379DB07E6D5206818
:103E00000379012BEAD18268417C90F9100002F01D
:103E10000102CDE90052FF22FFF758FDEAE700BF9B
:103E200030B5B42283B00446FF21006804F0D8FB0B
:103E300010B9002003B030BD251D20680379012B87
:103E400022D0022BF5D18368DB072A464FF0FF0111
:103E50005CBF2A46FF2105F0E7FA0028E9D0237964
:103E6000DA07EAD4CC212046FFF716FE0028E0D07E
:103E700002E02379DB07DDD520682A46FF2105F023
:103E800029FB0028F5D1D4E78268417C90F9100025
:103E900002F00102CDE90052FF22FFF717FDDCE737
:103EA0002DE9F04F89B00446CDE90623002004F146
:103EB000040B0490029103905D462046049FFFF797
:103EC000B7FD069BFE0003EBC70B20B90AE0237980
:103ED00013F0010A0CD020682A46FF2105F0FAFAF7
:103EE0000028F4D1079B049A1A7009B0BDE8F08F3E
:103EF0009B07F7D5F0212046FFF7CEFD0028F1D033
:103F0000069B083E334401270593D0463E46029B5C
:103F1000002B4AD0082E48D806F1FF3943FA09F998
:103F200009F0010920684FEAC912782104F058FB12
:103F30000028D7D020680379012B47D0022B43D12A
:103F40008368DB072A464FF0FF015CBF2A46FF214A
:103F500005F06AFA0028C5D0237913F00102E9D1EF
:103F600003F0600160294FEAD31C51D0029919B1C6
:103F7000082E01D8E145B5D1BCF1000F3AD01BF8AD
:103F800008303B430BF808307F00013617F0FF077D
:103F9000F6B2BCD108F101085FFA88F8B8F1080F51
:103FA00036D0029B0127002BB4D1049BD3B1039BD5
:103FB000B34217D9059B13F808301F4214BF4FF0C6
:103FC00001094FF00009ADE700208BE78268417CD2
:103FD00090F9100002F00102CDE90052FF22FFF734
:103FE00075FCB7E7039BA3EB0609B9FA89F94FEA19
:103FF000591997E71BF8081021EA07010BF8081078
:10400000990941EA531313F0010F08BFB246BBE709
:10401000402E06D8079B049A1B7893423FF64DAF7B
:1040200060E79BF807C00BF1FF370BF1060B17F8A1
:10403000011F082382EA010616F0010F4FEA52021F
:1040400018BF82F08C0203F1FF3318BFD2B213F015
:10405000FF034FEA5101EDD1BB45E8D19445D9D1D9
:10406000049B0133DBB20493BAF1000F3FF43AAF83
:10407000CDF80CA0CEE700BF10B500680379012B86
:1040800084B00C4618D0022B13D1836813F0010FB3
:1040900014BF2221A221032303AA04F07DFC30B126
:1040A000BDF90D3003EB83031B12E633238004B00C
:1040B00010BD002004B010BD8368417C90F9100051
:1040C00003F00103019303AB009322220323FFF7C4
:1040D000FDFB0028E4D1EAE738B5184D9DF814E05F
:1040E00005EB40144FEA401C94F8890400B938BD30
:1040F00084F89B24C4F89C3401220023490005F570
:10410000916584F89A2484F8A434049A84F898E495
:10411000022384F89914C4F8A02484F88A346544EE
:1041200008F0D2FF02460B462846FFF721F894F824
:104130008A34002BF4D194F8A40438BD3033002025
:1041400010B504682379012B84B011D0022B0CD157
:10415000A368DB074FF0F0024CBFFF217F21204610
:1041600004B0BDE8104004F0E7B9002004B010BD71
:10417000A268617C94F9100002F0010201920DF135
:104180000F020092F024FF228DF80F40FFF7A4FFEA
:1041900004B010BD70B505682B79012B84B00446BE
:1041A0000E4616D0022B11D1AB68E122DB074CBFC3
:1041B00011466121284604F0BFF938B12068324623
:1041C000FF2104B0BDE8704005F084B9002004B0C0
:1041D00070BDAA68697C95F9100002F001020DF12A
:1041E0000F0501920095E1228DF80F20FFF774FF73
:1041F000E3E700BF70B505682B79012B84B0044656
:104200000E4617D0022B12D1AB68DB074FF0C3026A
:104210004CBFE1216121284604F08EF938B12068B5
:104220003246FF2104B0BDE8704005F053B90020CC
:1042300004B070BDAA6895F91000697C02F0010213
:1042400001920DF10F020092C3228DF80F20E1229E
:10425000FFF742FFE2E700BF10B504682379CA43C5
:1042600041EA0211012B84B0CAB20FD0022B0AD14D
:10427000A368DB074CBFD2215221204604B0BDE821
:10428000104004F059B9002004B010BD8DF80F2083
:10429000A268617C94F9100002F001020DF10F0494
:1042A000CDE90042D222FFF717FF04B010BD00BFD6
:1042B00070B505682B79012B84B004460E461AD0E0
:1042C000022B15D1AB68DB074FF0F0024CBFE121A8
:1042D0006121284604F030F950B12246FF2152F8FE
:1042E000040B05F0F7F818B12379337004B070BDF2
:1042F000002004B070BDAA6895F91000697C02F036
:10430000010201920DF10F020092F0228DF80F20B0
:10431000E122FFF7E1FEDFE710B504682379012B06
:1043200084B011D0022B0CD1A368DB074FF0B4028C
:104330004CBFFF217F21204604B0BDE8104004F0AF
:10434000FBB8002004B010BDA268617C94F9100095
:1043500002F0010201920DF10F020092B424FF223B
:104360008DF80F40FFF7B8FE04B010BD10B504681B
:104370002379012B84B010D0022B0BD1A368DB076B
:104380000A4620464CBFA521252104B0BDE81040B7
:1043900004F0D2B8002004B010BDA26894F9100057
:1043A0008DF80F1002F00102617C0DF10F04CDE9D0
:1043B0000042A522FFF790FE04B010BD10B50468BE
:1043C0002379012B84B011D0022B0CD1A368DB0719
:1043D0004FF096024CBFFF217F21204604B0BDE87C
:1043E000104004F0A9B8002004B010BDA268617CA0
:1043F00094F9100002F0010201920DF10F020092F7
:104400009624FF228DF80F40FFF766FE04B010BD22
:1044100010B504682379012B84B010D0022B0BD186
:10442000A368DB070A4620464CBF8721072104B05A
:10443000BDE8104004F080B8002004B010BDA268B0
:1044400094F910008DF80F1002F00102617C0DF15B
:104450000F04CDE900428722FFF73EFE04B010BDF5
:1044600010B504682379C901012B84B0CAB20BD0FE
:10447000022B06D17821204604B0BDE8104004F09C
:104480005BB8002004B010BD8DF80F20A268617CDD
:1044900094F9100002F001020DF10F04CDE9004281
:1044A0007822FFF719FE04B010BD00BF10B50468F4
:1044B0002379012B84B011D0022B0CD1A368DB0728
:1044C0004FF055024CBFA5212521204604B0BDE880
:1044D000104004F031B8002004B010BDA268617C27
:1044E00094F9100002F0010201920DF10F02009206
:1044F0005524A5228DF80F40FFF7EEFD04B010BD46
:10450000F0B587B00023834A00930193136843F406
:104510008033136003E0009BB3F5A04F09D013680C
:1045200003F400330193009B01330093019B002BA4
:10453000F1D0784B1B6813F4003318BF01230193AB
:10454000019B012B01D000BFFDE7724B72491A6C31
:10455000724842F080521A640A6842F440420A608B
:104560009A689A609A6842F400429A609A6842F4A3
:10457000A0529A6058601A6842F080721A601A68F5
:104580009201FCD5664A40F205711160996821F0EC
:1045900003019960996841F00201A2F58062996077
:1045A000936803F00C03082BFAD1936803F00C0313
:1045B000042B00F08D80082B00F08F80594D5A4B52
:1045C000C5F87C3E534B59499868D5F87C2E584C19
:1045D000C0F303100144574891F86410CA4056498B
:1045E000C5F87C2EE160554A596FA260596B544A58
:1045F00021F080015963596F41F080715967196B3F
:104600000A431A635A6B5A639A6B9A631A6C4D4940
:104610000A431A64596C4C4A0A435A6402A948F284
:10462000FF73002602934FF6FF770396FEF77AFAA0
:1046300000F580600297FEF775FA00F5806002973A
:10464000FEF770FA00F58060FEF76CFA00F5806006
:10465000FEF768FA00F58060FEF764FA00F5806006
:10466000FEF760FA00F58060FEF75CFA00F5806006
:10467000FEF758FA0846FEF7F3FAD4F8FC30029A2F
:104680003249334843F08073C4F8FC30314BC3F8EF
:10469000B01F5E60196841F001011960D5F87C3ED9
:1046A0004FF47A71B3FBF1F3013BB3F1807F2A49F8
:1046B000B2FBF1F2C0F8EC2408D24FF0E022F02176
:1046C0005361072384F823109661136107B0F0BD8E
:1046D000144D224BC5F87C3E74E753685168114D68
:1046E00013F4800F01F03F01536814BF1B4A0E4AB8
:1046F000B2FBF1F1074A5268C2F30142C3F38813D7
:10470000013201FB03F35200B3FBF2F3C5F87C3E28
:1047100058E700BF003802400070004008544007CE
:10472000003C0240000000200024F400F8100020AB
:1047300000ED00E0000002400003FA050000000860
:10474000FF916700FFC9FE103357070055CEACC577
:1047500030330020001000E040420F0000127A00C9
:1047600082B0064B002201920193019B03EB800073
:104770000190019B196002B0704700BF50280040B3
:1047800010B51C2005F048FD1121044603F032FE4F
:104790004CB12368A2885A83C82008F0C3FC236860
:1047A000A2881A8310BDBDE81040C82008F0BABC2A
:1047B000704700BF704700BF704700BF10B5124C74
:1047C00094F8FA3423B9114B4FF480225A6110BD8A
:1047D0004FF0E022D2F8103D23F00603C2F8103D5E
:1047E000FDF76CFD94F8FA34002BECD0D4F80035CA
:1047F0009B68DB07E7D5D4F8FC25136823F0030199
:1048000061F307031360DEE730330020003C014012
:104810002DE9F04FB34CD4F8FC345A69D2078BB071
:1048200002D50BB0BDE8F08F5A699B6912EA030903
:10483000F7D0C9F3074319F4002F009340F0E1804B
:10484000009B590743D419F0020F5FFA89F603D091
:10485000D4F8FC3402225A61B9F1000FC0F2EE81A3
:1048600019F4006FC9F3072540F04A81330708D5D2
:104870009D4B9E48D3F880309847D4F8FC340822EA
:104880005A61F70600F1C481EE0600F16F81A906B6
:1048900000F1E880009BDA0609D5934B9348D3F8E2
:1048A00090309847D4F8FC344FF480125A61009B42
:1048B0009B06B6D58C4B8D48D3F894309847D4F8E6
:1048C000FC344FF400125A610BB0BDE8F08FD4F8FD
:1048D00000259369D26913401FFA83FABAF1000FD9
:1048E000B1D0DFF81882CDF80C90A8F11805002798
:1048F0001AF0010F78D0FEB2D4F8002504EB86033D
:104900001069D3F80815536B8968F340DB01DBB2FB
:1049100003430B4013F00109D9B240F0AB810A0701
:1049200040F1C781D8F8002008239360994619F018
:10493000800F59D0D5E94CC0D5F82431D8F800E023
:10494000ACEB00018B42DEF8182028BF0B4692B278
:104950000333B2EB930F47D9D4F8002594F8F394BE
:10496000323604EB8603CDE90178674698469446D3
:10497000874237D9D5F82431391A994228BF1946C8
:1049800001F1030BD5F828314FEA9B0BB9F1000F69
:1049900010D18AB203329210D8F8F8640AD048468F
:1049A000013053F8047B37608242F9D1D5E94C706D
:1049B000D5F8283108440B44B842C5F82831C5F869
:1049C0003401DEF818300AD195F81C11012202FAE0
:1049D00001F1DCF8342022EA0102CCF834209BB249
:1049E0009B45C5D3DDE901785FEA5A0A07F1010763
:1049F00008F1040805F128057FF47AAFDDF80C9082
:104A000021E7D4F800359D69DB691D402D0C3FF48A
:104A100017AF04F59E68DFF8D0B004F244560027C3
:104A2000C24608E06D0807F1010706F1040608F127
:104A300028083FF405AFEB07F4D5F9B204EB810386
:104A4000D4F80025D3F844359B6852691340D80741
:104A5000DAB200F13E81930740F1668133680222A9
:104A60009A60DFE7D4F80035D4F808159A6808682A
:104A7000C2F34102022A06BF032262F30A006FF367
:104A80000A0008605A6842F480725A6006A8FEF76D
:104A9000E7F8D4F8FC24D4F80015D368079D6FF329
:104AA0008D23D36088681249C0F34100014491F816
:104AB000D010032900F05E810E490F4801262944D9
:104AC00084F8F26481424FF04006A4F8F46400F2E6
:104AD000AA810E2161F38D234FF40051D3605161FF
:104AE000D8E600BF30330020F81000202038002026
:104AF000E4640708401E1BFF3F420F0038380020C7
:104B000000238DF8133094F802368DF81330B54B2E
:104B1000B548D3F888309847D4F80035D4F8FC2449
:104B2000986894F8FA344FF400615161002B3FF417
:104B30009DAEC2077FF59AAE94F80536012B7FF43F
:104B400095AE9DF81330032B7FF490AED4F8FC356E
:104B5000A6491A6842F001021A601A6842F003027C
:104B60001A600B6943F006030B617FE6D4F8006519
:104B7000D4F8FC147368002723F0010373600597D1
:104B8000059B43F020030593059B67F38A13059368
:104B9000059B0B610B690593BC46954B03E00A69C5
:104BA0000592013B02D0059A9006F8D494F8F124BE
:104BB00052B1904B03EB820EFF2253F8040F826038
:104BC000D86B73458260F8D10B2363F3070763F357
:104BD000070C4FF0FF33B3614FF00113F3617761BE
:104BE000C6F810C0336884486FF30A13336094F832
:104BF000F324D4F84435012A186100F0B4804FF44E
:104C000080534B61774B7848D3F8843098473EE621
:104C1000D4F8FC349A6922F010029A611A6AC2F33D
:104C20004340022802F00F0100F0AF80062800F098
:104C300086809A6942F010029A6125E694F8FA3467
:104C40003BB1D4F8FC25136823F0030161F307039B
:104C50001360D4F80025634B6348D3F88C10536875
:104C600023F0010353608847D4F8FC344FF000422E
:104C70005A61F5E5516BD8F800005A4B4FF0010C22
:104C80000CFA07FC21EA0C01516301229B6F826040
:104C900031465548984794F8F334012B00F0B08022
:104CA00019F0020F3FF443AED8F8003002229A60A8
:104CB0009AE6CB0604D5D8F8003010229A6093E625
:104CC000480658BF8946EBD5D8F8003040229A6094
:104CD0008AE694F8F324336801208242986007D171
:104CE0001A69D8F87C33C2F312029B1AC8F88C33C5
:104CF000DBF874305046984794F8F334012B7FF476
:104D000091AE002F7FF48EAE94F80136052B7FF420
:104D100089AED4F84435384A1A61384A5A611A685B
:104D20004FF080221A607DE610077FF57BAEDBF83E
:104D30007C3050469847336808229A6072E601EB4F
:104D4000810104EBC101D4F8C065D1F87C08C2F33D
:104D50000A1202443068C4F8BC0A3068C4F8C00AB9
:104D6000C1F87C2865E7254A5A611A684FF080220D
:104D70001A6044E7002184F8F2144FF40071A4F89B
:104D8000F414092161F38D23A6E647F6F070104272
:104D90003FF44FAFC2F30A1201EB810004EBC000F5
:104DA00002F1030C5FEAAC0CD0F87068D4F8C0E5EF
:104DB0004FEA810818BF002006D00130DEF80070ED
:104DC00046F8047B8445F8D1414404EBC101D1F895
:104DD00070081044C1F87008D1F87C080244C1F88A
:104DE0007C2826E7F81000202038002000ED00E0A5
:104DF000400D03003438002018000860EC3D00200E
:104E0000002F7FF44DAF94F80136042B7FF448AFA8
:104E1000D4F844352B4A1A612B4A5A611A684FF06C
:104E200080221A603CE72948A5F57401A1F51051CC
:104E3000814203D80D2161F38D234DE62449254895
:104E40002944814203D20C2161F38D2344E6224898
:104E5000A5F18C71A1F54341814203D80B2161F387
:104E60008D2339E61D491E482944814203D20A2177
:104E700061F38D2330E61B491B482944814203D24C
:104E8000092161F38D2327E61848A5F1B771A1F533
:104E90005851814203D2082161F38D231CE6144945
:104EA00014482944814203D2072161F38D2313E67C
:104EB000114912482944814234BF0621052161F37A
:104EC0008D2309E618000860EC3D0020DFC81000C3
:104ED0002013FBFE20D61300FF69180000D3CEFE7E
:104EE00040771B00C05BB3FEC091210040AC27009F
:104EF000C01D6AFE40E13300803C36FEE09C41006C
:104F000070B51A4D1A4BC5F8E43A1A4B85F8F01AE9
:104F1000002683F8276905F6E423C0E954330D23FE
:104F20000446C0F8583140F20113C0F85C6100F546
:104F3000A271A0F8443168F0FFFFE378C4F8B463CD
:104F40001F22C4F8B023012205F214459342C4F88D
:104F5000A853A4F89C2308BFC4F8AC5304F56771A8
:104F60002046BDE8704068F0E7BF00BF3033002046
:104F70005553425338220020F0B50B7813F06006E9
:104F800083B00C46054633D0202E2DD14A78FE2A18
:104F90006BD0FF2A63D14A88002A40F08B80CA88F0
:104FA000002A40F08780190600F184806148624B36
:104FB00080F82729C5F8B423EA78012183F834144E
:104FC000A5F89C1303F214431F21012AC5F8B0135E
:104FD000C5F8A83305F5677108BFC5F8AC33284696
:104FE00068F0AAFF002600E00026304603B0F0BDBE
:104FF0004B780A2B6AD00B2B63D0012BF5D18B8811
:10500000D9B21B0676D40196019BC06843F0100309
:105010000193019B036103690193484B03E002691B
:105020000192013B02D0019AD206F8D42846424FA1
:1050300068F072FE022321794022284668F09EFE25
:1050400097F83434022B6DD094F90420002ACCDA7E
:10505000012BCAD001212846FFF752FFC5E766F0B1
:10506000F1FB0226304603B0F0BD4E8816BBCC885B
:10507000012C1FD118061DD52F4FD7F84C349B6932
:105080009847C0B287F8F40AA0B1022307F6F427C4
:1050900085F811314FF48073C5E94E44C5E94A776C
:1050A000C5E94C46A5F81C3105F58E71284668F017
:1050B000D5FE9AE7284666F0C5FB0226304603B0C7
:1050C000F0BD1D4B4A8883F8F52A8EE7022280F84E
:1050D00011214FF48072A0F81C21194A0123C0E964
:1050E0004E33C0E94A22C0E94C3600F58E7168F0B3
:1050F000B5FE7AE70096009BC06843F0200300935A
:10510000009B61F38A130093009B03610369009382
:105110000A4B03E002690092013B87D0009A970690
:10512000F8D483E78121284666F0C4FB002387F882
:1051300034345AE73822002030330020400D030079
:10514000253E002010B50D4B93F82739022B07D0D0
:10515000033B012B02D80021FFF7D2FE002010BD37
:10516000074B93F82114044668F098FF0028F5DAFD
:1051700001212046FFF7C4FEF0E700BF38220020DF
:1051800030330020F8B5404E96F82759074655B100
:10519000012D06D13D4B93F8211468F07FFF0028C4
:1051A00032DB0020F8BD394CB0F8B433D4F8182401
:1051B000C4F8E82A1F2BD4F81C24C4F8EC2A08D120
:1051C000334BD4F814249A4203D194F821140129C2
:1051D0001FD994F8F63A04EBC3020133DBB2042B77
:1051E0004FF0050108BF002382F8F81A4FF4005170
:1051F00084F8F63A38460223C2F8FC1A84F83434AC
:10520000FBF7ECFF0020F8BD29463846FFF778FE93
:10521000C7E794F82234013B0F2BDAD868F03EFF41
:10522000002827DB96F82739013B022BB9D9B4F8BF
:10523000183B1BB3042286F82729164AC7F85C518D
:10524000C7E95422D4F81C2484F8F05A934228BFAA
:105250001346D4F8EC2AC7F8583140F20111A7F8E8
:105260004411D31A07F5A2713846C4F8EC3A68F035
:1052700063FE96E73846FBF7B1FF92E719463846DA
:10528000FFF73EFE8DE700BF3822002030330020BC
:10529000555342436C6F002010B54FEA511E024433
:1052A00000EB8E0C624529D901F01F014FF0FF344D
:1052B00004FA01F350F82E100B4093FAA3F3B3FA5B
:1052C00083F3DBB2202B16D10CF104018A4202D801
:1052D00017E08A4212D98C460431DCF8003093FA88
:1052E000A3F3B3FA83F3DBB2202BF2D0ACEB0000D4
:1052F00003EBC00010BD03EB4E1010BD4FF0FF30AC
:1053000010BD204610BD00BF30B503694268494D4D
:1053100083B00BB9002A65D0D0ED067AC46A013398
:1053200077EE807A0361631C012BC0ED067AC362BD
:1053300047D0D0ED075A90ED097AD5F8C81307EE9B
:10534000903A30EE656AF8EEE76A8A1AC6EE267A77
:1053500081688A4277EEA57A30EE670AC0ED087A56
:10536000A6EE007AC0ED077A80ED0A7A80ED097A20
:1053700001D803B030BD012B4EDD07EE904AF8EEA8
:10538000E77A87EE270AB5EEC00AF1EE10FA46DB9F
:10539000B5EE400AF1EE10FA44D4F1EEC07AF4EE24
:1053A000677AF1EE10FA3AD690ED057AB4EEE77A24
:1053B000F1EE10FA1AD5037B33B30323037003B065
:1053C00030BDD5F8C8338168DFED1B7A80ED080A5F
:1053D0009A1A8A4280ED070AC0ED097AC9D9B0EE5F
:1053E000670ADAE7D5F8C823426095E7D0ED047A7A
:1053F000D0ED066AF8EE677A022386EEA77A03708C
:1054000080ED067A03B030BDD5F8C81341600022A4
:1054100003618261C362ACE79FED070ABDE7DFED80
:10542000067AC1E701906BF00FFA0198F0EE407A2E
:10543000B5E700BF303300200000000070B52DED4F
:10544000028B044682B000F1480503460026B1EC09
:10545000017AD3ED067ADA6A77EE877A0132012A89
:10546000C3ED067ADA626ED093ED075A93ED096ABE
:1054700007EE902A77EE455AF8EEE77AC5EEA76A6E
:1054800076EE857AF0EE466A37EE677AC3ED087AF3
:10549000E5EE876AC3ED077AC3ED0A6AC3ED096AD0
:1054A0001833AB42D3D103693A4E426801330361EA
:1054B000D6F8C8339B1A8268934240D99FED368A4A
:1054C000E36A012B4DDD013B07EE903A94ED0A7A39
:1054D000F8EEE77A87EE270AB5EEC00AF1EE10FA89
:1054E0004EDBB5EE400AF1EE10FA4CD4F1EEC07A84
:1054F000F4EE677AF1EE10FA42D690ED057AB4EE4A
:10550000E77AF1EE10FA24D41834AC42D8D1D0EDB9
:10551000047AD0ED066A90ED0C7AD0ED125AF8EECE
:10552000677A022386EEA76A0370C7EE276A85EEC4
:10553000A77A80ED066AC0ED0C6A80ED127A02B09F
:10554000BDEC028B70BD83ED087A83ED077A5E6255
:10555000A6E7037B43B10323037002B0BDEC028BCB
:1055600070BDB0EE480AC1E70022D6F8C81341600A
:1055700003618261C362026343648264C365DEE7E0
:10558000F0EE487AB9E701906BF05EF90198F0EE21
:10559000407AADE73033002000000000F0EEC07A22
:1055A000B0EEE07AB4EEE77AF1EE10FAD4BFB0EEE6
:1055B000676AB0EE476AB5EE406AF1EE10FA48D07D
:1055C000B4EEE77AF1EE10FA54BFF0EE675AF0EE5F
:1055D000475AC5EE866ADFED202ADFED203ADFED7F
:1055E000204A9FED205A9FED203A9FED204A9FEDE3
:1055F000206AE6EEA23AA6EE834AE6EEA34AF7EE6A
:10560000005AA6EEA45AE6EE845AA6EE856AB1EEDA
:10561000466AC6EE256AB4EEE77AF1EE10FA48BFA4
:10562000DFED147AF5EEC00A48BF77EEE66AF1EED8
:1056300010FA48BFDFED107AB5EEC00A48BF77EE2A
:10564000E66AF1EE10FA48BFF1EE666AB0EE660A5D
:105650007047DFED0A6ADEE739094E3DE3B59EBECD
:1056600088FA16BE45FE7FBF99FB243F69A2163E0D
:10567000A7DFA8B4DB0FC93FDB0F4940A7DFA83481
:1056800091ED007AD0ED047AD0ED055A90ED064AFE
:10569000D0ED074A90ED085A90ED096AD0ED0A6AFC
:1056A000E7EE077AF7EE003AC0ED047A91ED007A62
:1056B000D1ED017AE7EE275A90ED0B7AC0ED055A4D
:1056C000D1ED025A91ED003AD0ED0C7AA3EE254AC5
:1056D00080ED064AD1ED005A74EEA54AC0ED074AA6
:1056E000D1ED014AD1ED005AA4EEA55A80ED085A39
:1056F00091ED015AA5EE056A80ED096AD1ED015AD6
:1057000091ED026AE5EE866AC0ED0A6AD1ED016AA2
:1057100037EE267A80ED0B7AD1ED026A91ED007AB0
:10572000E6EE877AC0ED0C7A91ED026AD1ED016A5E
:10573000D0ED0D7A90ED0E7A90ED0F4AD0ED104A33
:1057400090ED115AD0ED135AE6EE267A75EEA35A73
:10575000C0ED0D7AD1ED026AD0ED127A90ED006ABB
:10576000A6EEA67AD0ED016A80ED0E7A91ED027A6E
:1057700034EE074A90ED027A80ED0F4A91ED004A2F
:1057800074EE844AC0ED104AD1ED014A35EE245A38
:1057900080ED115A91ED025AC0ED135A77EE857AD9
:1057A000C0ED127AD1ED017AD1ED005A91ED025A95
:1057B00067EEA77AE5EEA57AE5EE057AA5EEA76A8B
:1057C00080ED006A91ED016AE6EE276AC0ED016A9C
:1057D000D1ED026AA6EEA77A80ED027A90ED037A07
:1057E00077EE277AC0ED037A704700BF2DE9F04FBE
:1057F00089B0CDE9011200F11009834600F13008AB
:10580000CE4607464E46054684460024CDF80C9009
:105810006246284684B1D2ED007A01463B4689466D
:10582000F3EC016A99ED007AE6EEC77A634501F17F
:105830001001C2ED007AF2D10432724500F1040089
:10584000E8D1032C04F1010A30D062463046ABEBBC
:1058500005099CB1D2ED047A009409EB00032946B6
:105860000C46F3EC016A94ED007AE6EEC77A8342C7
:1058700001F11001C2ED047AF2D1009CD2ED046A6C
:1058800016ED047AC6EE877A1032424500F1100018
:10589000C2ED007ADDD10CF1140C08F104080435D6
:1058A00014360EF1100E10375446B1E7DDE9022927
:1058B000002500230135059306930793042D52F824
:1058C000043B049305A80BF1140418D0F2EC017A00
:1058D00004A9C0ED007A4B46B1EC017AF3EC016A01
:1058E000E6EEC77AA342C0ED007AF5D10135042D6A
:1058F00009F1100900F1040004F11404E6D1019A41
:1059000008AE76ED017A022510320BF14004022D2B
:105910002046A2F1040142ED017A20D02346F3ECA7
:10592000016AB2EC017AE6EEC77A9842C1ED007ADC
:10593000F5D154ED016A87EEA67A6B1C81ED007AF1
:1059400014D076ED017A013D0A46022DA4F114042B
:10595000A0F11000A2F1040142ED017ADED154ED74
:10596000016A87EEA67A02ED017AEAE709B0BDE89E
:10597000F08F00BF10B584B00C4602466946103067
:10598000FFF734FFDDED007A9DED017ADDED026A6F
:10599000B6EE006A67EE867A27EE067A66EE866ACB
:1059A000F4EE677AF1EE10FAC4ED007A84ED017A34
:1059B000C4ED026A0DD6B4EE477AF1EE10FA13D6B2
:1059C000F4EE666AF1EE10FA78BF012016D604B044
:1059D00010BD9FED106AF0EEE77AF4EE467AF1EE34
:1059E00010FAE8DD0020F2E7DFED0A7AB0EEC77AC0
:1059F000B4EE677AF1EE10FAE2DDF3E7DFED057A57
:105A0000F0EEE66AF4EE676AF1EE10FAD4BF012018
:105A10000020DCE7FFFF7F7FDFED257AB4EEE70AA9
:105A2000F1EE10FA08DD9FED237A30EE470AB4EE6E
:105A3000E70AF1EE10FAF8DCDFED1F7AB4EEE70AC0
:105A4000F1EE10FA08D59FED1B7A30EE070AB4EE9E
:105A5000E70AF1EE10FAF8D4DFED187AB4EEE70AAF
:105A6000F1EE10FA18DD30EE670A37EEC00A60EE8C
:105A7000007A9FED137A9FED136ADFED136AA7EEAC
:105A8000876A9FED127AE7EE866A60EE275AA7EEE4
:105A9000A67AA5EE870A70479FED0D7AB4EEC70A85
:105AA000F1EE10FA44BF30EE270A37EE400ADEE787
:105AB000DB0F4940DB0FC940DB0F49C0DB0FC93F9B
:105AC0009A7C2E36FAAF4FB93587083CA4AA2ABE75
:105AD000DB0FC9BF10B53E4CB4FBF2F4A1420DD3AD
:105AE00000234FF07E52026043608360C360036115
:105AF0000023836143610362C36110BD07EE902AF6
:105B0000B8EE677ADFED337A27EE277AB7EE006AD0
:105B1000C6EE076A07EE901A9FED2F7AF8EE677AC5
:105B2000B0EE405A67EE877AC7EEA64AFDEEE47AF9
:105B300017EE902A2032402A47D8B0EE640AFFF7C9
:105B40006BFFB0EE404A9FED250A34EE800AFDEE71
:105B5000C07A17EE902A2032402A31D8FFF75CFF36
:105B6000F8EE006A60EE266A012B24D0F7EE007A88
:105B700037EEC00AF6EE005A60EE255A35EE055AA9
:105B8000B7EE007A84EE056A76EE077A37EE467A4B
:105B900080EE275A85EEA76AC6EEA75AC7EE276A97
:105BA00080ED006A80ED015A80ED026AC0ED035A73
:105BB000C0ED046A9CE7B0EE660AF7EE005ADDE736
:105BC000DFED076A9FED070ACEE79FED064ABAE7C9
:105BD00020A10700BD378635DB0FC940DB0FC93F69
:105BE0000000008000000000DFED077A30EE270A99
:105BF000FDEEC07A17EE903A2033402B00D80BE729
:105C00009FED020A704700BFDB0FC93F0000000094
:105C100091ED005A9FED520A35EE000A08B5FDEEEF
:105C2000C07A17EE903A2033402B7DD8FFF7F4FE70
:105C3000FDEEC57AB0EE403A17EE903A2033402B95
:105C40007BD8B0EE450AFFF7E7FEB0EE405AF1EE22
:105C5000402A91ED014A9FED420A34EE000AFDEE22
:105C6000C07A17EE903A2033402B74D8FFF7D4FE59
:105C7000F0EE404AB1EE402AFDEEC47A17EE903ABB
:105C80002033402B64D8B0EE440AFFF7C5FEB0EED7
:105C9000404AD1ED021A9FED320A31EE800AFDEE44
:105CA000C07A17EE903A2033402B4ED8FFF7B4FE5F
:105CB000F0EE403AFDEEE17A17EE903A2033402BB9
:105CC00040D8B0EE610AFFF7A7FE63EE836A20EECC
:105CD000037A63EE857A20EE055AF0EE475AB0EE6D
:105CE000666AE7EE845AA5EE446AE7EE047AA6EE09
:105CF000C45A63EEA43A62EEA42A22EE000A64EECD
:105D0000834AC0ED003A80ED010A80ED024AC0ED01
:105D1000035A80ED046AC0ED052A80ED065AC0EDF5
:105D2000077AC0ED084A08BDFDEEC57A9FED0D3A31
:105D300017EE903A2033402B83D9DFED0B2A9FEDED
:105D4000095A86E79FED070ABFE7DFED063AB1E79C
:105D50009FED044A9DE79FED042ADFED024A8BE7A1
:105D6000DB0FC93F00000000000000802DE9F04F6C
:105D700083B005469DF830400D9E0192002C14BF63
:105D80004FF030094FF020091C1E88464ADB16F8F8
:105D9000010B014600286CD0002C65D04FF0000AA2
:105DA000324601E0002C34D012F8013B2746013C7A
:105DB000002BF7D1BAF1000F3CD1023F002C65D087
:105DC000BA4645450AF1FF3A4946284601D2019BA9
:105DD0009847BAF1FF3FF4D10D9A107823463C1B47
:105DE00001469B4688B14FF0000A01339F1B454591
:105DF00006EB070B284601D2019B984716F8011BBA
:105E00000029F4D1BAF1000F18D1584603B0BDE80B
:105E1000F08FBAF1000F31D0014683460028F4D04C
:105E20002346E2E716F8010B634258B31C464FF0D5
:105E3000010AB5E7014683460028D6D1002C04F1BB
:105E4000FF36E2DD3446454506F1FF364946284631
:105E500001D2019B9847731CF5D10BF1010BA344B0
:105E6000584603B0BDE8F08F2346A2464FF0FF34FA
:105E7000BBE7671EA346002CA2D1C6E723464FF01E
:105E8000FF34ADE7E64383463446DCE723463C4631
:105E9000A6E700BF0FB430B583B006AB0C4853F88B
:105EA000042BD0F8B41CD0F8B00C019368F0D0FCEF
:105EB000084C0546D4F8B00C03685B699847002885
:105EC000F8D0284603B0BDE8304004B0704700BFAA
:105ED00030330020382200200EB410B583B005AB5B
:105EE000044653F8042B0749009301A8019468F075
:105EF000AFFC019B00221A7003B0BDE8104003B054
:105F0000704700BF250A00080CB470B5334CD4F8B4
:105F1000B83CA4B0002B4AD094F8C03C99423ED87B
:105F2000D4F8C8332E4AA2FB031292094FF47A71B7
:105F300001FB123304A82B49FFF7CEFF04AA29ABBB
:105F40000244CDE902322849289A064603A868F09F
:105F50007FFC039BD4F8B85C5A1C03920A221A7087
:105F6000039B5A1C039200221A702DB32B681B6AE4
:105F70001BB128469847D4F8B85C9DF8101049B179
:105F80000DF111042B6828461B68984714F8011B73
:105F90000029F7D124B0BDE8704002B07047D4F8B2
:105FA000C42C012303FA00F01042B9D1F2E7D4F86F
:105FB000BC3C002BB0D1EDE7D4F8BC3C002BE9D0C1
:105FC00030440222009204A98218FD2036F080FF9E
:105FD00024B0BDE8704002B0704700BF30330020ED
:105FE000D34D6210C8130808190A000830B54FF4E1
:105FF000004087B034F056FE58B14FF400410446DB
:1060000034F07AFE022806D1226848F201039A424F
:1060100024D007B030BD00234FF46121022294F94F
:1060200004008DE80E001A464FF4004134F06EFE75
:106030001C4BC3F8B80C0028EBD01B4A1B4B1C4C64
:106040001C481D490091CDE90332CDE901041B4BE9
:106050001B4A02210020FFF757FFDAE7114C002509
:106060004FF4004084F85C5F64F0BEFA0028D0D0A2
:10607000D4F8C83C83420AD0D4F8A43D83420BD064
:10608000D4F8803E98420AD0C4F8BC5CC1E704F65C
:10609000C843C4F8BC3CD0E704F6A453F9E704F5C0
:1060A0006863F6E730330020EC130808F81308089B
:1060B0000414080810140808081308081413080822
:1060C000D413080838B5194CD4F8605F033005EBD9
:1060D0009003B3F5007F19D820F003021448C4F8E8
:1060E000603F00EB8101C3F50073D1F86C0604F644
:1060F00064741044C1F86C060E4A04EB85049B00DE
:1061000004210020FFF700FF204638BD002108468B
:10611000094AFFF7F9FE094AD2F89830002443F003
:106120000073C2F89830204638BD00BF30330020DD
:1061300028440020181408083C1408080000001027
:10614000F0B5254B0268254983B00646002401E0DE
:1061500051F834309A4209D001340E2CF8D1002184
:106160001F4A0520FFF7D0FE002113E01D4F07EB6B
:106170008407D7F8505485B1717901EB410305EBE1
:10618000C30300221820C3E9032200FB01559E60CF
:106190001A75291D084603B0F0BD07216420FFF7DA
:1061A00091FF0146C7F8500470B1294664226FF090
:1061B00079F90A4BD7F8505403EBC404C5E90045FC
:1061C000ED616D63ED64D7E70190074A0520FFF7A5
:1061D0009BFE0199DEE700BF000001403C65070817
:1061E0004C140808303300207414080870B5066891
:1061F000F46982B00546002C3FD03379012B04F1BD
:10620000030205D0022B2CD00020A07002B070BD7C
:10621000B368717C96F91000009203F001030193BA
:106220000C220D23FDF752FBA0700028EED0B4F92C
:106230000A3007EE903AF8EEE77AC5ED077AB4F93E
:106240000C3007EE903AF8EEE77AC5ED087AB4F92B
:106250000E3007EE903AF8EEE77AC5ED097A02B013
:1062600070BDB36813F0010F30464FF00D0314BF3B
:106270000C218C2102F090FBD6E709211420FFF7B6
:1062800021FFF06104462E68B7E700BF38B5056806
:10629000EB690446E3B1987800B938BDB3F904203E
:1062A00007EE902AF8EEE77A0120C4ED047AB3F9FC
:1062B000062007EE902AF8EEE77AC4ED057AB3F9E6
:1062C000083007EE903AF8EEE77AC4ED067A38BD6A
:1062D00009211420FFF7F6FE0346E861DBE700BF63
:1062E00003681A46591C016012F8021B02605878B4
:1062F00041EA0020704700BF02681146531C03604A
:1063000011F802CB0160D31C5178036093781B0411
:1063100043EA0123111D0160D07843EA0C0343EAEC
:106320000060704712B370B50446864604E0981BBF
:1063300017D114EB0C0C15D01EF8013BA3F1410052
:10634000192811F8010BA0F1410598BF2033192D30
:10635000A2EB0E0C00F12006E9D91B1A04D100288B
:10636000E7D170BD604670BD184670BD10467047DD
:1063700010B40288C378184CA2F5FA6202F0030147
:1063800040F2B55C9208013B0CFB0233827801EBD2
:106390004101013A02EB810204EB42010279B1F8BA
:1063A000E4404179234403EB430302EBC3038479C4
:1063B0000A4A0089C3EB031301EB8303C3EB031306
:1063C000224402EB830200214FF47A73C2FB0301E3
:1063D0005DF8044B704700BFE464070880436D38E4
:1063E0002DE9F04117461E4605464FF47A72002308
:1063F0003846314669F096FA4449454A014482FBE1
:106400000143C8170B44C0EB631382FB03021A4419
:10641000D817404CC0EB621284FB02044FEAE27CC6
:106420003D48CCEBA40C80FB0C404FEAEC74C4EB71
:10643000E010C3EB0314A1EB8401A971C2EB0211BC
:10644000A3EB81036B710CEB4C03A2EBC30240F294
:10645000B55303FB10CCBCF5896F2A714FEA80005D
:1064600045DA40F2DA239C4548DCBCF5B77FB4BF7F
:1064700000220122294B02EB420103EBC1034FEA48
:106480004208B3F8FA3091B2254C08EB020E04EB47
:10649000CE0416344FF00B0E01E034F8023D634594
:1064A00020DDBEF1010EF8D11C4B424403EBC202C9
:1064B0004FF0010EB2F8E43085F802E000F5FA6022
:1064C0000CF1010C0844ACEB030C288085F803C0E8
:1064D0004FF47A7200233846314669F023FA2A8154
:1064E000BDE8F0810EF1010E5FFA8EFEE4E70321B4
:1064F00040F296530A464FF00608C5E7022140F2E3
:1065000029430A464FF00408BEE700BF80BC92C78B
:1065100089888888ABAAAA2A73B06D16E464070834
:10652000C865070830B52E4D84468E460FCD8DB018
:106530006C460FC40FCD0FC495E80F001CF0030F7D
:1065400084E80F000DD1274B274A03FB0CF3B2EB75
:10655000B30F43D3254AB2EB331F2CBF1D241C2499
:1065600000E01C240CF1FF33002B40F26D121946A1
:1065700002FB0CF2B8BF0CF1020102EBA1021C49B4
:106580001C4D019481FB0301DB17A3EB6110024456
:10659000C3EBE1131A44253285FB02301044D317B4
:1065A000C3EBA000C0EBC000ADF10403101A0DF165
:1065B000040C03EB8E0E01E05CF8044F031985FB1D
:1065C0000320C218D817C0EBA200C0EBC000E645FC
:1065D000A3EB0000F0D1201A0DB030BD1D24C1E79F
:1065E00028660708295C8FC2285C8F020AD7A3009F
:1065F0001F85EB519324499208B50D4B53E90223B3
:1066000052EA030C09D1002340F201124280838038
:10661000837103800381184608BD0649D1F8C81369
:106620008A1843F10003FFF7DBFE012008BD00BF1D
:10663000284B00203033002088422DE9F0414FF0F4
:1066400001043DD301FB04F4B0FBF4FC8C45F9D20A
:106650003CB3002616E0BCF1090F274698462C46AD
:1066600023DD002A14BF4FF0370E4FF0570EF444CD
:10667000B94288F800C003F1010306F1010610D801
:10668000B0FBF5FCB4FBF1F504FB1C00002EE2D1DD
:10669000BCF1000FDFDCA1420AD90CF1300C03F889
:1066A00001CB00221A70BDE8F0814FF0300EDEE71A
:1066B000B0FBF5FC2C4605FB1C00B5FBF1F5E7E74C
:1066C0008446C6E790422DE9F0410B460446154644
:1066D0000AD2B0FBF5F6134A05FB16441846135DC3
:1066E00000F8013BBDE8F081B0FBF2F69642B6FB44
:1066F000F2F706D20B4A05FB1767D15D03F8011BC1
:10670000EAE7BA42B7FBF2F807D9064A05FB187860
:1067100012F8081003F8011BEDE74046FFF7D2FF1F
:106720000346F2E790140808B5EEC00ADFED347AAC
:10673000F1EE10FACCBF30EE270A30EE670ADFED3B
:10674000317A20EE270A70B5FDEEC07A86B017EEDA
:10675000904A054684EAE470002303A9A0EBE470A4
:10676000CDE90033029365F055FC002CACBF20232B
:106770002D2303A88DF8003068F0ACFA01286E468E
:1067800028D0022832D003281CD003A930466FF04D
:10679000D9FD304668F09EFA0338C4B2224631462D
:1067A00028466CF0DFFC00232B55284668F092FA4F
:1067B0002E232B540130311928446FF0DFFD284679
:1067C00006B070BD302303A930468DF801306FF05C
:1067D000B9FDDEE7302303A930468DF801308DF88E
:1067E00002308DF803306FF0ADFDD2E7302303A9FE
:1067F00030468DF801308DF802306FF0A3FDC8E708
:106800006F12033A00007A440278202A034600F10E
:106810000100F9D0092AF7D02D2A29D02B2A03BF4D
:106820005A78B7EE000A0346B7EE000AA2F130012B
:10683000C8B20928DFED4C7A10D8F2EE046A07EEF0
:10684000101AB8EEC77A13F8012FA7EEA67AA2F1B4
:106850003001C8B20928F0EE477AF0D92E2A49D083
:10686000197801F0DF01452907D020EE270A70478B
:106870005A78BFEE000A0346D8E710B459782D299C
:1068800062D02B2954D0A1F13002092A03F101036F
:1068900055D80024002202EB820201EB420213F8D9
:1068A000011FA1F130000928A2F13002F3D9B2F59D
:1068B0009A7F134628BF4FF49A73072A50D9DFED09
:1068C0002B6A1A46B7EE007A083A072A27EE267A8C
:1068D000FAD803F007032BB1F2EE046A013B27EE6E
:1068E000267AFBD16CB3C7EE877A5DF8044B20EEB5
:1068F000270A70475978A1F13002D0B2092803F174
:106900000103AED8F2EE046AF0EE665A07EE102AE2
:10691000B8EEC77A13F8011F87EE266AA1F130029C
:10692000D0B2092866EEA56A77EE867AEED998E7A6
:106930009978A1F13002092A03F10203A9D9B7EE2F
:10694000007A67EE877AD0E79978A1F13002092AB8
:1069500003F1020388BFB7EE007AC4D8012499E797
:10696000B7EE007AB7E700BF0000000020BCBE4CC5
:1069700000B50378202B014600F10100F9D0092B66
:10698000F7D02D2B03BF4B784FF0FF3E01464FF061
:10699000010E0022A3F1300C5FFA8CF3092B03D90E
:1069A0000EFB02F05DF804FB02EB820211F8013FDE
:1069B0000CEB4202EEE700BF2DE9F04F93B044F03C
:1069C00071FB44F035FBAC4B0793B0F1000940F389
:1069D0002B814FF0000A9B46A84BA94CCDF804A090
:1069E00002935646D04604E008F50068C14540F3DE
:1069F000918020220AA9404644F0A0FAA14912221F
:106A00000AA86EF0E9FC05460028EDD1B04521D07A
:106A1000019A9D4F9D49CDF80CB002EB420307EB64
:106A20008307013238460192FFF756FADBF81C2043
:106A3000039B43F84C7BCBE90822954ACBF80C60CA
:106A4000CBF82820A8EB06060122CBE90466CBF898
:106A500008209B46029BD3F8F037CBF81C30464603
:106A6000122202F148030DEB030114F80A3011F869
:106A7000201C994202F101020CD04FF0000A202A9A
:106A8000EFD12036B1450AA9304639DB44F056FA39
:106A90000022E6E70AF1010ABAF1150FEFD19019C9
:106AA0000AA9202244F04AFA7A4909AA0AA86DF0F4
:106AB00069FB28B30027CDE90477039706973E4684
:106AC000731E042B00F29E81DFE803F09A8DA29ED4
:106AD0000300FFF74DFF0546069989B1DDE9042360
:106AE000039843EA42127B0143EAC023A1F2BC713E
:106AF00043EA650342EA412243EA0243CBF81C30F1
:106B0000019B642B00F0B480464608F50068C1453F
:106B10003FF76FAF019A642A00F0AA80B0457BD09E
:106B2000594C5A495A4F0C2303FB0244531C1A4632
:106B30002046A8EB06050193FFF7CEF9DBF81C30E1
:106B4000CBF80040CBE90365CBE908330123CBF850
:106B50001450CBF82870CBF80830019B1D1D4E4C0B
:106B60000299D4F84C61C1F8F0674C2202FB05F59C
:106B70006319002118466EF095FC4C2200216EF03E
:106B800091FCDFF820A144F805A0019D8762C0E9CF
:106B90000499C0E907664FF00108C0F80880466212
:106BA00005354FEA4903B3F1805F42DB029B3B4965
:106BB0003948D3F8F0574FF498726CF0D3FA36494D
:106BC000079A0C460B465D62C3E907554C339A425F
:106BD000F9D1A66826B9237913B12368002B63D1B4
:106BE00013B0BDE8F08FFFF7C3FE059029490020E0
:106BF00009AA6DF0C7FA013600287FF461AF6BE790
:106C0000FFF7B6FE0490F1E7FFF7B2FE0746EDE7A7
:106C1000FFF7AEFE0390E9E7019B1D1D002B40F03E
:106C2000EF801D4C0425BCE7144A02920425A3F50D
:106C300098744C2202FB05F56319184600216EF08A
:106C400031FC4C2200216EF02DFC0299C9F100624A
:106C50000346520012486051D1F8F0175962C3E957
:106C6000042202225A710122C3E907119A609DE7AA
:106C70006423074F019370E724510020F81000208F
:106C8000DC140808B8140808284B0020CC140808A5
:106C9000AD220008F4140808F44F002058660708D5
:106CA0000C150808FC140808C4E91166574A266444
:106CB000E663304637468E46D56C02F14C0355B339
:106CC000D3F808C01F64451EAC45C3E91177DF63E4
:106CD00013D0451CAC4517D0844581D10546002D05
:106CE0003FF47EAF106CC16B01F1010CC0F83CC0E9
:106CF0001864936428461A46DEE700283FF470AF14
:106D0000854253F80C2CEAD1107900283FF468AF83
:106D100053641A64EEE7714602222F46A64613E03A
:106D2000CB6B0A635B011DBF03F6FF7002F1FF33FB
:106D300003EB10331346C1E90477C1E90D3351F871
:106D40004C0F5A1C0136C8B10B79002BE8D10B69E6
:106D50000A63002B47D14C691046531E4863002C30
:106D60004AD004F6FF7C03EB1C33281A8B63C5184A
:106D700051F84C0F5A1C01360028E5D124493E2217
:106D8000C1F8882C3F22013BC1F88C2CC1F8A05CD3
:106D90004022204DC1F8902C7446C1F8AC6CC1F86B
:106DA0009C3C980F9A00C1F8845C3BB340F2FF15FD
:106DB000521940F10000520A42EAC05202F140006A
:106DC000024402EBC303C1F8982C134AC1F8940C97
:106DD000C1F8A44CC1F8A84CD80D5C0242E90240AD
:106DE000C1F8803CFCE603F6FF7C4C69531E03EBC4
:106DF0001C304863002CB4D11346B6E70122DDE70E
:106E0000064FACE6FFF7B4FD0690EFE6F44F002026
:106E1000382200201C150808B82E0020AD220008DA
:106E2000F0B5384D2B78082141F221008B4002E06B
:106E3000013993B209D013F4004F4FEA4302F7D05F
:106E400080EA430301399BB2F5D1B5F80120002A4D
:106E500055D0DFF8C0C02C4EB4452DD2ACF1060C95
:106E60000CEB0204B44227D2052A41F2210022D9B8
:106E7000A44514D00CF1FF3C04F1FF3E1CF8011FA7
:106E8000082283EA012313F4004F80EA43010ABF7A
:106E90005B008BB29BB2013AF5D1E645EED1228878
:106EA00062B1A11DB14206D2A118B142A44602D2DC
:106EB000052A0C46DCD800210846F0BDA71C264652
:106EC00041F2210016F8011B082283EA012313F482
:106ED000004F80EA43010ABF5B008BB29BB2013ACC
:106EE000F5D1B742EED16188084AC91AB1FA81F1E9
:106EF000231D49095B1BA2F8B03B0846F0BD044FB7
:106F0000BC1EDCE700000E0800001008284400202A
:106F100003000E0807000E082DE9F04F9B4B9C4A1A
:106F20008FB09A1ACDE9013203230393984B07934C
:106F3000029B0993019B08930023CDE90A33CDE915
:106F40000C33944A1369002BC0F2A181914B9249F2
:106F5000F322DA6000220C92019A01238A428DF812
:106F60003430C0F08C810B937E238DF828300822BA
:106F70004FF4FC4341F2210103E05B00013A9BB274
:106F800006D01804F9D581EA4303013A9BB2F8D13F
:106F9000824AADF81230824B934280F08E8103F129
:106FA000140801997A4B41F2210538F8120C38F88F
:106FB000142CC0F30B06B41DADF81440C2F30B043F
:106FC000120B8DF8182000270204ADF816408DF83A
:106FD00019705DD406338B4200F251810DF1140912
:106FE0000DF11A0A4C4601E0A24513D00B9B14F890
:106FF000011B03F138026A440133042B02F8101C10
:107000000B93F1D10AA907A8F9F72EFDA245CDE906
:107010000B70EBD10C9B002BC0F23181BDF81240FC
:1070200019F8013B84EA0324082327044CBF85EAAE
:1070300044046400013BA4B2F7D1CA45F0D158F82A
:10704000101C324607A8F9F7C1FD0028C0F21781CD
:1070500058F8102C91198A4210D0013A013912F8CF
:10706000013F84EA0324082320044CBF85EA44043A
:107070006400013BA4B2F7D19142F0D1474BADF887
:107080001240984574D2DDE9073108F114088CE705
:10709000B946CDF8008009F1010906335FFA89F994
:1070A0008B428DF8199000F2EA800DF1140A0DF16F
:1070B0001A0BD046002401E0C34513D00B9B18F8EF
:1070C000011B03F138026A440133042B02F8101C3F
:1070D0000B93F1D10AA907A8F9F7C6FCC345CDE97E
:1070E0000B40EBD10C9B002BC0F2C980BDF81240C5
:1070F0001AF8013B84EA0324082322044CBF85EAE2
:1071000044046400013BA4B2F7D1D345F0D1009B05
:1071100053F8102C02EB070A5146324607A8F9F73C
:1071200055FD0028C0F2AB800AEB06018A4511D05C
:107130000AF1FF32013912F8013F84EA03240823DF
:1071400020044CBF85EA44046400013BA4B2F7D19B
:107150008A42F0D1B9F1030FADF81240374402D0A2
:10716000DDE9073197E7DDF800800C4B98458AD3BD
:10717000DDE90731023300229942ADF814207ED3B5
:107180000DF115040DF1160516460FE0000010086C
:1071900000000E08003C024001000E08B0920808F2
:1071A000748D0808A54213D014F8012B0B9B03F132
:1071B000380169440133042B01F8102C0B93F1D1F1
:1071C0000AA907A8F9F750FCA542CDE90B60EBD15D
:1071D0000C9B002B53DBBDF81230082241F2210139
:1071E0001C0454BF5B0081EA4303013A9BB2F7D110
:1071F000082241F2210118044CBF81EA43035B00DD
:10720000013A9BB2F7D1ADF81230079B08990233CF
:107210008B4234D814460DF1120505AE01E0B5429B
:1072200013D00B9B15F8011B03F138026A4401339C
:10723000042B02F8101C0B93F1D10AA907A8F9F747
:1072400013FCB542CDE90B40EBD10C98002816DBBE
:107250000B9B13B3079A08991A448A420FD80AA9BC
:10726000C818C3F1040200216EF01CF90AA907A88E
:10727000F9F7FAFB002398420C900B930DDA039B6D
:10728000013B03937FF452AE052006F09DFD0F4BAA
:10729000536003F18833536058E69DF834307BB96E
:1072A0000028ECD10A4B1B787E2BEDD1FFF7B8FDFF
:1072B0000028E9D00FB0BDE8F08F0199044B59E7E1
:1072C000044A136943F000431361E9E7230167456A
:1072D00000000E08003C024070B545880B4604468D
:1072E000C5F30B052A46002118466EF0DBF821692C
:1072F000084A9142034602D3074A914205D319B185
:10730000BDE870401846084770BD2A46BDE8704089
:107310006BF028BFB09208086B9708082DE9F04180
:10732000944603EB43031CF8068B86B0144602EB2D
:10733000430315464FFA88F69CF80070A0EB070E41
:10734000821BBEF1000FB8BFCEF1000E002AB8BFFD
:1073500052429645B8BF65460CF1060CB8BF7EB2E6
:107360006345E9D1B0456F88A3F1060206D0BE4659
:10737000A24216D014F8068FB045F8D1B4F80280B6
:10738000CB1BA1EB080C002BB8BF5B42BCF1000F7C
:10739000B8BFCCF1000C6345BE46E9DD4746254643
:1073A000E5E76B7904932B7903932B78064A0091D8
:1073B000CDE9013E032103460120FEF7A5FD284645
:1073C00006B0BDE8F08100BF241508084FF4006343
:1073D000838170474FF40063838170474FF40063EB
:1073E00083817047074B10B403F11001002453F858
:1073F000042B824208BF43F8044C8B42F7D15DF85E
:10740000044B7047707F00200120704701207047B7
:107410002DE9F84F6D4DD5F810C0A88AB5F91E902A
:10742000B5F81AE0C0EB2C1303FB03F4B5F91830E0
:10743000241303FB04F44000B5F91630C0EBEC0054
:1074400003FB00F0A41304EBE024B5F91C30EC625C
:107450000F46A4F5FA31164683FB013281FB018CFD
:1074600012034FEAE97B42EA13524FEA033A09FB5F
:107470000CF308FB0B3BA9FB0839D9441B0A43EA70
:10748000096313EB0A0342EB292202F50042A3FB36
:107490000E390EFB029E4FEAEE734FEA6E0253EA7C
:1074A0006E0E4FF0000000F08580B5F9249009FBC6
:1074B0000CFEB5F922C08CFB011C4FEAE97A4FEAB9
:1074C0004C4C08FB0AEE4CEAD13CA9FB0898490455
:1074D00011EB0901F04448EB0C0C4018296BC1F585
:1074E0008019B5F9201009F0004E4FEAC978B8EBC1
:1074F00000080CEBC1014EEA590E6EEB010E18EBC1
:10750000080C4EEB0E011CEB080C4EEB01014FEA90
:1075100081194FEA8C1049EA9C691CEB000C41EB85
:107520000901890041EA9C714FEA8C0C1CEB080CA4
:107530004EEB01014FEA8C00890010EB080041EA94
:107540009C714EEB010168F0EDF9B5F92A20B5F90F
:1075500028E0B5F926504FEA6138430B43EAC143AE
:1075600002FB08FC4FEAE27903FB09C9A2FB032CEA
:10757000CC4402FB08F803FB0C88A2FB032CC44498
:10758000520E42EACC12121841EB6C6C4FEAEE73C9
:107590000EFB01F103FB0011AEFB00300144DB0CDC
:1075A00043EA4133D0184CEBE141000A40EA016064
:1075B00000EB05100FB1000A386026B104EB84041B
:1075C0008034241234600120BDE8F88F707F0020E1
:1075D00031B10A4BD3ED137AFDEEE77AC1ED007AB3
:1075E00052B1064B9FED067AD3ED147A67EE877A97
:1075F000FDEEE77AC2ED007A01207047707F00202F
:107600000000C8420120704710B4104B104C1B689A
:10761000606D1B1AFA2B0DD809B1E36D0B602AB10E
:10762000236E136001205DF8044B704701205DF864
:10763000044B7047074A1368002023F0040384F8C2
:10764000580013605DF8044B704700BFF836002007
:10765000707F00209C00001001207047044B002226
:1076600000215A669A66DA6619670120704700BFE2
:10767000707F00200F4B104A1B68116F5B1AFA2BAA
:1076800016D8D2ED196A92ED1A7AD2ED1B7AFDEE78
:10769000E66ABDEEC77A16EE903AFDEEE77AC3864B
:1076A00017EE103A038717EE903A43870120704790
:1076B00000207047F8360020707F00200048704797
:1076C000EC180020014B5B6F5B681847707F00204F
:1076D000024B5B6F08309B68184700BF707F00202B
:1076E000012070470120704701207047012070473A
:1076F0000120704731B10C4BD3ED1E7AF8EEE77ADA
:10770000C1ED007A72B1084BDFED086ADB6FA3F5BB
:10771000D543333B07EE903AF8EEE77A87EEA67A48
:1077200082ED007A704700BF707F00200000C842E1
:107730000120704701207047704700BF044B03EBE6
:107740008000D0F880300BB19B681960704700BF93
:10775000707F0020044B03EB8003D3F880300BB123
:107760009B68196027F0B4BC707F0020044B03EBCA
:10777000C00040F2FF739942A8BF1946818070474C
:10778000903E00200C4A137C7BB10C4B93F8C01048
:1077900059B193F8C11059B150690022FA2883F801
:1077A000C120A8BF4FF0FF3070476FF00100704755
:1077B0006FF00200704700BFEC180020707F0020BF
:1077C0000B4B93F8C22082B193F8C32052B1094900
:1077D00088690022B0F5967F83F8C320A8BF4FF0D8
:1077E000FF3070476FF0020070476FF00100704784
:1077F000707F0020EC180020024BD3F8C4305B6887
:10780000184700BF707F0020024BD3F8C4309B683C
:10781000184700BF707F0020024BD3F8C430DB68EC
:10782000184700BF707F0020014BD869704700BF28
:10783000EC180020044B93F8C83013B1034B186ABE
:1078400070476FF001007047707F0020EC18002037
:107850004B1EDBB2062B30B598BF214A214C98BF96
:1078600032F8135004F1580388BF4FF48075002894
:1078700008BF1C46A44620893CF8082B87B04FFA65
:1078800082FE90B12A1AA5EB0E03002AB8BF52421D
:10789000002BB8BF5B429A42BCBF4FFA80FE6446E1
:1078A0003CF8080F0028EDD122880F4B0F4893F8C1
:1078B000C9C0A3790593A38804930D4BBCF1000FB5
:1078C00008BF0346A078CDE90015CDE902200321C9
:1078D000084A0120FEF718FB204607B030BD00BF64
:1078E000E472070810190020707F00203416080881
:1078F0005C2A08083816080838B50568EB6904469C
:10790000E3B1987800B938BD9A88D2BA07EE902AC8
:10791000F8EEE77A0120C4ED047ADA88D2BA07EEED
:10792000902AF8EEE77AC4ED057A1B89DBBA07EEF8
:10793000903AF8EEE77AC4ED067A38BD09211420B2
:10794000FEF7C0FB0346E861DBE700BF38B504681B
:10795000E3690D467BB1987800B938BD5B89094A67
:10796000DBBA82FB0312DB17C3EB221303F26D13A6
:107970002B80012038BD09211420FEF7A3FB03460C
:10798000E061E8E77978787870B50568E8690C46D1
:107990001646A0B3D0F80130CCB1D0F805209FED49
:1079A0001B7ADFED1B5ADFED1B6A07EE902AF8EE1B
:1079B000677AB7EE006A77EEC77A77EEA77A87EE36
:1079C000A57A77EE467A67EEE67AC4ED007AAEB134
:1079D00007EE903A9FED107ADFED106A9FED106A86
:1079E000F8EEE77A67EE877A87EEA67ADFED0D6A22
:1079F00077EE467A77EEA67AC6ED007A70BD092159
:107A00001420FEF75FFBE861C4E700BF9AC9CC44CD
:107A10009AC94C460E76D7450000484300E0FF4423
:107A2000000048423393884370B50668F06982B01D
:107A30000D461446002848D0D0F80530DFED266A00
:107A40009FED267A07EE903AF8EE677A77EEE67ABF
:107A5000F3EE096A67EE877AB2EE047A67EEA67AE9
:107A6000F4EEC77AF1EE10FA22DCBAEE047AF4EE04
:107A7000C77AF1EE10FA1BD4D0F801302DB19FED8A
:107A8000187A67EE877AC5ED007A7CB107EE903AF6
:107A90009FED146ADFED146AB8EE677ADFED137AB2
:107AA000E7EE067A77EEA67AC4ED007A02B070BDF2
:107AB00017EE900A67F07AFA0D4ACDE90001042129
:107AC0000320FEF721FA02B070BD09211420FEF751
:107AD000F9FAF061B0E700BF00000046000080380E
:107AE0000AD778430319C83D33938843000048C23E
:107AF0008416080838B51446002944D0344B9FED4D
:107B0000356AD3ED337AB3F9E42093ED350AB8EE54
:107B1000E77AD3ED3A7AC7EE066A0D4604EE902A6C
:107B2000B3F9E020F8EEE77A05EE902AB3F9E22007
:107B300087EE864AF8EEE44A05EE102AF8EEE55A9A
:107B4000B3F9DE20D3ED367AB3F9DC30E6EEA45A91
:107B500006EE102AB8EEE77AB8EEC55AB8EEC66A55
:107B6000A6EEA57AA6EE856A07EE903AB8EEC00AB0
:107B7000F8EEE77AA6EE870AE6EE867AA4EE270A02
:107B800068F0DAFC28600CB3114BDFED125A93ED6C
:107B90003A7AB3F9D220B3F9D0309FED0F0AB8EE9C
:107BA000C76A07EE902A86EE257A06EE903AF8EE3E
:107BB000E77AF8EEE66A67EE277AB6EE006AE6EE56
:107BC000867A27EE800A68F0B7FC2060012038BD75
:107BD000707F00200000F04A0000C84230B50C4D14
:107BE00083B055F83030019183B107EE901A93EDD0
:107BF000047A93ED030AF8EEE77A0446A7EE870AC3
:107C000068F09AFC55F834309B68186003B030BDBA
:107C1000903E002070B52B4C94F8EC3082B023B924
:107C2000012084F8EC3002B070BDD4F8F050264A40
:107C300095F91030A96803EB830302EB8303052257
:107C4000ADF800208A07D3F8DC0011D502236A467C
:107C500001A966F01DFDAB689B071CD59DF805309A
:107C600003F0010383F0010084F8EC3002B070BD32
:107C70006B6913B11A689B885383144B14491A68B3
:107C8000144B4E68D200A3FB023292094B689B1B37
:107C90009A42FBD2DAE70D4B0D491A680D4B486842
:107CA0004FF4FA7606FB02F2A3FB023292094B680C
:107CB0001B1A9A42FBD26B69002BCFD01A689B88A3
:107CC0001383CBE7707F0020EC1800201C380020C5
:107CD000001000E0D34D6210244B254A30B5D3F894
:107CE000F04094F91030A16803EB830302EB8303A7
:107CF00083B08A078DF80700D3F8DC000AD501238A
:107D00000DF10702002166F0C3FCA3689B0714D5A0
:107D100003B030BD636913B11A689B885383154B58
:107D200015491A68154B4D68D200A3FB023292091F
:107D30004B685B1B9A42FBD2E1E70E4B0E491A6877
:107D40000E4B4FF4FA7000FB02F2A3FB02324868BC
:107D500092094B681B1A9A42FBD26369002BD7D059
:107D60001A689B88138303B030BD00BF707F00206A
:107D7000EC1800201C380020001000E0D34D6210E9
:107D80002DE9F04383B0002862D1344DD5F8F4607A
:107D900095F8EC30324F334CDFF8D48033B9002300
:107DA0000120C5F8F43003B0BDE8F083D5F8F090B9
:107DB00099F91030D9F8082003EB830307EB83030C
:107DC00005219207D3F8DC00ADF8001018D5022386
:107DD0006A4601A966F05CFCD9F808309B0721D5FA
:107DE0009DF8053003F0010385F8EC30002BD6D068
:107DF0001D4A12689642D1D8002003B0BDE8F08336
:107E0000D9F8143013B11A689B885383174B6168F3
:107E10001A68D200A8FB0232920963685B1A9A4280
:107E2000FBD2D4E7114B61681A684FF4FA7303FB75
:107E300002F2A8FB0232920963685B1A9A42FBD2F3
:107E4000D9F81430002BCBD01A689B881383C7E76E
:107E5000054B024D1E6806449AE700BF707F002064
:107E6000EC180020001000E0F83600201C3800203C
:107E7000D34D621010B50020FFF782FF00B910BD8E
:107E8000084C0620FFF728FF0123C72084F8EC30B8
:107E9000FFF722FF044B1B6803F5A4430833C4F823
:107EA000F43010BD707F0020F8360020F0B5044695
:107EB00089B000200E461546FFF762FF10B9204634
:107EC00009B0F0BD1D4F0620FFF706FF012387F81C
:107ED000EC3097F8F820CDF80CD002230093002363
:107EE0008DF804300293E2B1CDE9066505930522D1
:107EF000230E8DF8013004920DF10203220C1A704A
:107F0000D7F8F0009C70220A5A700379022B10D027
:107F10000B4B1B682C4406332046C7F8F43009B0DD
:107F2000F0BDCDE90526042207950DF10103049269
:107F3000E4E702A966F0FCFBEAE700BF707F0020DF
:107F4000F836002070B5054688B000200E4614466D
:107F5000FFF716FFE8B103220092174ACDF80CD0C4
:107F600092F8F81000238DF80430029399B9CDE906
:107F70000561042107940DF101030491D2F8F0008A
:107F80009D702A0C1A702A0A5A700379022B0DD0A0
:107F9000204608B070BD290E8DF801100521CDE9ED
:107FA000063405960DF102030491E7E702A966F095
:107FB000BFFB2046EDE700BF707F0020F0B5044610
:107FC00083B00020FFF7DCFE08B903B0F0BD374DE9
:107FD0000620FFF781FED82295F8F83000920121A3
:107FE000002285F8EC108DF804204BB3230A210EF3
:107FF000220CD5F8F0608DF803308DF801108DF863
:1080000002208DF80440052396F91020284902EB40
:10801000820201EB8202B168D2F8DC008A071BD52C
:108020006A46002166F034FBB3689B0727D5214BD5
:108030001B6803F59C530833C5F8F43003B0F0BD5A
:10804000230A220C8DF80230D5F8F0608DF801205B
:108050008DF803400423D7E7726912B11168928842
:108060004A83154A154C1168154A6768C900A2FB76
:10807000012189096268D21B9142FBD2D0E70E4BE5
:108080000E491A680E4B48684FF4FA7404FB02F26A
:10809000A3FB023292094B681B1A9A42FBD2736906
:1080A000002BC4D01A689B881383C0E7707F002020
:1080B000EC180020F83600201C380020001000E0EA
:1080C000D34D62102DE9F0410C4E356873691D40A7
:1080D00011D0DFF82C800127B5FA85F4C4F11F0414
:1080E00008EB840307FA04F4D3F8FC00036898470C
:1080F000A5437461F0D1BDE8F08100BF003C0140B0
:10810000707F002010B50B4CD4F83C0128B10A4A0E
:108110000321FAF727F9D4F83C010021FAF79EF978
:10812000D4F83C010549BDE8104040F62B4263F00D
:108130007DBE00BF707F0020009F240008A90020A2
:1081400010B5114CD4F83C0128B1104A6421FAF75B
:1081500009F9D4F83C010021FAF780F9D4F83C3150
:108160005B681A68B2F844306FEA43436FEA5343DE
:108170009BB2A2F84430138801219BB20B431380B9
:1081800084F8401110BD00BF707F0020009F2400C4
:1081900030B52DED028B574C94F86431022B85B02D
:1081A00019D0DFED557A79B19FED547A9FED546A7D
:1081B000DFED546A67EEA77A67EE877A87EE867AF4
:1081C00077EE267AC1ED007A0AB14F4B136005B005
:1081D000BDEC028B30BD94F808326BBB4B4B5B6837
:1081E0009B072DD5B4F9EC3100EE103AB4F9EA3121
:1081F000B8EEC00A07EE103A20EE000AB8EEC77AD1
:10820000B4F9EE31A7EE070A07EE903AF8EEE77AF6
:10821000A7EEA70AB5EEC00AF1EE10FAC1DBB5EE83
:10822000400AF1EE10FA5BD4F1EEC07AF4EE677A10
:10823000F1EE10FAB7D7B4E7344B5B68980704D473
:10824000D4F80432D3ED347AADE7314D0DF10E00A0
:10825000CDE900122DF090FBBDF80E30D5F8EC03FF
:10826000DFED2C5ADFED2C6A9FED2C7A1B1A07EEFE
:10827000903AF8EEE77AB0EE408A87EEA56ADDE93B
:108280000012A6EE267AFDEEC77AB0EE470A17EE88
:10829000903A2033402B20D8FDF7BEFBDDE90012D9
:1082A0001F4BD4ED727A6C7CA3F144001D462C3B2D
:1082B000002C08BF034695ED007AD3ED056AA8EEC1
:1082C000407A37EEA60A20EE000AA7EE070AB5EEBE
:1082D000C00AF1EE10FAA2DA63E79FED070ADFE7C2
:1082E000CDE9001268F0B0FADDE90012F0EE407A54
:1082F0009CE700BF707F002000000000CDCC9C3FB9
:1083000000409C4682E6C547331390439C00001012
:10831000F09700200000C84235FA8E3CDB0FC93FC1
:10832000F09B002010B50446C06900B110BD0921C2
:108330001420FDF7C7FEE06110BD00BF10B5174C5B
:1083400054F8200030B300EB400004EB800393F9B5
:108350000DC2BCF1FF3F1ED093F81502D0B104EB63
:108360000C0293F8140292F860E28C23142103FBB0
:108370000CFC00220CEB000304EB43030139B3F8BF
:108380006432704412FA83F2F4D10548A0FB023043
:10839000C0F30F1010BD002010BD00BF707F002083
:1083A000CDCCCCCC30B5032083B00D461446FFF7BE
:1083B000C5FF01909DB107EE900A9FED0B7AF8EE94
:1083C000677AF0EE006A67EE877AB8EE047AA7EE75
:1083D000A67ADFED067A67EE277AC5ED007A0CB152
:1083E000034B236003B030BD6740533A00007A442A
:1083F0003313904328B30368124A30B503F13F4367
:1084000003F57E039B0A054683B00C46D05C63F0FF
:1084100079FCA988009104F00303C4F381028DF86C
:10842000043028688DF80520C4F300136946C4F3AE
:1084300041148DF806308DF80740FAF773FB03B04E
:1084400030BD7047AC65070870B5114B114CA342A5
:1084500003D319E00C33A34216D293F805C08C4520
:10846000F8D193F804C0844501D00028F2D193F8E4
:1084700007E09645EED11D6895F804E0E645E9D1A0
:108480002E689E42E6D100E00025284670BD00BF60
:108490006C970808689808080379022B00D0704789
:1084A00010B590F91020224882B002EB8202083108
:1084B000694403244FF0000C4FF0010E00EB8202E0
:1084C0008DF800C08DF801E08DF802308DF8034082
:1084D000D2F8DC2011F8084C16498A4223D0A1F5C5
:1084E00078418A4221D001F580618A4219D11188F0
:1084F00021F04001090403EB8303090C118000EB18
:1085000083001388D0F8E81023F0380331F82410E2
:108510001B041B0C0B43138013889BB243F04003D6
:10852000138002B010BD6346E1E77346DFE700BF8A
:10853000EC1800200030014070B50446244894F93E
:108540001030A66803EB830300EB83031546B207E4
:10855000D3F8DC0082B00CD5019066F037F90198B1
:10856000294666F033F9A3689B0717D5012002B0AE
:1085700070BD636913B11A689B885383154B164A03
:108580001B6856684FEAC30C144BA3FB0C3C4FEA24
:108590009C1C53689B1B9C45FBD2DDE70D4B0E4991
:1085A0001A680E4B4FF4FA7000FB02F2A3FB023282
:1085B000486892094B681B1A9A42FBD26369002BE8
:1085C000D4D01A689B881383012002B070BD00BF0D
:1085D000EC1800201C380020001000E0D34D621081
:1085E00010B50379012B84B08E460DD0022B08D133
:1085F0008368DB0758BF01F07F0104B0BDE810407D
:108600009AE7002004B010BD144682688DF80F4030
:1086100002F0010201920DF10F020092417C90F9EB
:1086200010007246FBF758FD04B010BD10B50446AB
:10863000002221210068FFF7D3FF2068FC222021BF
:10864000FFF7CEFF206840222421FFF7C9FF2068F2
:108650000C222321FFF7C4FF206800222221FFF70C
:10866000BFFF012010BD00BF10B5044694220B21AE
:108670000068FFF7B5FF206871220121FFF7B0FF06
:10868000206800220421FFF7ABFF2068C8220521E3
:10869000FFF7A6FF206800220621FFF7A1FF206850
:1086A000C8220721FFF79CFF206800220821FFF75E
:1086B00097FF2068C8220921FFF792FF012010BD13
:1086C00010B504682379012B84B00ED0022B09D198
:1086D000A368DB074FF031024CBFF4217421204620
:1086E000FFF72AFF012004B010BDA268617C94F955
:1086F000100002F0010201920DF10F0200923124EC
:10870000F4228DF80F40FBF7E7FC012004B010BD08
:1087100010B504682379012B84B00BD0022B06D14D
:108720001A460821204604B0BDE8104004E70020A6
:1087300004B010BDA268617C94F9100002F001023F
:1087400001920DF10F020092022408228DF80F40D1
:10875000FBF7C2FC04B010BD10B504682379012BEF
:1087600084B00BD0022B06D101220821204604B090
:10877000BDE81040E0E6002004B010BDA26894F906
:108780001000617C8DF80F3002F0010201920DF1B2
:108790000F0200920822FBF79FFC04B010BD00BF3F
:1087A00030B505682B79012B85B0044611D0022B1A
:1087B0000CD101220B212846FFF7BEFE30B1206804
:1087C0001D22092105B0BDE8304009E7002005B0B1
:1087D00030BDAA6895F91000697C8DF80F3002F061
:1087E000010201920DF10F0200920B22FBF774FCC3
:1087F000E4E700BFF0B5054690F91000254C00EB0A
:10880000800004EB8000AC68D0F8DC00A40785B0E1
:1088100010D5CDE90223019065F0D8FFDDE90223F0
:108820000198002165F034FFAB689B0718D5012043
:1088300005B0F0BD6C6914B12668A4887483164C29
:10884000164E246877684FEAC40E154CA4FB0E4EF2
:108850004FEA9E1E7468A4EB070CE645FAD2D8E7EF
:108860000D4B0E491A680E4B4FF4FA7000FB02F2E2
:10887000A3FB0232486892094B681B1A9A42FBD24A
:108880006B69002BD3D01A689B881383012005B035
:10889000F0BD00BFEC1800201C380020001000E0E4
:1088A000D34D621030B50579012D83B08E460DD0C1
:1088B000022D08D18468E40758BF41F0800103B05D
:1088C000BDE8304096E7002003B030BD1446826812
:1088D000009402F00102417C90F91000019272466E
:1088E000FBF7FAFB03B030BD10B5174C84F8AD159B
:1088F000017984F8AE2501294FF0000282B084F896
:10890000AC2512D002290CD1032304F2AC52FF2172
:10891000FFF770FF002814BF00206FF00C0002B0BA
:1089200010BD6FF00C0002B010BD8268417C90F960
:10893000100004F2AC5402F00102CDE9004203231E
:10894000FF22FBF7C9FBE5E7707F00200068037991
:10895000012B0AD0022B07D183680E4A13F00103C2
:1089600015D00023512145E7704700B58368094AB7
:10897000417C90F9100083B003F00103CDE900239E
:1089800000235122FBF7A8FB03B05DF804FBD121C3
:1089900030E700BF1C860020F0B50546164695F965
:1089A0001020254802EB820200EB820283B0D2F84D
:1089B000DC00AA6892070FD5CDE9000365F006FF39
:1089C000019B00980022314665F062FEAB689B0770
:1089D00018D5012003B0F0BD6A6912B114689288FD
:1089E0006283164A1468164A4FEAC40E154C57683B
:1089F000A4FB0E4E4FEA9E1E5468A4EB070CE645FE
:108A0000FAD2D9E70D4B0E491A680E4B4FF4FA70A3
:108A100000FB02F2A3FB0232486892094B681B1A62
:108A20009A42FBD26B69002BD3D01A689B881383C0
:108A3000012003B0F0BD00BFEC1800201C3800205E
:108A4000001000E0D34D621030B50579012D83B0E0
:108A50008E460DD0022D08D18468E40758BF41F03E
:108A6000800103B0BDE8304096E7002003B030BD80
:108A700014468268009402F00102417C90F91000D3
:108A800001927246FAF722FF03B030BD10B50446DA
:108A90000068037982B0022B0CBF43210321062317
:108AA0006A46FFF7D1FF68B1BDF80010BDF802209B
:108AB000BDF8043049BA52BA5BBAE18662872387AF
:108AC00002B010BDE086A06302B010BDF0B506682C
:108AD000F56983B00446002D65D000232B70042374
:108AE0000DEB03023046FF21FFF7AEFF10B9002067
:108AF00003B0F0BD206804236A46FF21FFF7A4FFFE
:108B00000028F4D09DF804108A09023A012AEED90F
:108B10009DF8053003EB012343F6FF74C3F30D0307
:108B2000A342E4D0002BE2D09DF806109DF8072068
:108B300002EB012240F2FF71B1EB521F4FEA6216C5
:108B4000D5D0002ED3D09DF800C09DF8012002EBB7
:108B50000C22C2F30D02A242C9D0002AC7D09DF850
:108B600002709DF8034004EB0724B1EB541F4FEA59
:108B70006417BCD0002FBAD0991A0029B8BF494257
:108B8000FF29B4DCF11B0029B8BF4942FF29AEDC44
:108B900013445B10F2195210C5F805300123C5F8D3
:108BA00001202B70A4E709211420FDF78BFAF06156
:108BB0000546266891E700BF70B50668F46982B083
:108BC0000CB30025042325700DEB03023046FF2172
:108BD000FFF73AFFA8B19DF804108B091CD19DF84E
:108BE00005209DF806509DF8073002EB012292B255
:108BF00003EB0523C4F805205B1101222270C4F8A1
:108C0000013002B070BD054609211420FDF75AFA63
:108C1000F06104462E68D4E7034A04210320FDF7DF
:108C200073F9284602B070BDA81608082DE9F04176
:108C3000114C04F2AC5884F8AD15174600250223F8
:108C40004246FF21064684F8AC55FFF72BFE80B163
:108C5000424630460223FF21FFF7F6FE48B194F862
:108C6000AC2594F8AD3503EB022328463B80BDE8E4
:108C7000F0816FF00C00FAE7707F002030B5184DDE
:108C800095F8C23083B00BB903B030BD04460DF186
:108C90000501006864F0C8FB9DF8053073B9012137
:108CA0002068104A85F8AE154FF406440323FF21CF
:108CB000A5F8AC45FFF7F6FD03B030BD0DF1060297
:108CC00096212068FFF7B2FF074ABDF80630074932
:108CD000A2FB0323DB0801228B6185F8C320DEE7BA
:108CE000707F00201C850020CDCCCCCCEC1800205F
:108CF00010B5044600680379012B84B02DD0022BF7
:108D000028D1836813F0010F02AA4FF0060314BFA5
:108D10001F219F21FFF740FED0B1BDF80810BDF81C
:108D20000A20BDF80C30C9BA07EE901AD2BAF8EE94
:108D3000E76A07EE902ADBBAB8EEE77A07EE903AD8
:108D4000F8EEE77AC4ED046A84ED057AC4ED067A9C
:108D500004B010BD002004B010BD8368417C90F9C0
:108D6000100003F00103019302AB00931F220623BE
:108D7000FAF7ACFDD0E700BF10B5044600680379F0
:108D8000012B84B02DD0022B28D1836813F0010F62
:108D900002AA4FF0060314BF2521A521FFF7FCFD11
:108DA000D0B1BDF80810BDF80A20BDF80C30C9BA22
:108DB00007EE901AD2BAF8EEE76A07EE902ADBBA0D
:108DC000B8EEE77A07EE903AF8EEE77AC4ED076A74
:108DD00084ED087AC4ED097A04B010BD002004B017
:108DE00010BD8368417C90F9100003F001030193EA
:108DF00002AB009325220623FAF768FDD0E700BFF7
:108E000070B50668F46982B00546002C3FD033790E
:108E1000012B04F1040205D0022B2CD00020A070FD
:108E200002B070BDB368717C96F91000009203F037
:108E3000010301933B220E23FAF748FDA07000289E
:108E4000EED0A389DBBA07EE903AF8EEE77AC5EDEB
:108E5000077AE389DBBA07EE903AF8EEE77AC5EDD8
:108E6000087A238ADBBA07EE903AF8EEE77AC5ED86
:108E7000097A02B070BDB36813F0010F30464FF0AD
:108E80000E0314BF3B21BB21FFF786FDD6E7092166
:108E90001420FDF717F90446F061B8E700B5006843
:108EA0000379012B85B032D0022B25D1062302AAEB
:108EB000F721FFF771FDF8B19DF809209DF808C072
:108EC0009DF80A109DF80C309DF80BE0120142EA63
:108ED0000C3242EA111215491B010A63C1F8AC2693
:108EE0009DF80D2043EA0E3343EA12130B61C1F8DB
:108EF000B03605B05DF804FB0C4BD3F8AC16D3F8D4
:108F0000B026196300201A6105B05DF804FB836880
:108F1000417C90F9100002AA03F00103CDE900237F
:108F20000623F722FAF7D2FCC5E700BF707F0020C6
:108F300010B500680379012B84B029D0022B24D10D
:108F4000836813F0010F4FF0030303AA14BF1946FF
:108F50008321FFF721FDB0B19DF80C309DF90C1075
:108F60009DF80D209DF80EC01B04002943EA022342
:108F7000B8BF4FF07F410D4AA8BF002143EA0C0360
:108F80000B43C2F8E83004B010BD002004B010BD9F
:108F90008268417C90F9100002F00102032303ACC7
:108FA000CDE900421A46FAF791FCD4E7707F002021
:108FB00000B500680379012B85B02BD0022B25D199
:108FC000836813F0010F03AA4FF0030314BF0021BD
:108FD0008021FFF7E1FCB0B19DF80C309DF90C1039
:108FE0009DF80D209DF80EC01B04002943EA0223C2
:108FF000B8BF4FF07F410E4AA8BF002143EA0C03DF
:109000000B43C2F8CC3005B05DF804FB002005B07E
:109010005DF804FB8368417C90F9100003AA03F01B
:109020000103CDE9002303230022FAF74FFCD2E726
:10903000707F002010B5044600680379012B84B0CE
:109040003DD0022B36D1836813F0010F02AA4FF0F6
:10905000060314BF11219121FFF79EFC50B3BDF907
:10906000083006EE903ABDF90A30F8EEE66A07EEEF
:10907000103ABDF90C30B7EE086A07EE903A66EE8A
:10908000866AB8EEC77AFDEEE66A27EE067AF8EE53
:10909000E77A16EE903A67EE867ABDEEC77AFDEE75
:1090A000E77AE38617EE103A238717EE903A638744
:1090B00004B010BD0020E086A06304B010BD83683A
:1090C000417C90F9100003F00103019302AB00937F
:1090D00011220623FAF7FAFBC0E700BF10B50446D9
:1090E00000230068E386A3630279012A84B022D0BA
:1090F000022A1DD1836813F0010F02AA4FF0060364
:1091000014BF03218321FFF747FC78B1BDF90A3072
:10911000BDF80810BDF80C205B4201EB410103EBE8
:10912000430302EB4202E1862387628704B010BD4D
:10913000184604B010BD8368417C90F9100003F01C
:109140000103019302AB009303220623FAF7BEFB4F
:10915000DBE700BF70B500240668C48684633379FA
:10916000012B84B005461CD0022B17D1B36813F035
:10917000010F02AA4FF0060314BF2146802130469A
:10918000FFF70AFC40B1BDF80810BDF80A20BDF891
:109190000C30E9862A876B8704B070BD204604B086
:1091A00070BDB368717C96F9100003F00103019360
:1091B00002AB009322460623FAF788FBE2E700BFE2
:1091C00010B584B00023044600680293ADF80C305B
:1091D0008DF80E300279012A1ED0022A19D1836837
:1091E00013F0010F02AA4FF0070314BF4E21CE2146
:1091F000FFF7D2FBBDF80910BDF80B20BDF80D300C
:10920000C9BAD2BADBBA0120E1862287638704B0EB
:1092100010BD1A461946F6E78368417C90F91000A4
:1092200003F00103019302AB00934E220723FAF7E8
:109230004DFBDFE700B500680379012B85B00DD049
:10924000022B07D1012303AAFF21FFF7A5FB05B0DD
:109250005DF804FB002005B05DF804FB8268417CEA
:1092600090F9100002F00102019203AA0092FF227D
:10927000FAF72CFB05B05DF804FB00BF30B50446DF
:1092800000680379012B85B029D0022B1ED182689A
:1092900012F0010F18BF512103AA08BFD121FFF717
:1092A0007BFB98B1BDF80C30194A5BBA9BB2D36115
:1092B000D369B3F5C87F0EDC1649174AD1F8B43626
:1092C00015683233AB4218D305B030BD104B6FF088
:1092D0000102DA61F0E74FF0FF33D361ECE7836816
:1092E000417C90F9100003F00103019303AB00935C
:1092F00051220223FAF7EAFAD3E701F2AC62C1F88D
:10930000B456206800235121FFF7CCFA05B030BDD8
:10931000EC180020707F0020F836002000B50068AF
:109320000379012B85B008D0022B2FD0204B0022CF
:1093300083F8C82005B05DF804FB8368417C90F990
:10934000100003F0010303AACDE900230223002249
:10935000FAF7BCFA164B83F8C8000028EAD0BDF82B
:109360000C305BBA9BB2B3F5FA6F1AD21149124AAC
:10937000A1FB0313DB0807EE903AF8EEE77AFDEE67
:10938000E77AC2ED087A05B05DF804FB826812F056
:10939000010F18BF002103AA08BF8021FFF7FCFAC4
:1093A000D8E7054B4FF0FF321A6205B05DF804FBB9
:1093B000707F0020CDCCCCCCEC18002010B500681C
:1093C0000379012B84B00C461DD0022B18D1826882
:1093D00012F0010F14BF0021802103AAFFF7DCFA6D
:1093E00060B15CB19DF80D309DF90C20DB0903EBF9
:1093F000830302EB820203EB4203238004B010BD1F
:10940000002004B010BD8368417C90F9100003F087
:109410000103019303AB009300220223FAF756FAEB
:109420000028DED1EAE700BF70B50446254894F96C
:109430001030A66803EB830300EB83031546B207E5
:10944000D3F8DC0082B00ED5019065F0BFF901239E
:1094500001980022294665F01BF9A3689B0717D5E0
:10946000012002B070BD636913B11A689B885383F1
:10947000154B164A1B6856684FEAC30C144BA3FBE6
:109480000C3C4FEA9C1C53689B1B9C45FBD2DBE7C2
:109490000D4B0E491A680E4B4FF4FA7000FB02F2A6
:1094A000A3FB0232486892094B681B1A9A42FBD20E
:1094B0006369002BD4D01A689B881383012002B003
:1094C00070BD00BFEC1800201C380020001000E028
:1094D000D34D621010B50379012B82B08E460DD0AA
:1094E000022B08D18368DB0758BF41F0800102B02E
:1094F000BDE8104098E7002002B010BD1446826815
:10950000009402F00102417C90F910000192724631
:10951000FAF7DCF902B010BDF0B583B015460DF1D5
:1095200007021C4606460F46FFF7D4FF9DF80720AA
:1095300005EA0203A34201D103B0F0BD22EA05020D
:1095400022433946304603B0BDE8F040FFF748B843
:1095500030B5002385B00446C38683630DF107024E
:1095600000680221FFF7B6FF18B19DF80730DB074E
:1095700003D40025284605B030BD0623032102AAE6
:109580002068FFF761FA20680DF107020921FFF753
:10959000A1FF05460028ECD09DF8073013F00C0F12
:1095A000E7D1BDF80820BDF80C30BDF80A102068DE
:1095B000C2EB8232C3EB83339B0092008900E286C8
:1095C0002187638701220A21FFF70AF8284605B0A0
:1095D00030BD00BFF0B5484D95F8C03083B03BB109
:1095E00095F8B866012E044656D0022E36D00EB13C
:1095F00003B0F0BD012280210068FEF7F1FF206872
:109600000122FF21FEF7ECFF324631462068FEF7CB
:10961000E7FF95F8B92620689121FEF7E1FF314672
:1096200020680122FEF7DCFF32462068FF21FEF7AA
:10963000D7FF324620688021FEF7D2FF31462068EE
:109640000122FEF7CDFF2D4B2D491A680874012326
:10965000C5F8BC2685F8B83603B0F0BD0068284FC1
:1096600001AA1321FFF736FF9DF8043038745B0719
:1096700025D1D5F8C036002BBAD0204AD5F8BC1673
:10968000126892B2521A9342B2D24FF0FF320023C4
:109690007A6185F8B836ABE701AA0068184F002157
:1096A000FFF718FF9DF804303874DA07E1D4134A45
:1096B00002231268C5F8BC2685F8B83698E72068FA
:1096C000334601AA1E21FFF7BFF9BDF80430206818
:1096D00001220B215CBAFEF783FF0A4B3874A4B257
:1096E000A3FB0434E408012200237C6185F8C12037
:1096F00085F8B8367CE700BF707F0020F836002080
:10970000EC180020CDCCCCCC30B505682B79012BE2
:1097100085B0044600F09280022B08D1AB68DB07CD
:1097200002AA4CBF082188212846FFF77DFE9DF83C
:10973000083013F0100302D1184605B030BD206880
:10974000062302AA0021FFF77FF90028F5D09DF833
:1097500009209DF808109DF80A309FED3F6A12021B
:1097600002EB01421344140248BF03F17F4307EEAA
:10977000903AF8EEE77A9DF80C109DF80B409DF8B2
:109780000D20364BC7EE866A090201EB04410A44FC
:10979000090248BF02F17F4207EE902AB3F9482040
:1097A00007EE102AB3F94420F8EEE77A05EE102A06
:1097B00087EE864AB3F94020B8EEC77AB8EEC55AAC
:1097C000D3ED0F7AA6EE875AF8EEE75A04EE902A08
:1097D000E6EE855AB3F94620D3ED0E7A03EE902AD1
:1097E000F8EEE77AB3F94220E6EEA57A06EE102A03
:1097F000B3F93620F8EEE44AF8EEE33A07EE102A21
:10980000B8EEC66AB3F93420A6EEA36AE4EE247A71
:1098100005EE902AB8EEC77A66EE846AF8EEE55A4D
:1098200027EE047AB6EE005AA5EE857AE6EE867A41
:1098300083ED147AC3ED137A05B030BDAA68697C54
:1098400095F9100002F00102019202AA009208228A
:10985000FAF73CF86BE700BF00007848707F002003
:1098600070B505682B79012B84B0044662D0022BB9
:1098700010D1AA6802AE12F0010F18BF1946324685
:1098800008BF82212846FFF7CFFD18B19DF80830A8
:10989000DA0703D40025284604B070BD20680723EA
:1098A00032460321FFF7D0F805460028F2D02068A1
:1098B00011220A21FEF794FE9DF80E301B07E9D411
:1098C0002949BDF80830B1F8C42613FB02F3274A32
:1098D00093423EDBB3F5000F39DA002BB8BFFF33FC
:1098E0001B125B421BB2BDF80A20E386B1F8C636F4
:1098F00012FB03F31D4A93422FDBB3F5000F30DA5E
:10990000002BB8BFFF3343F30F22BDF80C30B1F882
:10991000C8162287154A13FB01F393421BDBB3F5EC
:10992000000F1CDA002BB8BFFF331B125B421BB2C7
:109930006387B0E7AA68697C95F9100002F001021C
:1099400002AE019200960222F9F7C0FF9DE7084B94
:10995000C9E7084BC7E7074BEAE7064AD5E7044BD8
:10996000E6E747F6FF72D0E7707F002001FF7FFF38
:109970000180FFFF0080FFFF30B505682B7987B0BD
:109980000022012B04468DF80F2035D0022B12D176
:10999000AB68DB070DF10F024CBF2721A72128463A
:1099A000FFF742FD28B19DF80F3013F0080305D1F1
:1099B000184607B030BD104607B030BD20680623FA
:1099C00004AA2821FFF740F820B3BDF91030BDF9F3
:1099D0001220002BB8BF03339B10E386BDF914306F
:1099E000002AB8BF0332002BB8BF033392109B107C
:1099F0002287638707B030BDAA68697C95F910009B
:109A000002F0010201920DF10F0200922722F9F7F4
:109A10005DFFC7E7E086A06307B030BD30B50546FF
:109A200000240068EC86AC630379012B87B02AD050
:109A3000022B0ED18368DB070DF10F024CBF2146CC
:109A40008021FFF7F1FC28B19DF80F4014F00804C5
:109A500002D1204607B030BD2868062304AA0121A0
:109A6000FEF7F2FF0028F5D0BDF81430BDF8101055
:109A7000BDF812205BBA49BA52BA5B42E9862A871E
:109A80006B8707B030BD22468468417C90F9100096
:109A900004F0010401940DF10F040094F9F716FF8E
:109AA000D1E700BF30B5044600202568E086A063FA
:109AB0002B79012B87B027D0022B10D1AB68DB07A5
:109AC0000DF10F024CBF062186212846FFF7ACFCA2
:109AD00028B19DF80F3013F0040302D1184607B0E7
:109AE00030BD2068062304AA0021FEF7ADFF002840
:109AF000F5D0BDF81010BDF81220BDF81430E18685
:109B00002287638707B030BDAA68697C95F9100089
:109B100002F0010201920DF10F0200920622F9F704
:109B2000D5FED5E730B5054600202C68E886A86349
:109B30002379012B87B046D0022B0FD1A368DB0716
:109B40000DF10B024CBF3421B4212046FFF76CFC11
:109B500020B19DF90B30002B02DB002007B030BD97
:109B600028680379012B3CD0022BF6D1836813F0CF
:109B7000010F03AA4FF0090314BF2421A421FEF70B
:109B80000BFF0028EAD09DF810209DF80F109DF8DB
:109B90001330120442EA0162C2F30F429DF8121020
:109BA0002A871B049DF80D2043EA01639DF80C10E1
:109BB000120442EA0162C2F30F42C3F30F43EA8682
:109BC0006B8707B030BDA268617C94F9100002F089
:109BD000010201920DF10B0200923422F9F776FE98
:109BE000B6E78368417C90F9100003F0010301930C
:109BF00003AB009324220923F9F768FEC1E700BFF5
:109C0000F0B541F0010285B00021294F294D2A4EBF
:109C10000446FEF7E5FC3B68C6F8BC36287416E03F
:109C2000A368DB070DF10F024FF0130120465EBF62
:109C30000DF10F0293212046FFF7F6FB9DF80F3040
:109C4000287413F007030ED1D6F8C0263ABB237947
:109C5000012B16D0022BE3D09DF80F30002013F01B
:109C600007032874F0D001220B212046FEF7B8FC30
:109C7000002211462046FEF7B3FC2874012005B0EF
:109C8000F0BDA268617C94F9100002F0010201921B
:109C90000DF10F0200921322F9F718FECEE7396892
:109CA000D6F8BC0689B2091A8A42D0D21846E6E72D
:109CB000F8360020EC180020707F002010B50368F3
:109CC000DA6B82B0044612B1904740B123685B6BF7
:109CD0001BB1214601A8984718B9FF23E38202B0BF
:109CE00010BDBDF80630013B9BB2F7E7F0B585B07B
:109CF000044618460D461646039364F0EBFF2844CD
:109D00002768A073E673204600240094039B7C69B7
:109D100032462946A04705B0F0BD00BF38B504461D
:109D20008B6801600D46984700230B4A226123751A
:109D30002B6B13B1204698472075084B93F8CC360F
:109D40001BB1237D23F0010323750023E38220460A
:109D5000BDE83840B2E700BF0001FF00707F00207F
:109D600010B5154BD3F8D04684B024B12379012B1C
:109D700010D0022B02D0002004B010BDA16811F059
:109D80000101024618BF8021204604B0BDE8104002
:109D9000FEF7D2BBA268617C8DF80F0002F00102D1
:109DA00094F910000DF10F04CDE900428022FAF77A
:109DB00093F904B010BD00BF707F00202DE9F04181
:109DC000264ED6F8D05684B09DB1B02280212846C8
:109DD000FEF706FC402280212846FEF701FC002207
:109DE00080212846FEF7FCFB102280212846FEF742
:109DF000F7FB4FF480644FF000080DF10F0795B1A9
:109E00002B79012B15D0022B0DD1AB6813F0010378
:109E10004FF000024FF04001284602BF1A46402191
:109E20002846FEF789FB013CA4B29CB1D6F8D05677
:109E3000E5E7AA6895F91000697C8DF80F8002F0BB
:109E40000102013CCDE90072A4B24022FAF744F9C4
:109E5000002CEBD104B0BDE8F08100BF707F002082
:109E60000B4B10B5D3F8D0468CB15038C2B280211C
:109E70002046FEF7B5FB002280212046FEF7B0FB0E
:109E800020461022BDE810408021FEF7A9BB10BD7E
:109E9000707F0020F0B5204C204F203800EB800070
:109EA000661DD7F8D05685B004440644E5B12B7939
:109EB0002278012B1DD0022B0AD1AB6813F0010FC1
:109EC0004FF04001284604BF40212846FEF734FBEE
:109ED0000134B442EAD155B100224021284605B0F0
:109EE000BDE8F040FEF77CBB0134B442F0D105B0D0
:109EF000F0BD8DF80F20AA6895F91000697C02F07A
:109F0000010201920DF10F0200924022FAF7E4F8EB
:109F1000D7F8D056DCE700BFF4720708707F002046
:109F20002DE9F041734ED6F8D05684B0002D00F0E4
:109F30009680D42280212846FEF752FB80221146CB
:109F40002846FEF74DFBA82280212846FEF748FB55
:109F50003F2280212846FEF743FBD322802128465A
:109F6000FEF73EFB002280212846FEF739FB402207
:109F700080212846FEF734FB8D2280212846FEF7FB
:109F80002FFB142280212846FEF72AFBA1228021E4
:109F90002846FEF725FBC82280212846FEF720FB35
:109FA000DA2280212846FEF71BFB12228021284658
:109FB000FEF716FB812280212846FEF711FBCF22F7
:109FC00080212846FEF70CFBD92280212846FEF787
:109FD00007FBF12280212846FEF702FBDB228021CD
:109FE0002846FEF7FDFA402280212846FEF7F8FABF
:109FF000A42280212846FEF7F3FAA62280212846D3
:10A00000FEF7EEFAAF2280212846FEF7E9FAA622F3
:10A0100080212846FEF7E4FAAE2280212846FEF78A
:10A02000DFFA202280212846FEF7DAFA002280217A
:10A030002846FEF7D5FAB02280212846FEF7D0FA4E
:10A04000402280212846FEF7CBFA002280212846B4
:10A05000FEF7C6FA102280212846FEF7C1FA4FF417
:10A0600080644FF000080DF10F0755B32B79012BD9
:10A070002FD0022B0DD1AB6813F001034FF000027B
:10A080004FF04001284602BF1A4640212846FEF7FD
:10A0900053FA013CA4B2002CE7D175B18122802192
:10A0A0002846FEF79DFAC82280212846FEF798FA36
:10A0B000AF2280212846FEF793FA012004B0BDE8C4
:10A0C000F081013CA4B2002CE3D1012004B0BDE832
:10A0D000F081AA6895F91000697C8DF80F8002F074
:10A0E0000102CDE900724022F9F7F6FFD6F8D0560A
:10A0F000CFE700BF707F0020FDF7E4BFFDF7E2BFB0
:10A10000FDF7E0BFFDF7DEBFFDF7DCBFFDF7DABF0F
:10A1100070B5254D254E3622002105F2D4606BF036
:10A12000C1F9D6F82C3100209847044690B306F5C3
:10A130009672D6F84C31C5F80C27984783684BB314
:10A1400005F2D462B0F800C09646104600210678A9
:10A15000032E00F106001FD001310929F7D10CF1BF
:10A16000FF3080B200231178022902F1060209D0E3
:10A170000133092BF7D1D5F81037082B0AD05A1C18
:10A18000C5F81027062202FB03E302210022197002
:10A190005A809880204670BD062303FB0151B1F818
:10A1A000D606013880B2DDE7707F0020EC18002071
:10A1B0002DE9F041174DD5F80C3706463BB31B6A25
:10A1C00098470746D5F810377488012BB38813D009
:10A1D0009C420FD87868D5F80C3704FB00F0DB6898
:10A1E0009847D5F80C3700209B689847B38801340E
:10A1F000A342EFD2BDE8F08139885A1C121B8A4273
:10A20000E6D1D5F80C37BDE8F0411B69184705F2D7
:10A210001477D7E7707F002010B50409013C032CA8
:10A2200018D80E4A32F8141000F00F0341FA03F266
:10A2300012F0010210D0012098400138084065F06A
:10A24000D9FB074B074A1B5D184400EB400002EBAB
:10A25000800010BD002010BD104610BDDC72070844
:10A26000D8720708602C00202DE9F04F54220446D4
:10A270000021C14893B06BF015F9C049621EE01C83
:10A280000E460C4612F8013F5D1E052D88BF0023C7
:10A29000824244F8043BF5D1B94AA2F1100353F8C5
:10A2A000040B012800F050819342F8D151F8043B8F
:10A2B000022B00F040819142F8D10320FDF792F883
:10A2C0000420FDF78FF80520FDF78CF80620FDF738
:10A2D00089F8A94DDFF8C092DFF8C0821A2600275E
:10A2E0002C7B002C40D02046FFF796FF95F90DA05F
:10A2F0008346E0B10368A3498BF8076003F13F434D
:10A3000003F57E039B0A0522C85C8BF80620002318
:10A310008BF8083061F0F6FC9B4ABBF804300492DD
:10A32000DBF80000039303A9F8F7FCFB2C7B002368
:10A33000302201E019F8332094422ED00133102B43
:10A34000F8D100200AEB4A0A08EBCA030122D3F82D
:10A35000641128618C180720C3F864412975A87519
:10A360006A7583F8602117440136F6B2202E05F194
:10A370000C05B5D177B1854CDFF824A2DFF8249223
:10A380000025237C7BB90135032D04F118040AF55F
:10A390008C7AF6D113B0BDE8F08F7D4A02EBC3038F
:10A3A000D3F8B802CEE7607961F0ACFC207961F0B7
:10A3B000A9FCA068F8F720FB2368A068CDF814A0DA
:10A3C0004C3304936369142202FB03F307930023C5
:10A3D000CDE90E33CDE9103306930893E368039378
:10A3E0004FF480624FF40063CDE909234FF400512C
:10A3F0004FF48073CDE90B134FF4003303A90D9391
:10A4000061F0E8FCA2686349136843F0010313603C
:10A41000D9F8043023F4733323F4477323F0030390
:10A4200043F44033C9F80430226863695068012B53
:10A4300020F0407020F48070D4BF0026012640EA4E
:10A44000062050609068014041F002019160D16A9D
:10A45000013B21F47001DBB241EA0353D362464B66
:10A46000012103F148074FFA85F802E00C33BB42A3
:10A470002ED0587D0028F9D093F90D004045F5D134
:10A48000187C9E7D01F1010C09285FFA8CFC30D804
:10A4900000EB400E06FA0EF6D2F810B00196072631
:10A4A00006FA0EFE019E2BEA0E0E46EA0E06166115
:10A4B000062930D8013901EB81011F2688408E40E2
:10A4C0006146D2F834C02CEA060630435063CDE72B
:10A4D000936843F400739360936843F480739360CC
:10A4E000936843F001039360936843F08043936063
:10A4F00049E7A0F10A0E0EEB4E0E4FF0070B06FADD
:10A500000EF60BFA0EFED2F80CB02BEA0E0E46EA4F
:10A510000E06D660CCE70C291FD8073901EB810164
:10A520001F2688408E406146D2F830C02CEA0606CD
:10A53000304310639AE796F860323322013386F88D
:10A54000242286F86032B8E696F860323120013372
:10A5500086F8180286F86032A8E60D3901EB810111
:10A560001F2688408E406146D2F82CC02CEA060691
:10A570003043D0627AE700BF7C810020707F0020EA
:10A58000807F0020AC650708030001003C1A002012
:10A59000E4720708FDF7FFC098750708EC18002063
:10A5A000D48100200023014010B503681A79022AE3
:10A5B000044603D000232371236010BD987AFFF76F
:10A5C0002BFE0028F6D040F61A610022C1800272EC
:10A5D0002021FDF70FFF00232371236010BD00BF72
:10A5E00070B506461C48336803F13F4303F57E030C
:10A5F0009B0A82B0C05C0C46154661F083FBB288B2
:10A600000092B2FA82F304F003028DF80420C4F33E
:10A61000810230688DF80520C3F11F03C4F30012D6
:10A6200064098DF80740C3F3CC0400EB840403F005
:10A6300007038DF806209B00226A0F269D4006FA2C
:10A6400003F322EA03032362226A15436946256263
:10A65000F8F768FA02B070BDAC6507082DE9F04F55
:10A66000AC4CAD4DAC4283B050D21E4602E00C342F
:10A67000AC424BD294F805C08C45F8D194F804C094
:10A68000844501D00028F2D194F807C09445EED15A
:10A690002568002D3BD000236B60AB60EB602B6125
:10A6A0006B61AB61EB612C6022792A71A779AF6095
:10A6B000217AE960012A33D0022A27D1E07AFFF714
:10A6C000ABFD94F90980A861A07A85F81080FFF7A6
:10A6D000A3FD6861F8B1914C08EB880A04EB8A0A83
:10A6E0004FEA8809DAF8DC30ABB19AF8EE3003B300
:10A6F0000E2200238671C27103720921FDF77AFED2
:10A700006B6923B11A689B88138300E000252846F3
:10A7100003B0BDE8F08F2846FFF746FF0025F6E7B7
:10A72000E07AFFF779FD627AA37A6B74A8612A74E4
:10A73000EDE79AF8E40061F0E5FA9AF8E4104A09C6
:10A74000012301F01F01023A8B40032A08D8DFE8F9
:10A7500002F0AEB4A80272494A6922EA03034B61CF
:10A7600009EB080304EB830308F1010A93F8E10005
:10A77000FFF752FD5FFA8AFA014620B140F60A332C
:10A7800080F808A0C38009EB080304EB8303009161
:10A7900093F8E300FFF740FD0099034620B140F62F
:10A7A0000A5280F808A0C28009EB080204EB82027A
:10A7B000CDE9001392F8E200FFF72EFDDDE900136A
:10A7C000834620B140F60A4280F808A0C28009EB17
:10A7D000080204EB820217F0040A92F8E52072D016
:10A7E00039B108464A2101930092FFF7F9FEDDE9ED
:10A7F00000232BB118462A210092FFF7F1FE009AA0
:10A80000BBF1000F03D058460A21FFF7E9FE09EB20
:10A81000080B04EB8B0B9BF8E070002F6ED109EB5B
:10A82000080304EB83033F4AD3F8DC30934200F083
:10A830009B803D4A934200F0AD803C4A934200F039
:10A840009E803B4A934200F084803A4A934275D0FE
:10A85000394A934200F0A9801A88BAF1000F02F435
:10A8600041510CBF032200220A4342F445721A8070
:10A870009A8B22F400621204120C9A8307221A8225
:10A880001A8892B242F040021A8077BBC8446869C5
:10A8900004EB8804012384F8EE3000283FF42DAF48
:10A8A00026E71F490A6922EA03030B6158E71C499E
:10A8B0004A6A22EA03034B6252E719490A6A22EA0A
:10A8C00003030B624CE739B108460A210193009259
:10A8D000FFF786FEDDE90023002B91D018460A2100
:10A8E0000092FFF77DFE009A8AE73846FFF794FC56
:10A8F0000028CBD0036882881A83C7E73846FFF761
:10A900008BFC00288BD09BF8E5200921FFF768FE1F
:10A9100085E700BF6C97080868980808EC180020C5
:10A92000003802400030014000380040003C004048
:10A9300000340140005001400054014002F56842DB
:10A94000516A41F480115162516A21F480115162BF
:10A9500082E702F58232516A41F400515162516A34
:10A9600021F40051516277E702F58432516A41F4D3
:10A9700080515162516A21F4805151626CE702F5B5
:10A98000FE32116A41F400411162116A21F4004162
:10A99000116261E702F50032116A41F480411162EF
:10A9A000116A21F48041116256E702F56442516A4E
:10A9B00041F400115162516A21F4001151624BE7D8
:10A9C000074B53F8203021B14BB11A689B88538351
:10A9D0007047002BFCD01A689B8813837047704720
:10A9E000C87207081D4B70B5D3F83C4174B193F899
:10A9F000403105465BB162685379032B2BD8DFE801
:10AA000003F021242702136840331D6070BDE06805
:10AA1000666881680A6822F001020A603168104A9B
:10AA2000767932F816608A8992B222EA06028A8121
:10AA300023740A8892B242F001020A800377FDF77C
:10AA40007FFBD8E713683433DFE713683833DCE77C
:10AA500013683C33D9E700231B60FFDE707F0020C2
:10AA6000E464070810B5224CD4F83C3183B194F863
:10AA700040216AB194F82427032A0AD0022A10D070
:10AA8000002384F84031FDF73DFB08B984F8250721
:10AA900010BD5A685379032B27D8DFE803F0232031
:10AAA0001D185A685379032B1FD8DFE803F00D0AED
:10AAB00007021368403300221A6010BD13683C334C
:10AAC000F9E713683833F6E713683433F3E71368AC
:10AAD000403364221A6010BD13683C33F9E71368F1
:10AAE0003833F6E713683433F3E700231B60FFDEE7
:10AAF000707F00202DE9F04F8A4B8B4C93F828A7EC
:10AB000093F8299793F82A87DFF824B283B00026B8
:10AB100003F22C7501964FF0010EAB78E978C3F182
:10AB2000FF039BB2002B49D10B4688468C460A4650
:10AB300089468A4601210191100240EA034017220A
:10AB400040EA0C0006EB020CACEB02030EFA02F139
:10AB50002A3301429BB214BF02210121013A44F879
:10AB60002310531CF0D1714B04351836AB42B6B2EA
:10AB7000D3D16C4A4FF44063A2F82C398023A2F859
:10AB80002E39019B2BB182F828A782F8299782F8E9
:10AB90002A87644C94F825376BB1D4F83C0150B146
:10ABA00040F62B41F7F774FDD4F83C0103B0BDE843
:10ABB000F04FF7F7A1BD03B0BDE8F08FB5F800C0C6
:10ABC000C3F1FF03ABFB0C7001FB03F340091B1245
:10ABD0000A46052800F2A280DFE800F08E7156399F
:10ABE0001F03ABFB0C084FEA5818C8EB0818ACEB76
:10ABF00088081FFA88F8C81AC8F13C0800FB08F852
:10AC0000ABFB08085FFA83F909EB58188A465FFA2C
:10AC100088F80121C44601918EE7ABFB0C02520972
:10AC2000C2EB0212ACEB820292B2A1EB030A02FB6E
:10AC30000AFAABFB0A2A5FFA83F909EB5A1A8C4627
:10AC40005FFA8AFA884601215246019174E7ABFB0C
:10AC50000C025209C2EB0212ACEB82091FFA89F90D
:10AC6000CA1AC9F13C0902FB09F9ABFB09295FFAD1
:10AC700083FA0AEB59198C465FFA89F98846012153
:10AC80001A4601914B4657E7ABFB0C025209C2EB47
:10AC90000212ACEB820292B2A1EB030802FB08F8AD
:10ACA000ABFB08285FFA83FA0AEB58181A465FFADA
:10ACB00088F80B4689460121C44601913CE7ABFB6D
:10ACC0000C025209C2EB0212ACEB820A1FFA8AFA9A
:10ACD000CA1ACAF13C0A02FB0AFAABFB0A2A5FFA5B
:10ACE00083F808EB5A1A5FFA8AFA9C4689460B46A3
:10ACF0000121524601911FE7A1EB03090CFB09F961
:10AD00005FFA83F8ABFB090908EB59195FFA89F977
:10AD10009C46012301938A464B460DE74B4652461B
:10AD2000C44609E7707F002008A900209C88002005
:10AD3000898888882DE9F041314F00243B461D79F0
:10AD4000232D03F1140304D00134092CF7D1BDE8FD
:10AD5000F08104EB840007EB8000FBF7F1F9DFF8EA
:10AD6000AC800646C8F83C010028F0D02846FFF722
:10AD700053FAC8F8300958B1142202FB047440F2A7
:10AD80001522C28000220272227A4A21FFF728FC93
:10AD900098F82437022B2AD0032B20D0FDF7B2F9E4
:10ADA00010B988F82507D2E7164843F2AC02002113
:10ADB0006AF078FB98F82437012B03D1124BFF225D
:10ADC000C3F8A82098F84031012288F82527002BE5
:10ADD000BDD1337C002BBAD1BDE8F0418AE6FDF746
:10ADE000AFF93046F7F73EFC64230360AFE7FDF7A9
:10ADF000A7F93046F7F736FC00230360A7E700BF4A
:10AE00008010002008A9002008D90020707F0020B1
:10AE10002DE9F04FA34FA7B000210A260C4607F6F4
:10AE200034154FF0050B01968DE097F8383D5E061E
:10AE300019D404F1020E43F04003BEF18C0F87F8E1
:10AE4000383D00F2E18004F1010C98340DEB040A66
:10AE50000CF198040DEB040C74464FF0040E0AF844
:10AE60008CEC0CF88C3C04F1020CBCF18C0F42F021
:10AE7000020E00F2C98004F198036B4403F88BECD6
:10AE800004F1040EBEF18C0F03F88CBC00F2BC8000
:10AE900004F19A060DEB060C4FF0060A0CF88CAC88
:10AEA00004EB0A0C4FEA8909BCF18C0F5FFA89F6B2
:10AEB00003F8891C00F2A88004F19C0EEE444FF0C8
:10AEC00007090EF88C9C04F1080EBEF18C0F03F8F4
:10AED000876C00F299800CF198060DEB060C0CF8CB
:10AEE0008CBC03F8852C04F10A028C2A00F28C80B9
:10AEF00004F1A0060DEB060E0EF88CAC03F8831CD3
:10AF000004F10C018C297FD804F1A20204F1A303FF
:10AF10006A446B4402F88C9C0C4603F88C8C410903
:10AF200000F01F0C55F82120012303FA0CF322EA4C
:10AF3000030345F82130019B013B01936CD0411C78
:10AF4000B1F5F07F68D23C222846FAF7A5F900282F
:10AF50005DDB07EB4003C0F30722B3F870395E07EF
:10AF6000C1B25FFA83F94FEA13283FF55EAF97F855
:10AF700038CD1CF0400F03D10CF0380ECE451BD05D
:10AF80002CF0780C4CEA030304F1020EDBB2BEF1A4
:10AF90008C0F87F8383D37D804F1010C98340DEB4D
:10AFA00004090CF198040DEB040C74464FF0040EE8
:10AFB00009F88CEC0CF88C3CA31C8C2B24D804F1E5
:10AFC00098060DEB060C0CF88B2C221D8C2A0CF825
:10AFD0008CBC19D804F19A036B444FF0060E03F8A9
:10AFE0008CEC0CF8891C04EB0E018C290CD804F1B4
:10AFF0009C0204F19D036A446B44072402F88C4CC4
:10B000000C4603F88C8C8AE76FF0004487E72046F3
:10B0100014B927B0BDE8F08FD7F8305D224A95F912
:10B020001030A96803EB830302EB83038A07D3F88C
:10B03000DC0023D5234603AA002163F029FBAB687B
:10B040009B0703D5012027B0BDE8F08F174B1849A7
:10B050001A68184B4FF4FA7000FB02F2A3FB02329D
:10B06000486892094B681B1A9A42FBD26B69002B05
:10B07000E8D01A689B8813830120CAE76B6913B173
:10B080001A689B885383094B09491A68094B4E6813
:10B09000D200A3FB023292094B689B1B9A42FBD25F
:10B0A000C8E700BF707F0020EC1800201C3800208B
:10B0B000001000E0D34D6210F0B52A4CD4F8300DEA
:10B0C00083B010B194F8363D0BB103B0F0BD0DF173
:10B0D00007028421012384F8363DFEF7FBF994F83A
:10B0E000382DD4F8300D42F004020421FDF778FA2F
:10B0F000D4F8300D0DF107028421FEF7EBF99DF82D
:10B10000073013F00406F3D1174D84F8383D31466B
:10B110003C2228466AF0C6F904F62E57314604F65A
:10B120006E1C01263CF8023F1A0A22F0200203F0AE
:10B13000040301F01F0013434FEA511E06FA00F00A
:10B1400001F1010104D055F82E30184345F82E00C6
:10B15000BC45E7D1FFF75CFE0028FBD184F8360D33
:10B1600003B0F0BD707F0020A488002070B5424D70
:10B17000D5F8304D82B0A4B395F8343D012B44D0BE
:10B18000022B30D1082194F910303C4A85F8371D44
:10B1900003EB830302EB830304208DF806008DF894
:10B1A0000700D3F8DC00A3688DF8051000228DF8A5
:10B1B00004209A0742D504230DEB0302002163F01B
:10B1C00067FAA3689B0722D52D483C22FF216AF02D
:10B1D00069F995F8353D23B9FFF76EFF012385F82E
:10B1E000353D02B070BD0DF10302A0212046FEF7EF
:10B1F00071F99DF8033003F00503012B37D0002BC4
:10B200002FD1D5F8304D0821BDE74821BBE71D4BB4
:10B210001D491A681D4B48684FF4FA7606FB02F286
:10B22000A3FB023292094B681B1A9A42FBD2636954
:10B23000002BC9D01A689B881383C5E7636913B1D3
:10B240001A689B8853830F4B0F491A680F4B4E683F
:10B25000D200A3FB023292094B689B1B9A42FBD29D
:10B26000A9E70B4A126840F2DC539A42B9D9D5F8E3
:10B27000304D482187E700BF707F0020EC18002088
:10B28000A48800201C380020001000E0D34D62107C
:10B29000F8360020F0B54B4B8BB04FF4005103F55E
:10B2A000707223F8021F9A42FBD1474E474C356813
:10B2B00004F63757323502E033689D4252D9D4F84C
:10B2C000300D3A468021FEF705F90028F4D110220E
:10B2D00003463F4E01250AE00EF8242C0132D2B27B
:10B2E000202A034601F8245C0CF1040C12D0981CAF
:10B2F00003F1280703F1290122280DEB070E694409
:10B300009C46E9D90132D2B26FF00043202AB446FC
:10B310001846ECD1BCF1220F51D800F128020DEBF8
:10B32000020003F1280201216A4400F8241C4C2188
:10B33000023302F8231CD4F8304D264994F910202A
:10B34000A56802EB820201EB8202D2F8DC00AA07B8
:10B3500022D501AA002163F09BF9A3689B0704D5BD
:10B360000BB0F0BD10220023B3E71B4B1B491A683A
:10B3700048684FF4FA7303FB02F24FF47A73B2FB9E
:10B38000F3F24B681B1A9A42FBD26369002BE7D099
:10B390001A689B881383E3E7626912B11168928887
:10B3A0004A830D4A0D4D11686E68C9004FF47A72D8
:10B3B000B1FBF2F16A68921B9142FBD2C9E76FF0D0
:10B3C0000043B8E7DE880020F8360020707F0020B8
:10B3D00001000080EC1800201C380020001000E064
:10B3E0002DE9F041334D95F8363D82B004460E46C6
:10B3F000002BFDD195F8372DD5F8300D194602F008
:10B40000F702012385F8363D85F8372DFDF7E8F87A
:10B41000E2B207460921D5F8300DFDF7E1F8B4F5A1
:10B42000807F3FD0D5F8300DDFF88C805022082186
:10B43000FDF7D6F8D5F8300D0DF10702A021FEF783
:10B4400049F848B9D8F83432B8F8382259690A426C
:10B4500014BF5A831A83EDE79DF8074014F02004C7
:10B46000F0D1E2B20A21D5F8300DFDF7B9F8321962
:10B47000D5F8300DC0210134FEF72CF8362CF0D170
:10B4800057B995F8372DD5F8300D02F0F702394647
:10B4900085F8372DFDF7A4F8002385F8363D02B076
:10B4A000BDE8F081D5F8300D40220A21FDF798F86B
:10B4B000B8E700BF707F0020602C00202DE9F04F1E
:10B4C000604E96F8364DC3B005460F46002CFDD1B0
:10B4D00096F8372DD6F8300D02F0F70201232146F9
:10B4E00086F8372D86F8363DFDF77AF8FF2D4FF0B8
:10B4F00009038DF8055088BFAD0801AA88BF05F083
:10B50000C008137098BFA04602234FF0000C4FF004
:10B510000A0B0DF1050A4FF00B0914E0B4F5827F18
:10B5200002F803B00AF8031017F80C3017D80CF122
:10B53000010CBCF1360F02F8059000F1060002F88C
:10B540000E30234614D09D1C48EA0C01B5F5827FCD
:10B5500003F104041846C9B203F1030EDED90CF15D
:10B56000010C6FF00044BCF1360F37482346EAD196
:10B57000B0F5827F63D8082111550DF10501A02097
:10B58000C8540233D6F8304D304894F9101001EB0E
:10B59000810100EB8101D1F8DC00A168890722D587
:10B5A000002163F075F8A3689B0731D5284CD6F8C5
:10B5B000300D0DF10302A021FDF78CFF48B9D4F83E
:10B5C0003432B4F8382259690A4214BF5A831A83B4
:10B5D000EDE79DF8033013F02003F0D186F8363DF7
:10B5E00043B0BDE8F08F616911B10D688988698346
:10B5F0001849194F0D681949D7F804C0ED00A1FB8F
:10B600000515AD097968A1EB0C018D42FAD2C7E7A7
:10B61000104B11491A68114B48684FF4FA7505FB35
:10B6200002F2A3FB023292094B681B1A9A42FBD228
:10B630006369002BBAD01A689B881383B6E76FF052
:10B6400000439FE7707F002001000080EC1800207D
:10B65000602C00201C380020001000E0D34D621048
:10B66000002ABCBF80185242002B30B53BDB5D186E
:10B670000028B7BF121A841814460020A4F11D0C2C
:10B680000029BCBF2B460021BCF1000FC8BFA2EBB4
:10B690000C04A5F10F02C8BF2418002AC4BF9B1ACE
:10B6A0005D1884421EDBC1F1010C114AAC44C1EBB0
:10B6B0000113CCEB0C1C00EB430301344FEA4C0CA0
:10B6C00002EB43024FF0200E8D42A8BF002304DBA3
:10B6D00022F813E01E339C45FAD10130A04202F15A
:10B6E0000202F1D130BD5C180D465B422146BFE736
:10B6F000E08800201B4B1C48196C1C4A10B441F018
:10B7000080510124196404625321FF24CA20546229
:10B71000506251625B6FDB0085B013D40023144983
:10B7200002930291029A134804320292029A136021
:10B7300003930391039B0393039B186005B05DF88B
:10B74000044B70470A4B002201920193019B019325
:10B75000019A084B12689A42E0D105B05DF8044B9B
:10B76000704700BF0038024000000E420028004031
:10B770005028004076614E6910B4674C0023224681
:10B7800092F90410012902F10C023CD00133072B7D
:10B79000F6D12246002392F90410022902F10C028C
:10B7A00047D00133072BF6D12246002392F904102B
:10B7B000032902F10C0257D00133072BF6D12246A0
:10B7C000002392F90410042902F10C0260D0013325
:10B7D000072BF6D1002394F90420052A04F10C0468
:10B7E0006AD00133072BF6D14C4B9B68DB037DD429
:10B7F00001795DF8044B01F0FD01A1F13100B0FACF
:10B8000080F040097047464A03EB430302EB830391
:10B81000D3F83C3D03B3434B93F83D2093F83CC031
:10B8200003799A4201D06345B3D101205DF8044BFE
:10B8300070473B4A03EB430302EB8303D3F83C3DE1
:10B8400063B1394B027993F83D1093F83C30914243
:10B85000EBD09A42A8D1E8E722469CE722460C3278
:10B8600012F9081C0329A7D12D4A03EB430302EB6D
:10B870008303D3F83C3D002B36D02C4B027993F850
:10B880003D1093F83C309142CFD09A4297D1CCE70B
:10B89000234A03EB430302EB8303D3F83C3D002B25
:10B8A00099D0234B027993F83D1093F83C309142A4
:10B8B000BBD09A428ED1B8E7194A03EB430302EB9F
:10B8C0008303D3F83C3D002B8ED01A4B027993F8BA
:10B8D0003D1093F83C309142A7D09A42A5D00F4B2F
:10B8E0009B68DB0384D501E022466AE7124C002303
:10B8F00022461179232902F1140203D00133092BC6
:10B90000F7D175E703EB8303026854F823309A42BA
:10B910007FF46EAF89E700BFAC8C00209C00001064
:10B92000707F0020000300204C05002098070020B5
:10B93000E4090020300C0020801000200D4B10B5D1
:10B9400003F1B40C4FF0000E02E014339C450FD00D
:10B950001A688242F9D1DA688A4218BFD9600EF1BA
:10B96000010403F1140318BF5FFA84FE9C45EFD174
:10B97000704610BD801000202DE9F04F3D4EDFF8DD
:10B980000091DFF800813C4D83B04FF0000B019037
:10B99000B2465F46DAF800404046002101E055F823
:10B9A0003100844203D001310E29F8D1FF214944EE
:10B9B00091F8941D012944D0022909D1DAF80C101C
:10B9C000480705D521F0040141F00801CAF80C1020
:10B9D0005046FFF7D1FE48B9264B0BEB8B0103EB2A
:10B9E0008101C96801F00C00042835D00BF1010B6E
:10B9F000BBF1090F0AF1140ACCD1204C3046FFF7F5
:10BA0000BBFEC0B9F368590703F00C0213D5042A32
:10BA100011D07A1CD5B2019A23F0080040F004003E
:10BA2000BA42014623F004031ED9F0603068FFF7E4
:10BA300085FF2844C7B21436B442DFD103B0BDE855
:10BA4000F08FDAF80C100B07C2D521F0080141F095
:10BA50000401CAF80C10BBE72046FFF76FFF01375F
:10BA6000FFB20744FFB2C1E73068F3601946FFF741
:10BA700065FFE0E7801000203C65070834110020D6
:10BA8000707F00200000014038B50446BDF810501A
:10BA90002160084619B11946F6F764FC206829466A
:10BAA000F6F7DCFC236859680B68B3F844206FEAAA
:10BAB00042426FEA524292B2A3F844201A8892B2EC
:10BAC00042F001021A804A79032A17D8DFE802F00F
:10BAD000110C070240330022A3601A6038BD3C33CA
:10BAE0000022A3601A6038BD38330022A3601A60B8
:10BAF00038BD34330022A3601A6038BD0023A36030
:10BB00001B60FFDE2DE9F04F85B00646BDF838A07A
:10BB10009DF83CB0894617469846FAF711FB054652
:10BB2000002843D0274C94F8A23D072B39D85C223B
:10BB300002FB03420021C2F8A41D82F8A81D5A1C72
:10BB4000D2B203EB430184F8A22DC3EBC10304F688
:10BB5000A4543079039204EB8304FEF75DFB50B3E9
:10BB6000039A80F8069002210272C1710390BBF122
:10BB7000000F12D11121FCF73DFC039B1A689B8832
:10BB800053832046CDF800A043463A462946FFF7A6
:10BB90007BFF204605B0BDE8F08F327AFEF720FD2E
:10BBA000EFE7094A00210420FAF7AEF90024204605
:10BBB00005B0BDE8F08FBBF1000FE2D11121FCF719
:10BBC00019FCDEE7707F0020CC1608082DE9F0474D
:10BBD0003E4D15F8743C82B03BB93D4A0221042029
:10BBE00002B0BDE8F047FAF78FB915F8737C15F885
:10BBF000723C0137FF1A102F0DDD10230221009334
:10BC000005F8711C334A3B4600210420FAF77CF901
:10BC100002B0BDE8F08715F8683C012B064611D04C
:10BC2000022B0BD161F01CF92B4B45F8643C15F845
:10BC3000681C11F0FD040BD0284ACFE7284B45F8CB
:10BC4000643CF4E761F00CF9264B45F8643CEEE700
:10BC50007368BB422FDB002FDADDDFF89880DFF856
:10BC600098A0DFF88490243604E00134BC4248F800
:10BC7000040FCDD0DAF8083035F8701C0091C3F30A
:10BC80000072019235F86E3C174AB9FBF3F356F88F
:10BC9000040F9BB20321FFF735FF0028E5D1134ABB
:10BCA000052601462346042005F8716C02B0BDE864
:10BCB000F047FAF729B9042000930D4A05F8710CF2
:10BCC0003B462146FAF720F9A2E700BF6890002022
:10BCD000081708082417080855770008B01708083F
:10BCE0003D770008D1F0020840420F00881708088D
:10BCF00050170808EC7F00209C00001030B5036846
:10BD00002C4C2DED028BA34283B0F0EE408AB0EEB6
:10BD1000608A13D004F58064A3420FD004F57054F8
:10BD2000A3420BD004F58064A34207D004F58064DD
:10BD3000A34203D0204B1C68640801E01E4B1C6822
:10BD40000192B4FBF1F202F57F420023FF32120CA4
:10BD50000093B4FBF2F4B4FBF1F52246ABB202213E
:10BD6000FFF7D0FEC0B1B5EE408AF1EE10FA17D061
:10BD700007EE904AF8EE677A27EE888A9FED0F7AF1
:10BD8000C8EE076A0123037127EE667AC0ED046AE4
:10BD9000A8EEA77A80ED037A03B0BDEC028B30BD2C
:10BDA00007EE905AB8EE678A07EE904AF8EE677A87
:10BDB000E4E700BF000001407C0E002000007A4450
:10BDC0002DE9F04F2DED028B804B1F780C2F87B0A3
:10BDD00000F3B9807E4BDFF850829B7988F8003001
:10BDE000032B21D91A1F022A00F2A680052B00F08E
:10BDF000CB80062B0CBF4FF47A544FF47A64754A0B
:10BE00007549764D05921646754A46F8602C4FF0F6
:10BE1000000A00224FF0000B4A60C5E900AB714AEE
:10BE2000B2FBF4F20A6005E06A4A059211466E4AD6
:10BE300041F8602C6D4A12F81330002B00F0B080EE
:10BE40000368BB42C0F2B680002F40D0DFF8DCA10F
:10BE5000674E9FED688A039700F108050024DAF821
:10BE6000082098F8003055F8040BC2F30072062B36
:10BE700078D8DFE803F055493D3104040400052B70
:10BE80006ED05D495D4F062B18BF39464FF0000B51
:10BE90000192CDF800B00A4614230221FFF732FECA
:10BEA000814650B100F11403194600680493122230
:10BEB0005FF0BCFF049B002869D146F83490E30092
:10BEC000F358002B51D0039B0134A342C7D107B0D4
:10BED000BDEC028BBDE8F08F3D4BDFED490A998840
:10BEE000B0EE600AFFF70AFFE30046F83400E7E728
:10BEF000DFED440A9FED440A4FF4FA61FFF7FEFEBE
:10BF0000E30046F83400DBE7DFED400A4FF47A71D6
:10BF1000B0EE600AFFF7F2FEE30046F83400CFE728
:10BF20009FED340AF0EE480A4FF4C871FFF7E6FEC1
:10BF3000E30046F83400C3E7264A05921146344A26
:10BF400041F8602C76E72349324A0C230120009304
:10BF500001F8710C3B4600210420F9F7D5FFB6E744
:10BF60002D4993E7002346F834302346059C2B4A9D
:10BF7000052004F8710C0021042007B0BDEC028BF1
:10BF8000BDE8F04FF9F7C0BF4FF4FA5437E7184651
:10BF90005946482269F086FA012389F804308CE773
:10BFA0001F4A0221042007B0BDEC028BBDE8F04F10
:10BFB000F9F7AABF05980093032100F8711C194AEC
:10BFC0003B4600210420F9F79FFF80E79400001012
:10BFD000D43F002068900020503E0020583E0020B2
:10BFE0006D77000840420F00DD7B0008B865070848
:10BFF000903E00206F12833A001BB700C0C62D0090
:10C0000000000000ACC5A737ACC5A7366F120339D6
:10C0100039770008EC170808808D5B007418080851
:10C0200018180808381808084A3E00209C0000101C
:10C0300010B5104CD4E90423A16882B002FB03F3CD
:10C040008B428DF8070012D06368E0680DF107019C
:10C05000184467F087F863682269A168134462692D
:10C06000B3FBF1F0013201FB10336360626102B097
:10C0700010BD00BF683E002010B53220FEF7CCF89E
:10C0800090B1044601214FF40873C3800172FCF79C
:10C09000B1F92168114BA0884883002203F8582C7D
:10C0A00043F85C4C03F8572C3520FEF7B5F80446EE
:10C0B00090B14FF408720223C28003720121FCF791
:10C0C00099F92168054BA0884883002203F8502C79
:10C0D00043F8544C03F84F2C10BD00BF689000206B
:10C0E00010B50379012B84B00C4621D0022B1DD151
:10C0F0008368DB070DF10F024CBF01218121FDF7A1
:10C1000093F99DF80F30114A1074C3F3C002C3F3C2
:10C11000001CC3F38001A270C3F38012DB0984F812
:10C1200000C06170E270237104B010BD0020E8E728
:10C1300082680DF10F0102F00102CDE900121A46EA
:10C14000417C90F91000F7F7C1FBDAE7EC1800200A
:10C150002DE9F04182B014460E4601AA5021054651
:10C16000FDF7B8F99DF80430DFF8F080394F01335E
:10C170005B00DBB24621238001AA2846FDF7AAF91D
:10C180009DF804305A1C2378A28008FB03F303F5C2
:10C19000FA73A7FB03139909DB0902FB0133A7FB21
:10C1A00003239B0901AAE360512102232846FCF7DF
:10C1B0004BFC2378BDF8041008FB03F349BA03F5E0
:10C1C000FA73A7FB0323CAB2C1F307218A400132E5
:10C1D00092B29909DB0902FB0133E280A7FB03233A
:10C1E0009B09238201AA70212846FDF773F99DF867
:10C1F000043001335B00DBB201AA638071210223AA
:10C200002846FCF721FCBDF80420134BF178187484
:10C2100052BAD3B2C2F30722934001339AB22281B9
:10C2200019B1E388D31A9AB22281A1780B4B09483D
:10C2300003FB01F101F5FA71A0FB01139909DB0978
:10C2400002FB0133A0FB03239B09638202B0BDE81C
:10C25000F08100BFD34D6210EC180020002F3A008F
:10C260002DE9F043934EDFF854828FB00546002746
:10C270004FF4FA7309AA89210068C6F8C03686F817
:10C28000C070FDF727F99DF82420286842F00102CC
:10C290008921FCF7A5F93A4688212868FCF7A0F91E
:10C2A000012280212868FCF79BF90122FF212868E0
:10C2B000FCF796F93A4639462868FCF791F909AA3D
:10C2C00091212868FDF706F99DF82430286886F842
:10C2D000B93639460122FCF783F93A46FF2128682E
:10C2E000FCF77EF93A4680212868FCF779F909AA1B
:10C2F00060212868FDF7EEF89DF82420286842F0B8
:10C3000012026021FCF76CF920238DF8253009AA70
:10C310000223442128688DF82470FCF7C3FAFF2219
:10C3200001212868FCF75CF92C6801228021204655
:10C33000FCF756F90122FF212046FCF751F93A4655
:10C3400039462046FCF74CF9FF2106222046FCF72F
:10C3500047F909AA83212046FDF7BCF89DF824205F
:10C36000832142F004022046FCF73AF90722FF211C
:10C370002046FCF735F9012281212046FCF730F9EF
:10C38000012280212046FCF72BF994216B222046C4
:10C39000FCF726F93A4683212046FCF721F9464F5F
:10C3A000D8F800303874C6F8BC3614E0A368DB0750
:10C3B00009AA4FF0830120465EBF09AA83212046C7
:10C3C000FDF732F89DF82430387483B9D6F8C036BA
:10C3D000002B40F0AA822379012B00F09982022BD6
:10C3E000E4D09DF8243000203874002BEED0832157
:10C3F00001222046FCF7F4F809AA92212046FDF715
:10C4000069F80022812120469DF82490FCF7E8F885
:10C41000FF2106222046FCF7E3F809AA83212046E3
:10C42000FDF758F89DF82420832102F0FB022046F6
:10C43000FCF7D6F80122FF212046FCF7D1F80122B3
:10C4400000212046FCF7CCF80022FF212046FCF713
:10C45000C7F8204600228021FCF7C2F8062307AA6D
:10C46000B0212868FCF7F0FA0122FF212868FCF7C8
:10C47000B7F800224F212868FCF7B2F82C224E2191
:10C480002868FCF7ADF80022FF212868FCF7A8F81F
:10C490004FEAD9182868B422B621FCF7A1F8002485
:10C4A000B8F1000F18BF4FF00C0809F07F0EA4463A
:10C4B000012017E0707F0020EC180020F8360020E3
:10C4C000E64503F0070317D011F81C2C42FA03F3DA
:10C4D000DB070CF1010104F1010448BF5FFA81FCA4
:10C4E000302C12D0E3B20EAA02EBD301984503F030
:10C4F000070200FA02F2E3D911F81C3C013423EAE6
:10C500000202302C01F81C2CECD1062307AAB02122
:10C510002868FCF7C7F90122FF212868FCF760F8BA
:10C52000002211462868FCF75BF80022FF212868EA
:10C53000FCF756F8002209212868FCF751F8002280
:10C5400010212868FCF74CF8002211212868FCF71C
:10C5500047F8012224212868FCF742F8FF22252110
:10C560002868FCF73DF8002275212868FCF738F8A8
:10C570000122FF212868FCF733F82C224E2128687D
:10C58000FCF72EF8002248212868FCF729F82146FC
:10C5900020222868FCF724F80022FF212868FCF7F5
:10C5A0001FF8214609222868FCF71AF800225421B6
:10C5B0002868FCF715F8042231212868FCF710F8E8
:10C5C000032232212868FCF70BF8832240212868D7
:10C5D000FCF706F8252246212868FCF701F800221E
:10C5E00060212868FBF7FCFF002227212868FBF761
:10C5F000F7FF062250212868FBF7F2FF00225121A5
:10C600002868FBF7EDFF962252212868FBF7E8FF28
:10C61000562108222868FBF7E3FF224657212868A5
:10C62000FBF7DEFF002261212868FBF7D9FF00221B
:10C6300062212868FBF7D4FF002264212868FBF7F9
:10C64000CFFF002265212868FBF7CAFFA0226621E0
:10C650002868FBF7C5FF0122FF212868FBF7C0FF10
:10C66000322222212868FBF7BBFF142247212868C9
:10C67000FBF7B6FFFF2249212868FBF7B1FF002234
:10C680004A212868FBF7ACFF0022FF212868FBF74E
:10C69000A7FF0A227A212868FBF7A2FF00227B214C
:10C6A0002868FBF79DFF212278212868FBF798FF77
:10C6B0000122FF212868FBF793FF342223212868F9
:10C6C000FBF78EFF002242212868FBF789FFFF223B
:10C6D00044212868FBF784FF262245212868FBF7C0
:10C6E0007FFF052246212868FBF77AFF402211468A
:10C6F0002868FBF775FF06220E212868FBF770FFFC
:10C700001A2220212868FBF76BFF4022432128686A
:10C71000FBF766FF0022FF212868FBF761FF032279
:10C7200034212868FBF75CFF442235212868FBF799
:10C7300057FF0122FF212868FBF752FF0422312115
:10C740002868FBF74DFF09224B212868FBF748FFBB
:10C7500005224C212868FBF743FF04224D2128685D
:10C76000FBF73EFF0022FF212868FBF739FF00227C
:10C7700044212868FBF734FF202245212868FBF775
:10C780002FFF082247212868FBF72AFF282248218B
:10C790002868FBF725FF002267212868FBF720FFA8
:10C7A000042270212868FBF71BFF012271212868F1
:10C7B000FBF716FFFE2272212868FBF711FF00220B
:10C7C00076212868FBF70CFF002277212868FBF709
:10C7D00007FF0122FF212868FBF702FF01220D213C
:10C7E0002868FBF7FDFE0022FF212868FBF7F8FE12
:10C7F000012280212868FBF7F3FEF8220121286836
:10C80000FBF7EEFE0122FF212868FBF7E9FE01227B
:10C810008E212868FBF7E4FE012200212868FBF73F
:10C82000DFFE0022FF212868FBF7DAFE00228021CC
:10C830002868FBF7D5FE04220A212868FBF7D0FE02
:10C840002C6809AA84212046FCF744FE9DF8242088
:10C85000842102F0EF022046FBF7C2FE01220B21E9
:10C860002868FBF7BDFE2868039005A9FFF738FC90
:10C87000039809AA05A9FFF76BFC9DF81430002B5B
:10C8800066D00C9C04F684549DF81630002B56D0CC
:10C890000C9B03F2B22304EB43049DF8173023B141
:10C8A000BDF8343003F525731C449DF8183023B1CE
:10C8B000BDF8363003F226231C44DFF8EC822868EA
:10C8C00048F83C4CE8220121FBF78AFE44F61F633E
:10C8D0009C423874286803D9214660F0DFFD28683F
:10C8E00001221146FBF77CFE402138742868FDF7D1
:10C8F00087F950B1012128680222FBF771FE00215F
:10C9000038742868FDF77CF928BB0FB0BDE8F083C8
:10C91000A268617C94F9100002F00102019209AA58
:10C9200000928322F6F7D2FF4CE5D8F80020D6F823
:10C93000BC1692B2521A9342BFF44DADE5E79DF892
:10C940001530002BA9D00C9B03F525731C44A4E7DC
:10C9500040F6363498E7E82201212868FBF740FECC
:10C96000002402234FF0200C09AA442128688DF8E6
:10C9700025C08DF82440FBF795FFD5F8009005A958
:10C980004846FFF7ADFB09AA05A94846FFF7E0FBBB
:10C99000502257214846FBF723FE082256214846DD
:10C9A000FBF71EFE082250214846FBF719FEBDF892
:10C9B00034204FF47A7148F20E6301FB0233764A59
:10C9C000934240F2E680754AA2FB03231B0C5A1ED9
:10C9D00032F0FF0309D023465208013322F0FF0151
:10C9E0009BB20029F8D11B029BB21343C3F3072269
:10C9F000DBB28DF810208DF8113004AA02235121EA
:10CA00004846FBF74FFF0C9A4FF47A7148F20E63D9
:10CA100001FB0233624A934200F2B9805F4AA2FBF3
:10CA20000332120C013AD2B246214846FBF7D8FD38
:10CA300058F83C4C387444F61F639C4205D9214693
:10CA4000484660F02BFD58F83C4C04AA01214846AA
:10CA5000FCF740FD02229DF8108001214846FBF7BB
:10CA6000BFFD00214846FDF7CBF84246012148466C
:10CA7000FBF7B6FD2D6805A92846FFF731FB09AA8B
:10CA800005A92846FFF764FB482211462846FBF714
:10CA9000A7FD082247212846FBF7A2FD03223221E9
:10CAA0002846FBF79DFD072230212846FBF798FD1D
:10CAB0000122FF212846FBF793FD20223021284642
:10CAC000FBF78EFD0022FF212846FBF789FD062299
:10CAD00070212846FBF784FDBDF83610314A4FF42B
:10CAE0007A7046F6440300FB0133A2FB03239DF852
:10CAF00017201B0B1AB1BDF82A2013449BB2002B40
:10CB000043D05A1E32F0FF0309D0002352080133EC
:10CB100022F0FF019BB20029F8D11B029BB2134304
:10CB2000C3F30722DBB28DF810208DF8113004AA70
:10CB3000022371212846FBF7B5FE44F61F639C4291
:10CB4000387403D92146284660F0A8FC04AA0121C4
:10CB50002846FCF7BFFC9DF8104002220121284620
:10CB6000FBF73EFD00212846FDF74AF82246012149
:10CB70002846FBF735FD642201233874C6F8C02629
:10CB800086F8C0300FB0BDE8F0831A46CBE7FF222D
:10CB90004AE7234622462CE71B0C0100950370F45C
:10CBA0001B280D014963A4136890002010B5184C90
:10CBB00084F8AD15017952BAA4F8AE2501294FF0D9
:10CBC000000282B084F8AC2512D002290CD10423D3
:10CBD00004F2AC52FF21FBF70DFE002814BF002029
:10CBE0006FF00C0002B010BD6FF00C0002B010BD71
:10CBF0008268417C90F9100004F2AC5402F001020A
:10CC0000CDE900420423FF22F7F766FAE5E700BF0B
:10CC1000707F00202DE9F04FA24FA34D0668002140
:10CC20003C4685B0834685F8C2105A37C4F12D09B9
:10CC300005F2AC5A884615E0022A0FD1B26812F00C
:10CC4000010F4FF0030352464FF0FF01304601BF82
:10CC500003235246FF213046FBF7CCFDBC421AD0DD
:10CC600014F8011F327985F8AE1509EB0403012A87
:10CC700085F8AC8585F8AD35DED1B368717C96F961
:10CC8000100003F00103CDE900A3FF220323F7F70F
:10CC900023FABC42E4D14FF40743A5F8AC35402356
:10CCA00085F8AE3552460323FF213046FBF7FAFDE7
:10CCB00000238DF80E300DF10E01304660F0B4FB0C
:10CCC0009DF80E30002BF6D04FF40640A5F8AC05C9
:10CCD0000120764A85F8AE050323FF213046FBF795
:10CCE000E1FD4FF40740714AA5F8AC050024032389
:10CCF000FF21304685F8AE45FBF7D4FD4FF40060C8
:10CD0000A5F8AC050920694A85F8AE050323FF2183
:10CD10003046FBF7C7FD4FF43063A5F8AC35634AE6
:10CD200085F8AE4530460323FF21FBF7BBFD002805
:10CD30007FD0DBF800600DF10E025E213046FBF77C
:10CD400075FFBDF80E30B3F5D77F00F0A38079D81A
:10CD5000512B75D040F29480AD2B00F09B80D62BE8
:10CD600040F08A80212408BB0A224B213046FBF781
:10CD7000BBFD0F2260213046FBF7B6FD0D2263217B
:10CD80003046FBF7B1FDB82269213046FBF7ACFD18
:10CD900040F60D7278213046FFF708FF40F60E622C
:10CDA0007A213046FFF702FF002875D0DBF800003B
:10CDB000212160F089FADBF800400DF10E02DE213E
:10CDC0002046FBF733FFBDF80E309FED397AC3F3F1
:10CDD0000903ADF80E3003EB8303DB0007EE903A56
:10CDE000F8EEE77A204667EE877A0623FCEEE77ACC
:10CDF0004FF4D84417EE902A110E85F8AE15110C99
:10CE000052BA85F8AF15A5F8B025FF215246A5F80E
:10CE1000AC45FBF747FD4FF407414023DBF800002A
:10CE2000A5F8AC1585F8AE3552460323FF21FBF774
:10CE300039FD85F8C20005B0BDE8F08F1E2BB5D1D5
:10CE4000142490E740F2E132934221D00AD940F213
:10CE50008F42934203D040F291529342A6D14FF4B5
:10CE6000FA7480E740F2D922934211D040F2E122D5
:10CE7000934209D1642476E7602B3FF473AF95E7C2
:10CE80001D2BDBD10F246EE7B3F5E67FF2D08DE7E3
:10CE9000C82468E7322466E72146304660F014FA79
:10CEA00084E700BF18760708707F00201C850020EB
:10CEB0009A99893F03682DE9F041DF691FB13B462C
:10CEC000BDE8F0411847002A164611DD04460D461C
:10CED0000E4400E023689B68204698470028F9D05C
:10CEE000236815F8011B1B6820469847AE42F1D114
:10CEF000BDE8F081DEE700BF224B1B6813F0100F86
:10CF0000214B03D033F8382C520717D413F81E2CBA
:10CF100002BB13F8102C53F8143C52B143B120B1AA
:10CF20001A689B88138370474BB31A689B88538396
:10CF3000704780F00100002BF1D1F9E713F81E2CA7
:10CF4000B2B913F8102C53F8143C002AECD1002B82
:10CF5000E6D1704753F81C2C002AE9D058B19268EA
:10CF600033F8181C094BB3FBF1F35B1013607047E7
:10CF700053F81C2C22B1936800221A607047704746
:10CF8000704700BF980000106890002040420F00DA
:10CF9000BFF34F8F0549064BCA6802F4E0621343A2
:10CFA000CB60BFF34F8F00BFFDE700BF00ED00E097
:10CFB0000400FA0508B572B600224FF0FF31930065
:10CFC00003F1604303F561430132082AC3F880107E
:10CFD000C3F88011F3D1FFF7DBFF00BF012108B5D3
:10CFE0000846F7F7BDFBFFF7E5FF00BF00B583B0CC
:10CFF0000D49002200920091009B04330093009B96
:10D000001B68012B02D003B05DF804FB0192019173
:10D01000019B064904330193019B1A600B6883F35B
:10D0200008884B689847FEE7502800400000FF1F23
:10D0300010B4EFF31183102282F31288094C0A48CE
:10D0400022684FF0E021013222608A6940F80C2CFE
:10D05000002240F8082C0A69DBB283F311885DF8DE
:10D06000044B7047F83600206890002030B4EFF38E
:10D070001182102383F312884FF0E023D2B2996912
:10D08000186910F4803F0D481EBF012140F8081CAC
:10D0900099690B4B1D6850F8083C82F311880948C8
:10D0A00004684FF47A7202FB04F02B44401A00210A
:10D0B000B0FBF4F030BCE3FB020170476890002045
:10D0C000F83600201C380020124B5B68C3F30803BD
:10D0D000FBB9EFF31183E3B930B40F4A0F4C4FF0B3
:10D0E000E02C1168DCF8180013688B42F9D154F871
:10D0F0000C1C8142F5D30A4A15684FF47A7404FB7C
:10D1000005F20021101AB0FBF5F0E3FB040130BC7E
:10D110007047ABE700ED00E0F83600206890002093
:10D120001C38002090B170B5461EFFF7CDFF0446B5
:10D130000D46FFF7C9FF031B61EB0502B3F57A7FCC
:10D1400072F10003F5D3013EEFD270BD704700BF0E
:10D150002DE9F041046888B00546B6227E212046BC
:10D16000FBF73EFA4FF06408FFF7AEFF06460F46A6
:10D17000FFF7AAFF831B61EB0701B3F57A7F71F11B
:10D180000003F5D3B8F10108EED102212046FBF7E8
:10D1900083F9636913B11A689B885383FFF794FF7F
:10D1A00006460F46FFF790FF831B61EB0702B3F5BE
:10D1B0007A7F72F10003F5D3636913B11A689B8813
:10D1C00013834FF00A08FFF77FFF06460F46FFF76D
:10D1D0007BFF831B61EB0701B3F57A7F71F10003DD
:10D1E000F5D3B8F10108EED142467C212046FBF789
:10D1F000F7F9FFF769FF06460F46FFF765FF831B48
:10D2000061EB0702B3F57A7F72F10003F5D30022D8
:10D2100059212046FBF7E4F9FFF756FF06460F4673
:10D22000FFF752FF831B61EB0702B3F57A7F72F1C0
:10D230000003F5D35E22002371498DF807200DF11C
:10D240000702CDE902320122CDE90531049202A99B
:10D250004FF4A4722046079261F06AFA4FF00A0870
:10D26000FFF732FF06460F46FFF72EFF831B61EBE9
:10D270000701B3F57A7F71F10003F5D3B8F1010826
:10D28000EED1012259212046FBF7AAF9FFF71CFF36
:10D2900006460F46FFF718FF831B61EB0702B3F545
:10D2A0007A7F72F10003F5D38C2240212046FBF7F0
:10D2B00097F9FFF709FF06460F46FFF705FF831BA7
:10D2C00061EB0702B3F57A7F72F10003F5D3032215
:10D2D00041212046FBF784F9FFF7F6FE06460F468C
:10D2E000FFF7F2FE831B61EB0702B3F57A7F72F161
:10D2F0000003F5D3AA6B434E95F83500B6FBF2F266
:10D30000092391B2404AFAF709F84388B6FBF3F6CD
:10D310002E640279422142F0C0022046FBF760F9F8
:10D32000FFF7D2FE05460E46FFF7CEFE431B61EB2C
:10D330000602B3F57A7F72F10003F5D30822432188
:10D340002046FBF74DF9FFF7BFFE05460E46FFF7F7
:10D35000BBFE431B61EB0602B3F57A7F72F100035B
:10D36000F5D3042258212046FBF73AF9FFF7ACFE2B
:10D3700005460E46FFF7A8FE431B61EB0602B3F518
:10D380007A7F72F10003F5D30A2253212046FBF77E
:10D3900027F9FFF799FE05460E46FFF795FE431B5A
:10D3A00061EB0602B3F57A7F72F10003F5D3002238
:10D3B0007C212046FBF714F9FFF786FE05460E4652
:10D3C000FFF782FE431B61EB0602B3F57A7F72F131
:10D3D0000003F5D306227D212046FBF701F9FFF774
:10D3E00073FE04460D46FFF76FFE031B61EB05025B
:10D3F000B3F57A7F72F10003F5D308B0BDE8F08190
:10D400007476070840420F00BC7707082DE9F04307
:10D41000A44A0468816BA44EB6FBF1F183B00546C3
:10D420000F2389B290F83500F9F778FF002143887F
:10D43000B6FBF3F607462E642046FBF72DF80022D4
:10D4400076212046FBF7CCF80F224E212046FBF731
:10D45000C7F84FF00F09FFF737FE06468846FFF77B
:10D4600033FE831B61EB0801B3F57A7F71F1000392
:10D47000F5D3B9F10109EED17A794F2102F00F020B
:10D480002046FBF7ADF84FF00F09FFF71DFE0646EB
:10D490008846FFF719FE831B61EB0801B3F57A7F1D
:10D4A00071F10003F5D3B9F10109EED17A79502178
:10D4B00002F00F022046FBF793F84FF00F08FFF73A
:10D4C00003FE06460F46FFF7FFFD831B61EB0701D6
:10D4D000B3F57A7F71F10003F5D3B8F10108EED10D
:10D4E000FF2252212046FBF77BF84FF00F08FFF791
:10D4F000EBFD06460F46FFF7E7FD831B61EB0701D7
:10D50000B3F57A7F71F10003F5D3B8F10108EED1DC
:10D5100095F83510072941D0644E96F8C900FAF7FE
:10D5200097F90546012276212046FBF759F8AA789B
:10D530000C212046FBF754F82A790D212046FBF7F1
:10D540004FF8AA79AB88120142EA1322D2B20E2117
:10D550002046FBF745F84FF4807196F8C900FAF7BA
:10D5600077F90546022276212046FBF739F8AA789A
:10D570005200032102F0FE022046FBF731F82A791F
:10D5800004212046FBF72CF8AA79AB88120142EA65
:10D590001322D2B205212046FBF722F80022762181
:10D5A0002046FBF71DF8032214212046FBF718F84C
:10D5B0000F27FFF789FD05460E46FFF785FD431B44
:10D5C00061EB0602B3F57A7F72F10003F5D3013FF8
:10D5D000EFD13A4663212046FBF702F86427FFF7B4
:10D5E00073FD05460E46FFF76FFD431B61EB060218
:10D5F000B3F57A7F72F10003F5D3013FEFD1082232
:10D6000065212046FAF7ECFF0DF107026421204660
:10D61000FBF760FF9DF8072022F0100242F0600245
:10D62000642120468DF80720FAF7DAFF0F27FFF76D
:10D630004BFD05460E46FFF747FD431B61EB060217
:10D64000B3F57A7F72F10003F5D3013FEFD10DF10D
:10D6500006024D212046FBF73DFF9DF8062002F013
:10D660003F0242F040024D2120468DF80620FAF795
:10D67000B7FF0F27FFF728FD05460E46FFF724FDED
:10D68000431B61EB0602B3F57A7F72F10003F5D319
:10D69000013FEFD103212046FAF7FEFE03B0BDE8BB
:10D6A000F08300BFF477070840420F00707F00202E
:10D6B000F0B5002283B004460A210068FAF790FF13
:10D6C0001427FFF701FD05460E46FFF7FDFC431B3F
:10D6D00061EB0602B3F57A7F72F10003F5D3013FE7
:10D6E000EFD120680F220A21FAF77AFF0A27FFF705
:10D6F000EBFC05460E46FFF7E7FC431B61EB060219
:10D70000B3F57A7F72F10003F5D3013FEFD12068C2
:10D71000032301AA1021FBF797F90A27FFF7D4FC8E
:10D7200005460E46FFF7D0FC431B61EB0602B3F53E
:10D730007A7F72F10003F5D3013FEFD19DF8042009
:10D740009DF805009DF80610194B8032803080311D
:10D75000A3F8C426A3F8C6063A46A3F8C81620685C
:10D760000A21FAF73DFF0A27FFF7AEFC05460E46F1
:10D77000FFF7AAFC431B61EB0602B3F57A7F72F157
:10D780000003F5D3013FEFD10DF103022068022120
:10D79000FBF7A0FE0DF1030220680921FBF79AFEBA
:10D7A000206811220A21FAF71BFF012003B0F0BD07
:10D7B000707F0020F0B5002283B004460A21006883
:10D7C000FAF70EFF1427FFF77FFC05460E46FFF71A
:10D7D0007BFC431B61EB0602B3F57A7F72F1000319
:10D7E000F5D3013FEFD120680F220A21FAF7F8FEA6
:10D7F0000A27FFF769FC05460E46FFF765FC431B49
:10D8000061EB0602B3F57A7F72F10003F5D3013FB5
:10D81000EFD12068032301AA1021FBF715F90A278D
:10D82000FFF752FC05460E46FFF74EFC431B61EB2B
:10D830000602B3F57A7F72F10003F5D3013FEFD111
:10D840003A4620680A21FAF7CBFE0A27FFF73CFC8C
:10D8500005460E46FFF738FC431B61EB0602B3F5A5
:10D860007A7F72F10003F5D3013FEFD10DF103028E
:10D8700020680221FBF72EFE0DF10302206809212A
:10D88000FBF728FE206801220A21FAF7A9FE0120F1
:10D8900003B0F0BDF8B57822044600210068FAF71D
:10D8A0009FFE0527FFF710FC05460E46FFF70CFC10
:10D8B000431B61EB0602B3F57A7F72F10003F5D3E7
:10D8C000013FEFD1206820220121FAF789FE0527C8
:10D8D000FFF7FAFB05460E46FFF7F6FB431B61EB2D
:10D8E0000602B3F57A7F72F10003F5D3013FEFD161
:10D8F00020683A460221FAF773FE6426FFF7E4FB3C
:10D9000004460D46FFF7E0FB031B61EB0502B3F590
:10D910007A7F72F10003F5D3013EEFD10120F8BD0B
:10D9200070B52422044641210068FAF759FE90B9E7
:10D930000526FFF7C9FB04460D46FFF7C5FB031B91
:10D9400061EB0502B3F57A7F72F10003F5D3013E76
:10D95000EFD1012070BD206820223021FAF740FE6F
:10D960000028E5D0206806223121FAF739FE002888
:10D97000DED0206800223421FAF732FED8E700BF5B
:10D98000F8B5072204460A210068FAF729FE0527A0
:10D99000FFF79AFB05460E46FFF796FB431B61EB2C
:10D9A0000602B3F57A7F72F10003F5D3013FEFD1A0
:10D9B000206824224121FAF713FE0527FFF784FB94
:10D9C00005460E46FFF780FB431B61EB0602B3F5ED
:10D9D0007A7F72F10003F5D3013FEFD12068C022B6
:10D9E0004221FAF7FDFD0526FFF76EFB04460D46C2
:10D9F000FFF76AFB031B61EB0502B3F57A7F72F157
:10DA00000003F5D3013EEFD10120F8BDF8B50122A6
:10DA1000074610210068FAF7E3FD00B9F8BD1426A7
:10DA2000FFF752FB04460D46FFF74EFB031B61EB6D
:10DA30000502B3F57A7F72F10003F5D3013EEFD111
:10DA40003868A022BDE8F8401121FAF7C9BD00BF2F
:10DA5000F0B583B0002304468DF802301427FFF799
:10DA600033FB05460E46FFF72FFB431B61EB060217
:10DA7000B3F57A7F72F10003F5D3013FEFD1394658
:10DA80000DF102022068FBF725FD0DF10202802155
:10DA90002068FBF71FFD7C238DF8053020688DF88A
:10DAA0000470032301AA60218DF80670FAF7FAFECC
:10DAB0001427FFF709FB05460E46FFF705FB431B3E
:10DAC00061EB0602B3F57A7F72F10003F5D3013FF3
:10DAD000EFD139460DF1030220688DF80370FBF792
:10DAE000F9FC62238DF80430C4238DF8053004233B
:10DAF0008DF806302068032301AA6021FAF7D2FED0
:10DB00001427FFF7E1FA05460E46FFF7DDFA431B3F
:10DB100061EB0602B3F57A7F72F10003F5D3013FA2
:10DB2000EFD139460DF1030220688DF80370FBF741
:10DB3000D1FC1D238DF8053008238DF806302068B0
:10DB40008DF8047001AA03236021FAF7ABFE1427B5
:10DB5000FFF7BAFA05460E46FFF7B6FA431B61EB2C
:10DB60000602B3F57A7F72F10003F5D3013FEFD1DE
:10DB700039460DF1030220688DF80370FBF7AAFC0B
:10DB800020680DF102021E21FBF7A4FC012003B066
:10DB9000F0BD00BF2DE9F041C2B282B00E233121A9
:10DBA0000220FCF75BFDDFF858810746C8F8F0005B
:10DBB000002860D00321FAF76FFC3226FFF784FAC1
:10DBC00004460D46FFF780FA031B61EB0501B3F530
:10DBD0007A7F71F10003F5D3013EEFD197F9103050
:10DBE000404C8DF8016003EB830304EB83039F2219
:10DBF000D3F8DC00BB6801929A0757D504230DEBDC
:10DC00000302694660F044FDBB689B0737D59DF869
:10DC100002009DF801209DF80330334900020025E1
:10DC200040EA02401843C4E90155304B304A258090
:10DC3000A5812F462E4601E011469A68884202D1FE
:10DC40009E88DD8801270833002AF5D19FB1A58180
:10DC50002680002E44D04FF480736380ABB21B0249
:10DC600003FB06F6B6F1807FC4E90136A27330D813
:10DC7000012388F8EC30384602B0BDE8F0811D4B36
:10DC80001D491A681D4B48684FF4FA7505FB02F2EE
:10DC9000A3FB023292094B681B1A9A42FBD27B69A2
:10DCA000002BB4D01A689B881383B0E77B6913B14B
:10DCB0001A689B8853830F4B0F491A680F4B4D68A6
:10DCC000D200A3FB023292094B685B1B9A42FBD243
:10DCD00094E70123B72088F8F830F9F7FDFFC7E78C
:10DCE0003746C8E7EC1800201620C2005078070815
:10DCF0001720C2001C380020001000E0D34D621035
:10DD0000707F00202DE9F043002383B01A463621AE
:10DD10000120FCF7A3FCDFF87C90074649F8040CCF
:10DD200060B34FF005089626FFF7CEF904460D467E
:10DD3000FFF7CAF9031B61EB0501B3F57A7F71F1B7
:10DD40000003F5D3013EEFD10DF10702314638460D
:10DD5000FBF7C0FB044668B9B8F10108E3D199F8B4
:10DD600000300C2B08BF0223384608BFC9F8043026
:10DD7000FCF71AFC204603B0BDE8F08399F80030A8
:10DD80000C2B01D00446F5E70123C9F80430044602
:10DD9000F0E700BF6890002070B5006801220921FB
:10DDA000FAF71EFC6426FFF78FF904460D46FFF7CD
:10DDB0008BF9031B61EB0502B3F57A7F72F1000367
:10DDC000F5D3013EEFD170BD2DE9804883B0431CEF
:10DDD0000193DFF83C810A230093D8F82812D8F881
:10DDE0003432B8F82C02B8F83822DDF804B0488391
:10DDF0004FF0320A1A834FF005094C69204214BFD4
:10DE00004883088359690A4214BF5A831A83012040
:10DE1000FFF772F856465746FFF756F904460D4687
:10DE2000FFF752F9001B61EB0501B0F57A7F71F144
:10DE30000003F5D3013FEFD1D8F82832B8F82C22EF
:10DE400059690A4214BF5A831A83D8F83432B8F891
:10DE5000382259690A4214BF5A831A830020FFF7F7
:10DE60004BF8FFF731F904460D46FFF72DF9001B7B
:10DE700061EB0501B0F57A7F71F10003F5D3013E46
:10DE8000EFD1B9F1000F0BD0B9F1010910D0B8F8FA
:10DE90002C02D8F82812B8F83822D8F83432ACE777
:10DEA0000BF1FF3BBBF1000F19D04FF00009EEE77B
:10DEB0004FF4FA76FFF708F904460D46FFF704F928
:10DEC000001B61EB0501B0F57A7F71F10003F5D31A
:10DED000013EEFD14FF0FA0ABBF1000FE5D14FF44C
:10DEE0007A76FFF7F1F804460D46FFF7EDF8031BCD
:10DEF00061EB0501B3F57A7F71F10003F5D3013EC3
:10DF0000EFD1009B013B00937FF467AFFFF766F80A
:10DF1000602C00202DE9F043814A0568816B814C1B
:10DF2000B4FBF1F185B00646102389B290F83500B4
:10DF3000F9F7F4F900214388B4FBF3F4074634649D
:10DF40002846FAF7A9FA80226B212846FAF748FBFF
:10DF50004FF09609FFF7B8F804468846FFF7B4F883
:10DF6000031B61EB0801B3F57A7F71F10003F5D370
:10DF7000B9F10109EED1032268212846FAF730FBF6
:10DF80004FF09609FFF7A0F804468846FFF79CF883
:10DF9000031B61EB0801B3F57A7F71F10003F5D340
:10DFA000B9F10109EED103226B212846FAF718FBDB
:10DFB000FFF78AF804468846FFF786F8031B61EBF3
:10DFC00008010F2B71F10003F6D310226A212846B5
:10DFD000FAF706FBFFF778F804468846FFF774F86F
:10DFE000031B61EB08010F2B71F10003F6D3002234
:10DFF0006C212846FAF7F4FAFFF766F804468846DB
:10E00000FFF762F8031B61EB08010F2B71F10003AE
:10E01000F6D37A7919212846FAF7E2FAFFF754F88D
:10E0200004468846FFF750F8031B61EB08010F2BED
:10E0300071F10003F6D318221B212846FAF7D0FA13
:10E04000FFF742F804468846FFF73EF8031B61EBF2
:10E0500008010F2B71F10003F6D318221C2128466A
:10E06000FAF7BEFAFFF730F804468846FFF72CF8B7
:10E07000031B61EB08010F2B71F10003F6D33A7912
:10E080001A212846FAF7ACFAFFF71EF807460C46A5
:10E09000FFF71AF88C4208BF8742F9D003212846BF
:10E0A000FAF7FAF93068062302AA4321FAF7CCFC02
:10E0B00028B3BDF80810BDF80A30BDF80C20C9BA65
:10E0C00007EE901ADBBAD2BAF8EEE76A07EE102A2A
:10E0D00007EE903AB8EEC77AF8EEE77AC6ED076A2F
:10E0E000C6ED087A86ED097AFDEEE77ACDED017A84
:10E0F0009DF90430013305D005B0BDE8F083D6EDBD
:10E10000087AF1E7D6ED077AFDEEE77ACDED017AF0
:10E110009DF904300133EFD10620FFF755FE00BF13
:10E120000079070840420F00437A5A1C0344D2B2D8
:10E1300042729972037A934200D97047002AFCD048
:10E1400010B5044604F10A01D0E9003098470023D5
:10E15000637210BD274E3568F06808B52CF086FE56
:10E1600028462CF083FEF06841798B073BD50021CF
:10E170000846FCF725FC00210120FCF721FC1E4C81
:10E18000F06803685B689847C8B92B6828465B68E5
:10E1900098470028F4D0D4F828222B68B4F82C1221
:10E1A000DB685183284698470146F0680268136887
:10E1B0009847D4F82832B4F82C221A83E0E7F068A4
:10E1C000D4F834220368B4F83812DB6851839847D6
:10E1D0002B6801461B6828469847D4F83432B4F8B7
:10E1E00038221A83D1E7036841F002019B699847FE
:10E1F000BDE700BFB8D90020602C00200FB410B5D7
:10E2000082B004AB0B4C53F8042BA06B0A4901936A
:10E2100060F01EFBA46B627A32B1D4E9003004F1E5
:10E220000A0198470023637202B0BDE8104004B0B1
:10E23000704700BFB8D9002029E100082DE9F84354
:10E24000DFF8648004460F461646002540F6340980
:10E250002046202168F085F80446D0B103461C46CC
:10E2600013F8010B2028FAD02046F8F781FB484527
:10E27000A8BF4846B0F5617FB8BF4FF46170A0F504
:10E280006170A8FB0030C0084DB17870337801335D
:10E2900033700DB90125DBE72046BDE8F8833870FF
:10E2A000337801333370F4E71F85EB5130B583B019
:10E2B00005460846019160F00DFD019904460246AD
:10E2C0002846F8F72FF820B92A5DA2F13001092974
:10E2D00002D8002003B030BD22F02002413A192AB2
:10E2E000F8D90134281903B030BD00BF18B1036854
:10E2F0001B6A03B118470020704700BF10B50C46D9
:10E3000020B10368DB6A0BB1984768B9074B00205E
:10E31000C4E90000C4E90200C4E906332D2130221B
:10E320002061217584F8202010BD00BF7C6F080893
:10E330000178F1B1F8B50F4F0546002602E015F857
:10E34000011FA9B1BC6B637A5A1C2344D2B262721A
:10E350009972237A9342F2D8002AF0D004F10A018C
:10E36000D4E900309847667215F8011F0029E9D1F9
:10E37000F8BD7047B8D9002070B504460E48FFF7C5
:10E38000D7FF2046FFF7D4FF0C48FFF7D1FF0C4B17
:10E390009E8F16B970BD013EFCD0FEF795FE044677
:10E3A0000D46FEF791FE031B61EB0502B3F57A7F84
:10E3B00072F10003F5D3EEE79C180808847A080888
:10E3C000B8D9002030B583B00E4C01900E480091B2
:10E3D000FFF7AEFFDDE900320C49A06B60F038FAC0
:10E3E000A56B6A7A32B12B68686805F10A01984713
:10E3F00000236B7294F83E3013B1012384F83F3050
:10E4000003B030BDB8D90020A418080829E10008DD
:10E410000FB470B582B006A951F8040B0191FFF753
:10E42000D1FF0E48FFF784FF0D4B9E8F36B902B027
:10E43000BDE8704004B07047013EF8D0FEF744FEDE
:10E4400004460D46FEF740FE031B61EB0502B3F5E3
:10E450007A7F72F10003F5D3EEE700BF847A0808F3
:10E46000B8D9002070B58379044603F007008CB05A
:10E470001546062800F29880DFE800F009112C2EDE
:10E48000313A04004E480CB0BDE87040B6E60E7854
:10E4900013F0C00308D0402B7BD00CB070BD13F03C
:10E4A000C00391F90060F6D146483146FFF7A6FE59
:10E4B000002DF2D0A37913F0C00FEED1424B227A97
:10E4C000E17953F8222033F9211040480CB0BDE81F
:10E4D000704093E60E88DBE7B1F90060D8E7096881
:10E4E00013F0C0030E4635D13948FFF787FEDFE74A
:10E4F00091ED000A6846F8F717F901463048FFF732
:10E500007DFE002DC9D0A37913F0C00FC5D1E379EA
:10E510002D4D35F9233000EE103A6846B8EEC00AAA
:10E52000F8F702F901462B48FFF768FEA37903F0DC
:10E53000C003402B2FD0237A05EB830393ED000A11
:10E54000B8EE400A6846F8F7EFF801462148FFF7B1
:10E5500055FEA2E7402BA0D1E379472B0FD81A4AEA
:10E5600002EBC30393F89C21914208D2D3F898316F
:10E5700053F8210018B10CB0BDE870403EE62046CB
:10E5800069461EF023FA14486A463146FFF740FFF9
:10E5900083E73146E0E7E37905EBC30595F89C3165
:10E5A000013B00EE103ACBE713F0C00301D11E4649
:10E5B0007AE7402B7FF471AF00210E46CCE700BF15
:10E5C000442808086C2408088C790708B018080843
:10E5D000681E0808004F0808B818080800283DD031
:10E5E0000378002B3AD02DE9F04F87B0594905AA9E
:10E5F00065F0C8FD0446002800F0A1804FF0000B34
:10E60000DFF87C91DFF87C81DFF87CA15D465F4616
:10E610004FF0FF360BE0BBF1000F26D04D4905AAA5
:10E62000002065F0AFFD0BF1010B044610B3BBF108
:10E63000010F15D0BBF1020FEDD14946204667F01E
:10E64000EAFE00286DD045F001054146204667F0FE
:10E65000E2FE00285ED045F00205DFE73E48D7E63F
:10E660002046F8F785F90746D8E72046F8F780F9FD
:10E670000646D3E770B2394A002392F9001081426E
:10E6800025D00133072B02F10C02F6D1002F4FD019
:10E69000002D08BF03250023EDB2CDE901530097FB
:10E6A0001A4619462CF032FB044600284DD02C485F
:10E6B000DFF8D8803A463146F7F7ECFB3146294877
:10E6C000F7F7E8FBD8F8000021465BF08DFCDFF897
:10E6D000BC8003EB430308EB83035C6C002CD5D0B8
:10E6E00021483146F7F7D6FB5DB16179A94208D0E0
:10E6F0001E482A46F7F7CEFB2368E9B29B692046FD
:10E700009847E36A002BD9D01948F7F7C3FB0023D9
:10E71000E362D3E72046514667F07DFE00289AD198
:10E720007CE71449204667F076FE00288BD18CE701
:10E7300011483146F7F7AEFB07B0BDE8F08F4FF058
:10E74000FF3025462746064695E731460B48F7F742
:10E75000A1FBF1E7E8700808CC190808F8D90020F7
:10E760002C1908089C1908084C190808641908088D
:10E7700084190808B43B0808E41808080C190808AC
:10E78000D8180808DC180808E0180808B8D90020CC
:10E79000002868D02DE9F04F90F800C085B00446FD
:10E7A000BCF1000F2AD000F100475A4E8646023FC6
:10E7B00001466346722207E0984526D1B94212D03D
:10E7C00011F8013F16F8012FA3F14105192DA2F10F
:10E7D000410098BF2033192802F12008ECD99A4251
:10E7E00013D1002AEAD14C4C0023C4F8203E84F80F
:10E7F000273EA4F8283E05B0BDE8F08F0021012097
:10E8000005B0BDE8F04F5BF049BC444E214663467D
:10E810006C2207E098452AD1B94212D011F8013F85
:10E8200016F8012FA3F14105192DA2F1410098BF5F
:10E830002033192802F12008ECD99A4217D1002A76
:10E84000EAD1374B1B685B07D5D4334C94F9263E8D
:10E85000002BD0D194F9213E002BC5DC05B0BDE8DA
:10E86000F04F52F0F5BB002101205BF017BC2D48A2
:10E87000732307E065455BD1774513D01EF801CFC0
:10E8800010F8013FACF141011929A3F1410298BFF1
:10E890000CF1200C192A03F12005EBD9634547D16F
:10E8A000002BE9D11C4B002293F9270E83F8202E70
:10E8B0001C46164693F8D2140129A1F1030509D08C
:10E8C000052D07D90EB184F8270E174805B0BDE80D
:10E8D000F04F9DE593F8D314A52903F1140303D059
:10E8E0000132782AE6D1EDE7012803D0013840B2A1
:10E8F0000126F5E70D4984F8200E0023013284F843
:10E90000212E81F8943084F8273E05B0BDE8F04F01
:10E9100050F0FEB9D8190808F0970020E01908084F
:10E9200098000010002A0808CC190808B8D900205F
:10E93000DFF880A22046F8F71BF89AF9947007FADE
:10E9400080F5772D064600F2D1802046202167F021
:10E9500008FD8046002800F01C810346984613F805
:10E96000012B202AFAD04046F8F702F801245FFA7A
:10E9700080F94046202167F0F4FC8046002800F032
:10E980000D810346984613F8012B202AFAD0404601
:10E99000F7F7EEFF01340090E4B24046202167F023
:10E9A000E0FC8046002800F0F7800346984613F804
:10E9B000012B202AFAD04046F7F7DAFF0134019004
:10E9C000E4B24046202167F0CCFC8046002800F0ED
:10E9D000BF800346984613F8012B202AFAD0404600
:10E9E000F7F7C6FF01340290E4B24046202167F0F9
:10E9F000B8FC8046002800F0A9800346984613F82A
:10EA0000012B202AFAD04046F7F7B2FF01340FFA63
:10EA100080FBE4B24046202167F0A3FC02460028B8
:10EA200000F0B58003461A4613F8011B2029FAD0DE
:10EA300010460392F7F79CFF0134039A0FFA80F80F
:10EA4000E4B21046202167F08CFC002856D0034623
:10EA50001A46013311782029FAD010460392F7F7AD
:10EA600087FF039A03461BB210462021039367F0E9
:10EA700078FC039B002800F0938002461046013288
:10EA800001782029FAD00393F7F772FF04F0FD0410
:10EA9000042C039B08BFC2B27FF417AFB9F1010F7A
:10EAA00004D9A9F1030105293FF60FAF22B1A52A28
:10EAB0002FD0482A7FF409AF3DB33B4905EB8505CC
:10EAC00001EB850181F8D2940098C1F8C004019847
:10EAD000C1F8C4040298C1F8C804A1F8CCB4A1F8E4
:10EAE000CE84A1F8D03481F8D32484E62F4930486D
:10EAF0007723002205B0BDE8F04F89E45FFA88F281
:10EB000003468046062CC9D0DFE6274981F8275EF8
:10EB1000D8E7FDB9244C0099C4F8C0140199C4F891
:10EB2000C4140299A4F8D03484F8D294C4F8C81458
:10EB3000A4F8CCB4A4F8CE8484F8D32401230137FC
:10EB40003E448AF8946084F8273E54E6834661E7A1
:10EB500002904AE7144C009805EB850504EB85010B
:10EB6000A1F8D03494F8273EC1F8C0040198C1F848
:10EB7000C4040133029881F8D294C1F8C804A1F802
:10EB8000CCB4A1F8CE8481F8D3245BB2D7E7804619
:10EB900057E704468146ECE6019012E70090FCE658
:10EBA0000134E4B20246ADE7F0970020E819080806
:10EBB000F4190808B8D900202DE9F04782B03E4981
:10EBC00001AA65F0DFFA002872D04FF0000A4FF07A
:10EBD000FF34394DD1465646D0462746BAF1040F88
:10EBE00009D8DFE80AF0443E380E03000378482BCA
:10EBF00046D0562B41D03148FFF70AFC02B0BDE8A1
:10EC0000F087F7F7B5FE3F280646F4D8002001AAA2
:10EC1000294665F0B7FA0AF1010A0028DED1BAF1F7
:10EC2000040F3AD02FDDBAF1050FE4D1244AB30125
:10EC300003F47C6308F03F0843EA0803B9F1000FCE
:10EC400001D043F40053962101FB074402EB440436
:10EC5000A4F89830D2E7F7F78BFE3F288046D5D945
:10EC6000C9E7F7F785FE95280446CFD9C3E7F7F73C
:10EC70007FFE03280746C9D9BDE74FF00109C5E764
:10EC80004FF00009C2E7BAF1020FB4DC0D49234688
:10EC90003A4601205BF088FAB0E7094A962303FB65
:10ECA000074302EB4303B3F89890C9F34039BEE73A
:10ECB0004FF0FF373C46E9E7E8700808CC19080830
:10ECC000B8D9002050DA00202DE9F04F8FB0974FCF
:10ECD000974C984E009182464FF0020905E00B34A4
:10ECE000BC4200F08D8094F80690B56B6A7A32B120
:10ECF000D5E9003005F10A01984700236B7209F04D
:10ED000038035345EBD18A4B8B48E51A8B4B0022D5
:10ED100003FB05F5ADB21621134605E00132342A96
:10ED200000F0EA8010F8011F0B449BB29D42F5D21F
:10ED3000834B03EB4202B2F80C14824A824B93429B
:10ED400080F0F1801D4603E01435954280F0EB80A1
:10ED50002B88C3F30B038B42F6D120461DF0FAFE3D
:10ED6000D5F80880054608EB000B20461DF050FF43
:10ED700009F00703062B15D8DFE803F0A49B938A5C
:10ED80004504AC00D0ED007A9BED007AB4EE677AD2
:10ED9000F1EE10FA0CBF01230023009A92063DD534
:10EDA000002B9CD10DF10809494620461DF00EFEAE
:10EDB000009B5B0640D465484946FFF71FFA0022D6
:10EDC00059462046FFF74EFB6148FFF7B1FAB38F73
:10EDD000002B84D09946FEF777F905468846FEF762
:10EDE00073F9401B61EB0801B0F57A7F71F1000304
:10EDF000F5D3B9F10109EED10B34BC427FF473AF06
:10EE00000FB0BDE8F08F026858F805309B1A009AE1
:10EE1000B3FA83F392064FEA5313C1D40DF10809F4
:10EE20004946204601931DF0D1FD009B13F0400F91
:10EE3000019BC0D0002BBED146484946FFF7DEF902
:10EE4000D9F80030444A934259D00022594620460E
:10EE5000FFF708FB3E48FFF76BFAB38F002BAAD0F1
:10EE6000CDF804A0A2461C46FEF72EF905468846BA
:10EE7000FEF72AF9401B61EB0801B0F57A7F71F1CA
:10EE80000003F5D3013CEFD15446DDF804A092E72E
:10EE9000B0F9002038F905309B1AB3FA83F35B0907
:10EEA0007BE7028838F805309B1AB3FA83F35B09D5
:10EEB00073E790F9002018F905309B1AB3FA83F331
:10EEC0005B096AE7027818F805309B1AB3FA83F3F6
:10EED0005B0962E709F0C009B9F1400F184B1BD07C
:10EEE000227A53F8222001460132584666F074FA1D
:10EEF000B0FA80F35B0950E74FF6FF711DE799F810
:10EF00000430002BA1D118F80530202B9DD11348D7
:10EF10005946FFF773F99DE7E27903EBC20393F8D3
:10EF20009C21013ADFE700239B68FFDEF2A7070878
:10EF3000908D0708B8D90020647D0708A38B2EBAEE
:10EF40008C790708B0920808748D0808141A08080C
:10EF5000847A0808201A08086E616D652C1A080862
:10EF600080B51848184DFFF7E3F91848FFF7E0F9A6
:10EF7000AC6B627A32B12146606851F80A3B98471F
:10EF8000002363722F683B6838465B699847B0B9C5
:10EF90000A26FEF799F804460D46FEF795F8031B7E
:10EFA00061EB0502B3F57A7F72F10003F5D3013E00
:10EFB000EFD13B6838465B6998470028E8D00120CC
:10EFC00007F006FC341A0808B8D90020501A0808BF
:10EFD00030B42F4C94F84835012B86B002D006B0DF
:10EFE00030BC704794F84D350A2B04D0294806B040
:10EFF00030BCFFF79DB941218DF80110264900234F
:10F00000152009788DF80200CDE90333EB20CDE916
:10F010000133A6228DF803008DF80410B2200321DD
:10F020008DF805008DF814308DF800208DF806104D
:10F03000EC460DF1120541F2210083EA0223082279
:10F0400013F4004F80EA43010ABF5B008BB29BB20E
:10F05000013AF5D1654502D01CF8012FEDE7C3F365
:10F0600007228DF814308DF81320EC461523C4F8D0
:10F07000B835BCE80F00094D0FC59CE8030045F802
:10F08000040B0748297006B030BCFFF751B900BF28
:10F09000B8D900205C1A0808841A002020DF00205C
:10F0A0006C1A0808F8B52D482D4FFFF741F92D4887
:10F0B000FFF73EF9BE8F002E40D1BC6B627A32B1B1
:10F0C0002146606851F80A3B984700236372002587
:10F0D00087F8BC55C7F8FC5587F8005622F0E4FCC9
:10F0E0002148FFF725F9BC6B627A2AB12146606896
:10F0F00051F80A3B984765723F683B6838465B6940
:10F100009847B0B90A26FDF7DFFF04460D46FDF724
:10F11000DBFF031B61EB0502B3F57A7F72F100039D
:10F12000F5D3013EEFD13B6838465B69984700282C
:10F13000E8D0002007F04CFB013EBED0FDF7C4FF35
:10F1400004460D46FDF7C0FF031B61EB0502B3F556
:10F150007A7F72F10003F5D3EEE700BF881A080842
:10F16000B8D90020847A0808501A0808F8B52B4C42
:10F1700094F83E301BB194F83F30002B41D101256B
:10F180002748FFF7D5F884F8075684F83C56F7F778
:10F19000C3FE244B24481B6884F83256002684F8AA
:10F1A0003C6684F80766C4F81436FFF7C1F8A56B0F
:10F1B0006A7AFAB927683B6838465B699847B0B9FC
:10F1C0000A24FDF781FF05460E46FDF77DFF401B33
:10F1D00061EB0601B0F57A7F71F10003F5D3013CD4
:10F1E000EFD13B6838465B6998470028E8D000209B
:10F1F00007F0EEFAD5E9003005F10A0198476E7282
:10F20000D8E70A48FFF704F90948FFF701F9002396
:10F2100084F83E3084F83F30F8BD00BFB8D90020F4
:10F220000C1B0808F8360020501A0808B41A080801
:10F23000EC1A0808F8B5394B394D1B68D5F840660B
:10F24000002B69D01B6A9847B48872884368A41A57
:10F2500004FB0334002C4AD03248FFF769F83248E7
:10F26000FFF766F83148FFF763F8AF8F87BB304888
:10F27000FFF75EF8AC6B627A002A45D14FF47A77DB
:10F28000FDF722FF04460E46FDF71EFF031B61EB50
:10F290000602B3F57A7F72F10003F5D3013FEFD197
:10F2A00028682BF0E3FD234B1A784AB122493846EF
:10F2B00051F837300BB19B68186001379742F7D18E
:10F2C00002210120F5F74CFAFDF774FE013FCED084
:10F2D000FDF7FAFE04460E46FDF7F6FE031B61EB52
:10F2E0000602B3F57A7F72F10003F5D3EEE7134817
:10F2F000FFF71EF8AD6B6A7A2AB12B68686805F1D2
:10F300000A0198476C72F8BD2368606804F10A012D
:10F31000984700236372B1E7094895E77C8600208F
:10F32000B8D900209C180808141B0808847A08081B
:10F33000501A080894000010903E0020341B080862
:10F34000848600202DE9F84F1A4F1B48DFF870A083
:10F35000DFF870B0DFF8708007F54C790024FEF715
:10F36000E7FF796811B15846FEF748FF1CB1134812
:10F370002146FEF743FF4046FEF7DAFFBAF83C604D
:10F380003EB94F4514D03869BC691037E7E7013EF4
:10F39000F7D0FDF799FE04460D46FDF795FE001BDC
:10F3A00061EB0501B0F57A7F71F10003F5D3EEE76B
:10F3B000BDE8F88F007E0708641B0808781B080862
:10F3C000B8D90020701B0808847A080870B50C486A
:10F3D000FEF7AEFF0B4B9E8F16B970BD013EFCD001
:10F3E000FDF772FE04460D46FDF76EFE031B61EB52
:10F3F0000502B3F57A7F72F10003F5D3EEE700BFA3
:10F40000847A0808B8D900202DE9F041354F3B68CF
:10F41000002B64D01B6A98478368002B59D0324870
:10F42000DFF8D880FEF784FF3048FEF781FFB8F898
:10F430003C601EBBD8F84006FAF7BAFE002388F8F5
:10F44000443688F84536C8F848363B6813B15B68DF
:10F45000984710BB6426FDF737FE04460D46FDF7BE
:10F4600033FE031B61EB0501B3F57A7F71F10003F5
:10F47000F5D3013EEFD1E8E7013EDBD0FDF724FEF6
:10F4800004460D46FDF720FE031B61EB0501B3F5B5
:10F490007A7F71F10003F5D3EEE71548FEF748FFD8
:10F4A0001248FEF745FFB8F83C601EB9BDE8F08190
:10F4B000013EFBD0FDF708FE04460D46FDF704FEB5
:10F4C000031B61EB0502B3F57A7F72F10003F5D3FC
:10F4D000EEE70848FEF72CFFBDE8F04176E7064866
:10F4E0009AE700BF7C860020941B0808847A0808ED
:10F4F000A01B0808801B080884860020B8D90020BB
:10F5000070B525490522044666F040FF10BB234C28
:10F5100094F83E3023B9012284F83E2084F83F302D
:10F520001F48FEF705FF1F48FEF702FFA68F16B91A
:10F5300070BD013EFCD0FDF7C7FD04460D46FDF74A
:10F54000C3FD031B61EB0502B3F57A7F72F1000383
:10F55000F5D3EEE714490322204666F017FFA8B959
:10F560000E4C94F83E3013B194F83F3053B90F4825
:10F57000FEF7DEFEFFF72AFF002384F83E3084F812
:10F580003F3070BD0A48FEF743FFF5E7BDE8704025
:10F590000848FEF73DBF00BFA81B0808B8D90020E7
:10F5A000B01B0808847A0808A8320808C81B080895
:10F5B000B41A0808DC1B0808800601D5002930D1E0
:10F5C0000CB470B5184C1949A06B82B007AB069A01
:10F5D00001935FF03DF9A56B6A7A32B12B686868D8
:10F5E00005F10A01984700236B721148FEF7A0FE4F
:10F5F000A68F3EB9012002B0BDE8704002B070474E
:10F60000013EF7D0FDF760FD04460D46FDF75CFDB9
:10F61000031B61EB0502B3F57A7F72F10003F5D3AA
:10F62000EEE70020704700BFB8D9002029E10008AC
:10F63000847A0808F0B5044683B070B302785AB3F0
:10F6400000F10040434D21460238722307E0974203
:10F6500037D1884214D011F8012F15F8013FA2F1DB
:10F66000410EBEF1190FA3F1410C98BF2032BCF13D
:10F67000190F03F12007EAD9934222D1002BE8D1D8
:10F68000354B364AC3F84C26C3F85026C3F85426E7
:10F69000C3F8582603B0F0BD1446314D314E35F84D
:10F6A000241005EB840332465888CDE90010012070
:10F6B000234600210444FFF77FFF042CEFD103B061
:10F6C000F0BD2046F7F754F9032805462FD8204609
:10F6D000202166F046FE0446002839D003461C4629
:10F6E00013F8012B202AFAD02046F7F741F9012719
:10F6F00006462021204666F034FE034688B11846AF
:10F7000001330278202AFAD0F7F732F94FB1A6F286
:10F71000EE2240F2DC539A4203D8A0F2EE229A4243
:10F720000ED9114803B0BDE8F040FEF771BE0F4995
:10F730000F480323002203B0BDE8F040FEF768BE87
:10F74000054B03EB8505A5F84C66A5F84E06A1E729
:10F750000746CEE7D8190808B8D90020E803D00733
:10F7600004E00020EC1B0808CC190808001C08085D
:10F77000F41908082DE9F04387B040B30378074631
:10F780002BB300F10040564E39460238722207E092
:10F790009C4532D1814212D011F8013F16F8012F59
:10F7A000A3F14105192DA2F1410498BF2033192C72
:10F7B00002F1200CECD99A421FD1002AEAD1494823
:10F7C0006022002107B0BDE8F04365F06BBE454DF7
:10F7D000454F0024D5E9010615F80C1B0091CDE931
:10F7E0000106012023463A4604440021FFF7E4FEC7
:10F7F000082CEFD107B0BDE8F0833846F7F7B8F82A
:10F80000C3B2072B054647D82021384666F0A9FD2C
:10F810000446002856D003461C4613F8012B202A24
:10F82000FAD02046F7F7A4F8071E18BF01270126D3
:10F830002046202166F095FD044600284ED0034660
:10F840001C4613F8012B202AFAD02046F7F790F82F
:10F8500001368046F6B22046202166F082FD03463E
:10F8600098B39946013399F80020202AF9D04846E8
:10F87000F7F77EF80136044620214846F6B266F0D6
:10F8800070FD08B10136F6B2032E0ED0174807B04E
:10F89000BDE8F043FEF7BCBD15491648072300221A
:10F8A00007B0BDE8F043FEF7B3BD134B6DB205EBF7
:10F8B000450503EB850383F85C76C3F86086C3F8DF
:10F8C000644697E706460746B2E72021059066F0B2
:10F8D00048FD059B1C460028D4D1D7E78046BAE7EF
:10F8E000D819080814E00020081C0808CC190808DA
:10F8F000201C0808F4190808B8D900202DE9F041A7
:10F9000084B010B103780446CBB9384C384F002589
:10F9100094F8820294F88362B4F880120091CDE9E1
:10F92000010601202B463A4605440021FFF744FE1C
:10F93000102D04F10404EBD104B0BDE8F081F7F719
:10F9400017F80F2805462CDC2046202166F009FD1B
:10F95000044628B103461C4601332278202AFAD0F7
:10F96000244B254FA035012603EB85082046F6F7EA
:10F97000FFFF37F8021B8842034606F1FF3219DC0D
:10F98000012A4FF02C01204626D0022A1CD0A8F8CC
:10F99000BC3666F0E6FC441C60B1032ECCD00136C8
:10F9A000E4E7164916480F23002204B0BDE8F041F1
:10F9B000FEF72EBD0D4B1348002243F8252004B05E
:10F9C000BDE8F041FEF724BD0A4A02EB850585F843
:10F9D000BF3604B0BDE8F08188F8BE3666F0C1FCE1
:10F9E0000028E7D0441C0136C0E700BF74E00020C7
:10F9F000301C0808B8D9002040810708441C0808BA
:10FA0000F4190808CC1908082DE9F04188B000283D
:10FA100044D003780446002B40D000252D2B5FD026
:10FA2000A3F13002092A5BD9202B53D1637801342A
:10FA3000002BF3D1052D4DD1BDF9142093B20F2B1E
:10FA400048D8BDF91610A1F5FA739BB2B3F5FA6F59
:10FA500040D8BDF91800A0F5FA739BB2B3F5FA6F60
:10FA600038D8BDF91A40A14234DCA04232DB8142D1
:10FA700030DCBDF91C5005F17D039BB2FA2B29D86F
:10FA8000214B03EBC202A2F8AC19A2F8AE09A2F80E
:10FA9000B04982F8B25908B0BDE8F0811B4CDFF8DC
:10FAA00074800025B4F9020094F90670B4F904607A
:10FAB00034F9081BCDE9001001202B46CDE902677F
:10FAC000054442460021FFF777FD102DEAD108B02A
:10FAD000BDE8F0810E4808B0BDE8F041FEF798BCE3
:10FAE000042DF7DC2046F6F743FF08AB03EB450394
:10FAF000013523F80C0C14F8013FA3F13002092A58
:10FB0000F9D9002B8AD195E7B8D9002064E3002009
:10FB1000CC1908084C1C0808F0B58BB007465FF0FC
:10FB2000D9F810F0FF0432D03C4E07F1050C3946ED
:10FB3000722205E098423FD1614512D016F8012F9C
:10FB400011F8013BA3F14105192DA2F1410498BF21
:10FB50002033192C02F12000ECD99A422CD1002A32
:10FB6000EAD12F482F4A904238BF40F2FF3103D3E9
:10FB700020E0143090421DD20388C3F30B038B4264
:10FB8000F7D129490BB0BDE8F040F7F7A5BB264DEA
:10FB9000264FA968D5E90006CDE9010601202346D4
:10FBA000009104443A460021FFF706FD082C05F1B8
:10FBB0000C05EED10BB0F0BD1D4905AA384664F026
:10FBC000E1FA78B11A4E06AD0024F6F7D1FE05AA87
:10FBD00045F8040B31460020013464F0D3FA30B10B
:10FBE000042CF2D11348FEF713FC0BB0F0BD042C2B
:10FBF000F8D1069B072BF5D80F4A1048DDE90741DD
:10FC000003EB430302EB8303099AC3F8344AC3F8B6
:10FC10002C1AC3F8302AFFF77FFFCBE7D819080862
:10FC2000748D0808B0920808E4E30020641C0808FA
:10FC3000E8700808CC190808B8D90020907808089E
:10FC40002DE9F04385B05C4903AA64F09BFA0028D3
:10FC500000F096800024DFF88491584FDFF880810F
:10FC600025464FF0FF36002D45D0012D48D154498F
:10FC70000446412305E09E4548D1494513D011F87B
:10FC8000013FA3F14102192A14F8012BA2F1410C02
:10FC900098BF2033BCF1190F02F1200EEBD99A4224
:10FCA00034D1002BE9D10024434903AA00200135B7
:10FCB00064F068FA0028D6D1012D63D0022D1FD13F
:10FCC000404D414FAC55DFF81081044604E0A64298
:10FCD00004D001340E2C16D0731CF8D12B5D07EB29
:10FCE00083034246D3F8BC3700930021234601200A
:10FCF000FFF762FCEDE7F6F73BFE0D280646D3D989
:10FD00003248FEF785FB05B0BDE8F0833049044674
:10FD10004D2305E09E4517D18F4213D011F8013FC6
:10FD2000A3F14102192A14F8012BA2F1410C98BF4A
:10FD30002033BCF1190F02F1200EEBD99A4203D106
:10FD4000002BE9D10124AFE72249532305E09C456C
:10FD5000D6D1414512D011F8013FA3F14102192A31
:10FD600010F8012BA2F1410498BF2033192C02F1A5
:10FD7000200CECD99A42C3D1002BEAD1022493E79C
:10FD80004FF0FF36DFF840800E4F134D002404E0A3
:10FD9000A64204D001340E2CB5D0721CF8D1E35D1C
:10FDA00008EB83032A46D3F8BC370093002123468F
:10FDB0000120FFF701FCEDE7E87008087E1C0888C9
:10FDC000781C0808048D00208C790708CC190808D5
:10FDD000801C0808F8670808881C0808761C088832
:10FDE000F667088810F040002FD00CB470B50C46B0
:10FDF00082B029B1002002B0BDE8704002B0704767
:10FE0000174EB56B6B7A5A1C2B44D2B223216A72FF
:10FE100099722B7A934219D9069A124907AB284650
:10FE200001935EF015FDB46B627A32B1D4E9003013
:10FE300004F10A01984700236372FFF7C7FA012013
:10FE400002B0BDE8704002B070477047002AE3D0AE
:10FE5000D5E9003005F10A0198476C72B56BDBE714
:10FE6000B8D9002029E100082DE9F0473B4C86B0C5
:10FE7000904681460D4616460027A4F2CC7AB8F18A
:10FE8000000F56D030782B78834254D000210023C5
:10FE90001A4605E00133392B5CD004EBC30212791A
:10FEA0009042F7D1F07805914FF4617C192212FB52
:10FEB00000C00390B0780AEBC30312FB00C20292A9
:10FEC000707893F8D137264ACDE900303B46484652
:10FED000FFF788FF0599287800231A4605E00133CB
:10FEE000392B37D004EBC30212799042F7D1E8786E
:10FEF0004FF4617C192212FB00C00390A8780AEB32
:10FF0000C30312FB00C2029293F8D10795F801C017
:10FF1000134ACDE9000C3B4648460137FFF74CFB3E
:10FF2000282F05F1040506F10406A8D106B0BDE8A6
:10FF3000F0874146CFE76A7873789A42A6D1AA78CB
:10FF4000B3789A42A2D1E978F378C91AB1FA81F16B
:10FF500049099CE700235B79FFDE00BF5881070851
:10FF6000A01C0808002875D0F0B5037883B00446BB
:10FF7000002B5AD0F6F7FCFC2728054661DC00234D
:10FF8000601C20218DF8073066F0EBF9AE000446C6
:10FF900018B303461C4613F8012B202AFAD020463A
:10FFA000F6F7E6FC002818DB0023C1B21A462B48FE
:10FFB00005E00133392B00EBC3020ED05279914298
:10FFC000F7D12749274A01EBC303324493F8D037CE
:10FFD00082F88C3A01238DF807302046202166F004
:10FFE000C0F9044698B103461C4613F8012B202A99
:10FFF000FAD02046F6F7BCFC152808D8194B334434
:020000040801F1
:1000000083F88D0A9DF8073001338DF80730164FBD
:10001000B11C0DF1070239442046FEF70FF99DF897
:100020000730042B08D103B0F0BD0F490022012096
:1000300003B0BDE8F04017E7002347F8253003B0D0
:10004000F0BD0A490A482723002203B0BDE8F0406A
:10005000FEF7DEB904490022012005E758810708B0
:100060008C790708B8D9002044E40020441C080813
:10007000F41908082DE9F04F89B002F15403444EF9
:10008000444FDFF818A10693904681460C4615466A
:1000900094F90430404A92F90010994202F10C029E
:1000A0000AD09642F7D1069B0C359D4204F10C0410
:1000B000EED109B0BDE8F08FB8F1000F3FD095F94F
:1000C000042093422B683CD0687995F806C095F8D7
:1000D00008B095F807E00021009357F82E300493FC
:1000E00057F82B30039357F82C30029357F82030F1
:1000F00001934846134652460791FFF773FE94F961
:1001000004300799E279206857F822200492227A75
:1001100057F822200392A27957F82220029262799E
:10012000009057F82220019248465246FFF744FAC1
:10013000069B0C359D4204F10C04A9D1B9E7414658
:10014000E0E721686879994206D095F806C095F8ED
:1001500008B095F807E0BEE7617995F806C08142DE
:1001600004D095F808B095F807E0B4E7A17995F8C0
:1001700008B0614502D095F807E0ACE7217A95F820
:1001800007E05945A7D1E1797145A4D10121A3E741
:100190004CDA002084720708F8D90020B41C080843
:1001A000D8B10278CAB12DE9F04F89B0461CF6F7F4
:1001B000DFFB5A4D014647B22A46002392F904005C
:1001C000B84202F10C020CD00133072BF6D154488F
:1001D00009B0BDE8F04FFEF71BB9504900220120DD
:1001E00048E703EB430305EB830595E8070005AB00
:1001F00083E8070081462021304666F0B2F86B792B
:100200000293EB7903932B7A95F806A0019383462A
:10021000002800F0818003461A78202A9B4603F1CB
:100220000103F9D02B2A69D02D2A3DD118469B46CF
:10023000F6F79EFB012303FA00F029EA00090224E5
:10024000013401275846202166F08BF8661EF6B26D
:1002500007F1FF3898B3834610F8013B202BFAD002
:100260005846F6F785FB00232E491A4601E051F85F
:10027000042F90425FFA83FE03F1010303D0112B98
:10028000F5D1E0B98646B8F1020F13D0B8F1030FEB
:1002900018D0B8F1010F10D0042FCDF808E038D0F5
:1002A0000134E4B20137CDE75846F6F761FB02248A
:1002B0008146C5E7CDF804E0D646F246F0E7DDF822
:1002C0000CE03446012C13D9029B8DF81930019BA8
:1002D0008DF81C30CDF814908DF81AA08DF81BE025
:1002E00005AB93E8070085E8070009B0BDE8F08F8B
:1002F0000D4809B0BDE8F04FFEF78AB818469B4696
:10030000F6F736FB012303FA00F049EA000902245C
:1003100096E7DDF80CE0D5E7012491E7AC8C0020EE
:10032000D41C080884720708CC1908082DE9F04F7E
:1003300089B0DFF8E8A0079281460C4615460026F2
:100340004FF019084FF4617739E0A378A878834219
:100350002B7839D06A7895F803C095F804E095F8C1
:1003600005B0002118FB027218FB0373CDE90232BD
:10037000CDE900B0CDE904CE334652464846069159
:10038000FFF730FD069923790593E37804936278AB
:10039000237818FB027218FB0373CDE90232A378AD
:1003A0000193627900923346524648460136FFF780
:1003B00003F9142E04F1060405F1060519D0079B74
:1003C000002BC2D10799DEE722789A426A7806D0DC
:1003D00095F803C095F804E095F805B0C1E7617899
:1003E00095F803C0914207D095F804E095F805B060
:1003F000B7E709B0BDE8F08FE17895F804E0614512
:1004000002D095F805B0ACE7217995F805B07145B3
:10041000A7D161795945A4D10121A3E7E81C0808B7
:10042000002800F0AC802DE9F047037882B0074641
:1004300033B956490022012002B0BDE8F04775E704
:10044000F6F796FA1328044600F39080781C0023F0
:1004500020218DF8073065F084FF4C4E04EB4405F5
:100460004FEA4508670006EB4505814698B103460B
:10047000994613F8012B202AFAD04846F6F778FA65
:10048000032808D8424B3A1903EB420383F8310B97
:1004900001238DF807304846202165F062FF814630
:1004A000B0B10346994613F8012B202AFAD04846EA
:1004B000F6F75EFA152803460AD89DF80710344A65
:1004C00001318DF80710391902EB410282F82E3BF9
:1004D0000DF1070229464846FDF7B0FE202165F0E0
:1004E00040FF824600284ED003469A4613F8012B5F
:1004F000202AFAD05046F6F73BFA3B28034642D86A
:100500009DF80790224A391909F1010902EB4102CD
:100510005FFA89F98DF8079082F82F3B5046202129
:1005200065F01FFFA8B10346184601330278202A60
:10053000FAD0F6F71DFA15280BD8154B3C4409F1F3
:10054000010903EB44045FFA89F98DF8079084F8F8
:10055000300BB9F1060F06D0002346F808300D48DD
:10056000AB80FDF755FF02B0BDE8F0870A490B48A4
:100570001323002202B0BDE8F047FDF749BF03494D
:1005800000220120D2E69DF80790C7E7E4E40020AE
:10059000B8D90020CC190808441C0808F419080828
:1005A0002DE9F04F2DED088B99B0DFF820B10792BF
:1005B00082460C461546002660E0F4EE4A8AF1EECB
:1005C00010FA77D1B4EE6A9AF1EE10FA72D1F4EE25
:1005D0004B9AF1EE10FA0CBF0121002114A80691EC
:1005E000F6F7A2F8B0EE4A0A074610A8F6F79CF80C
:1005F0000DF13009B0EE6A0A05904846F6F794F816
:100600000DF120080490B0EE4B0A4046F6F78CF846
:10061000059B049A0390CDE9007302920699334634
:100620005A465046FFF7DEFBB0EE480A14A8F6F72C
:100630007BF8B0EE680A074610A8F6F775F8B0EE3A
:10064000490A034648469946F6F76EF8B0EE690A3D
:10065000034640469846F6F767F833460390CDE9DF
:10066000019800975A46002150460136FEF7A4FF34
:100670000C2E04F1100405F1100522D094ED008A2F
:10068000B5EE408AF1EE10FA1BD0079BD4ED018A3B
:1006900094ED029AD4ED039A73B195ED000A95EDAD
:1006A00001AAD5ED02AA95ED03BAB4EE408AF1EEA7
:1006B00010FA82D0002191E70DF130090DF12008E8
:1006C000B2E719B0BDEC088BBDE8F08F081D080833
:1006D0002DE9F041A0B3037806468BB3411C6C4C66
:1006E0000530722207E09D4238D1884214D011F8BB
:1006F000013B14F8012FA3F1410EBEF1190FA2F135
:10070000410C98BF2033BCF1190F02F12005EAD942
:100710009A4223D1002AE8D15E4991F8A62B4FF4E2
:10072000C87002FB00F001F6CC3301F68C420344A2
:100730000244002143F8101F9342FBD1BDE8F08131
:10074000544991F8A63B4FF4C87000FB0311BDE873
:10075000F041002201F6DC31012021E73046F6F7B6
:1007600007F90B28044600F289802021304665F005
:10077000F8FD0546002800F0898003461D4613F861
:10078000012B202AFAD02846F6F73EF8414A92F883
:10079000A63B03EB830303EB8303234402EB031326
:1007A00003F6DC3383ED000A01262846202165F09C
:1007B000D8FD0546B8B103461D4613F8012B202A83
:1007C000FAD02846F6F720F8324A92F8A63B03EB17
:1007D000830303EB8303234402EB031303F6DC33AD
:1007E000013683ED010A2846202165F0BAFD054651
:1007F000B8B103461D4613F8012B202AFAD028462B
:10080000F6F702F8234A92F8A63B03EB830303EBC7
:10081000830302F6CC32234402EB0313013683ED4B
:10082000060A2021284665F09CFD034608B31846B9
:1008300001330278202AFAD0164D95F8A67BF5F7F9
:10084000E3FF07EB870303EB830305F6CC35234473
:1008500005EB0313032E83ED070A0AD14FF4C87387
:1008600003FB075505F110010022BDE8F04101200E
:1008700096E6BDE8F0410848FDF7CABDBDE8F04185
:10088000064907480B230022FDF7C2BD06468CE748
:10089000D8190808B8D90020CC190808441C080841
:1008A000F41908082DE9F04F91B0DFF82CB1069249
:1008B00081460C469046002509AF0BAE39E01A463A
:1008C00041493046F5F708FB069B002B48D098F8C5
:1008D00000C02378634545D000213C4B059300239D
:1008E0000493B8F912300393B8F91030384A0293E0
:1008F0000192CDF800C02B465A4648460791FFF7B3
:1009000071FA07990597237D0493B4F91230039384
:10091000B4F9102014F8203B0093CDE901622B4676
:100920005A4601354846FEF747FE082D08F12008D3
:1009300047D004F1150A04225146384665F048FDB7
:10094000D4E902320021082B8DF8281072F1000141
:10095000B5D320493046F5F7BFFA069B002BB6D138
:100960001946CFE7D8E90213E268A0689A4208BFA7
:100970008842B1D1227D98F814309A42ACD19AF8CD
:10098000002098F815309A42A6D19AF8012098F8DC
:1009900016309A420AF1010A9ED11AF8012F98F8EE
:1009A00017309A4298D19AF8012098F818309A4254
:1009B00092D12169D8F81030C91AB1FA81F14909E8
:1009C0008BE711B0BDE8F08F6C2408089078080818
:1009D000141408081C1D0808281D0808002800F029
:1009E00092802DE9F04F037883B080463BB300F14D
:1009F000004E41469E48AEF1020E722207E09C4531
:100A000024D1714512D011F8013F10F8012FA3F144
:100A10004107192FA2F1410698BF2033192E02F188
:100A2000200CECD99A4211D1002AEAD191484FF416
:100A30008072002103B0BDE8F04F64F033BD8D49F2
:100A40000022012003B0BDE8F04F2BE74046F5F748
:100A50008FFF83B2072B07464CD82021404665F014
:100A600080FC8146002800F0F5800346994613F883
:100A7000012B202AFAD04846F5F77AFF01260FFA13
:100A800080F82021484665F06CFC002800F0E580E5
:100A900002461378202B1046114602F10102F8D0CD
:100AA000002B00F0D280002500F1100C2C460BE04A
:100AB000D2B211F8013F240113F0DF0F44EA15749C
:100AC00042EA051500F0C380A3F130028C45D2B292
:100AD000A3F1610E1BD0092AEBD9BEF1050FA3F1DA
:100AE0004109A3F15702E3D9B9F1050F0FD8373BFC
:100AF000DAB2DEE7604961480723002203B0BDE8AF
:100B0000F04FFDF785BC5B4900220120CAE60023B7
:100B100001930136F6B2202165F023FC82460028BD
:100B200000F0A38003469A4613F8012B202AFAD03E
:100B30005046F5F71DFF01360FFA80F9F6B2504620
:100B4000202165F00EFC8246002800F08C800346D0
:100B50009A4613F8012B202AFAD05046F5F708FFE1
:100B600001360FFA80FBF6B25046202165F0F9FB02
:100B70008246002875D003469A4613F8011B2029A7
:100B8000FAD05046F5F7F4FE013643B20093F6B2C0
:100B90005046202165F0E5FB002860D0024610F8A1
:100BA000013B202BFAD00136F6B2032E47D91FFAAB
:100BB00088F3022B43D809F226239BB2B3F5E16FE9
:100BC0003DD80BF226239BB2B3F5E16F37D89DF8E1
:100BD00000A0BAF1060F32D8104600925EF07AF803
:100BE00004282CD8019B53B32549009A25483FB2CD
:100BF00001F56F6301EB471181F8F08EA1F8009FBA
:100C0000A1F802BF81F804AF03EB47110B46C1E91D
:100C100002541533511E033211F8014F055D05F0E2
:100C20000305022D264608BFA4F1200603F8016B38
:100C30000C780CB19142EFD103B0BDE8F08F1248AF
:100C400003B0BDE8F04FFDF7E3BB1D461C46012392
:100C500001935EE70646804613E701905BE70B4A87
:100C6000A3E7009094E783467EE7814667E700BFED
:100C7000D8190808A8E800204C1D0808F41908082D
:100C8000B8D90020F1880808CC190808907808081D
:100C90002DE9F047DFF8D4A088B0914680460C4695
:100CA00015460026B9F1000F35D0627A6B7A9A4268
:100CB0002A6832D06868B5F90A70B5F90CC095F8A1
:100CC00008E00021CDE90020CDE90237CDE904CECE
:100CD0003346524640460791FFF784F80799237A36
:100CE0000593B4F90C300493B4F90A300393637A92
:100CF0000293626854F8107B3346CDE90072404697
:100D000052460136FEF758FC112E05F11005C9D1E7
:100D100008B0BDE8F0874946E1E72168686891427C
:100D200006D0B5F90A70B5F90CC095F808E0C8E727
:100D30006168B5F90A70814204D0B5F90CC095F824
:100D400008E0BEE7B4F90A10B5F90CC0B94202D008
:100D500095F808E0B5E7B4F90C1095F808E061459E
:100D6000AFD1217A7145ACD10121ABE75C1D0808F8
:100D7000002800F0E8802DE9F04F037883B00646A4
:100D800043B300F100407E4C31460238722207E046
:100D90009D4226D1814214D011F8013F14F8012F51
:100DA000A3F1410EBEF1190FA2F1410C98BF2033FF
:100DB000BCF1190F02F12005EAD99A4211D1002A9B
:100DC000E8D170484FF48872002103B0BDE8F04FBD
:100DD00064F068BB6B490022012003B0BDE8F04F0E
:100DE00056E73046F5F7C4FDC3B2102B054600F2B6
:100DF000A1802021304665F0B4FA0446002800F0B6
:100E0000B48003461C4613F8012B202AFAD0204652
:100E1000F5F7AEFD012607462046202165F0A1FA30
:100E20000446002800F0A68003461C4613F8012B58
:100E3000202AFAD02046F5F79BFD01368046F6B20F
:100E40002046202165F08DFA0446002800F09080AD
:100E500003461C4613F8012B202AFAD02046F5F74A
:100E600087FD012881467AD80136F6B22046202136
:100E700065F077FA824600287ED003469A4613F83A
:100E8000012B202AFAD05046F5F772FD00F5B47315
:100E9000B3F5347F044662D80136F6B250462021BD
:100EA00065F05FFA8346002868D003469B4613F836
:100EB000012B202AFAD05846F5F75AFD00F5B473F5
:100EC000B3F5347F82464AD80136F6B2584620211F
:100ED00065F047FA0346002839D09B4601339BF85A
:100EE0000020202AF9D05846F5F742FD0346013686
:100EF00058462021B3F1000B18BF4FF0010BF6B29A
:100F000065F02FFA08B10136F6B2062E27D11E4B36
:100F10006DB203EB0513C3F8F07FC3F8F48F83F8C9
:100F2000F99FA3F8FA4FA3F8FCAF83F8F8BF03B01A
:100F3000BDE8F08F154916481023002203B0BDE824
:100F4000F04FFDF765BA0F4900220120A0E62021ED
:100F5000019065F006FA019B9B460028D3D10D480D
:100F600003B0BDE8F04FFDF753BA0646074653E716
:100F700081467BE7804663E704468FE78246A5E724
:100F8000D8190808A8E90020B8D900207C1D080855
:100F9000F4190808CC1908082DE9F04F91B0DFF8D2
:100FA00090A081468846174600240BAE22E078596F
:100FB000029A1B79049082428DF814302DD00125BD
:100FC0000DF1180B594604A885F0010558F0BCFF37
:100FD000CDF800B02346524629464846FEF702FFA8
:100FE000234600965246294648460134FEF7E4FA65
:100FF000802C19D004EB840508EB050358F8050094
:101000001B790290314602A88DF80C3058F09CFFF5
:101010007B19002FCBD13D46E2E79DF80C20DBB2D7
:101020009A42CCD10025CBE711B0BDE8F08F00BFCC
:10103000901D0808002800F0DF802DE9F04F0378AC
:1010400089B00446002B3DD0F5F792FC7F28054679
:101050003FDC2046202165F084F9044628B1034690
:101060001C4601332278202AFAD07249DFF8D89141
:1010700005EB8503CA180027A8000126CF5003906E
:1010800017714FF02C0C0297BA460197B846BB4631
:1010900032462378701EC0B223B30DF1140E002126
:1010A00005E00EF8013B14F8013F0131DBB1634567
:1010B00000F0A6800A29F4D15F4809B0BDE8F04FDE
:1010C000FDF7A6B95B490022012009B0BDE8F04F49
:1010D00062E75A495A487F23002209B0BDE8F04F21
:1010E000FDF796B9194601F120030DEB030101F854
:1010F0000CBCBCF1000FDFD1431E0134032B00F206
:101100008E80DFE803F06C4F280205A8F5F730FC6D
:101110001028A8BF002000F00F00039A454B029949
:101120002A44484D1344154407F00F07019A85F8E7
:10113000BD2640EA081047EA01174FEA281885F84B
:10114000BC7685F8BEA6D87083F8048009B0BDE8E7
:10115000F04F3BF01FBE9DF8141005A8E9B1DFF871
:10116000ECE000234FF0430C01E01EF801CB8C456E
:101170003BD00133082BF8D1DFF8D4E000234FF047
:10118000540C01E01EF801CB8C4530D00133072B05
:10119000F8D110F8011F0029E1D1013619F801CB6F
:1011A000F6B276E79DF8143005A983B9F5E7452B2B
:1011B0002DD0532B2DD0572B2DD0552B2DD0442B4C
:1011C00008BF052306D011F8013F002BE5D04E2BB8
:1011D000EDD1002302FA03F348EA0308F3E705A878
:1011E000F5F7C6FB01220746D7E70193C4E702FAE9
:1011F00003F34AEA030ACCE70E4900220120CBE6BA
:1012000001F120030DEB030101F80CBC74E701238D
:10121000E0E70346DEE70323DCE70423DAE705A87B
:10122000F5F7A6FB052E02904FF00102B5D1002084
:1012300073E700BF74E00020CC190808441C0808BC
:10124000F4190808B8D90020218307082983070862
:10125000318307082DE9F04F87B001F53073DFF8CF
:10126000C8A005919146054602F5307B04930027FE
:10127000DDF81080002415E01BF804100191711AAC
:10128000B1FA81F1490900940391FEF7ABFD03998E
:10129000CDE900463B46524628460134FEF78CF91C
:1012A000062C09D018F8016B3B4652462846B9F186
:1012B000000FE1D14946EBE7049B01370633062FC7
:1012C0000BF1060B0493D3D1059BDFF85C8003F28E
:1012D000E32A4FF4397417E019F804100191791AD0
:1012E000B1FA81F1490900960391FEF77BFD03995C
:1012F0000623CDE9006742462846FEF75DF9013432
:1013000040F2ED239C420BD01AF8017F062342469F
:101310002846A4F53976B9F1000FDDD14946E7E753
:1013200007B0BDE8F08F00BF9C1D08082DE9F04F05
:101330008FB0DFF8B890099282460C461546002619
:1013400031E02868BDF828100C9080B2AB88ADF869
:1013500034308142B5F9023095F801C095F804E0C7
:101360002A7835D00021CDE9023ECDE9002CCDF818
:10137000108033464A4650460891FEF733FD0899DF
:10138000069A0192079A00923346CDE903B8029774
:101390004A4650460136FEF70FF9202E04F10604A6
:1013A00005F106051FD0A388ADF82C30B4F9027002
:1013B000637820680693237894F804B094F9058044
:1013C0000A9007937FB1099B002BBAD11946D7E742
:1013D000BB42C7D1BDF82C00BDF83410411AB1FA98
:1013E00081F14909BFE70FB0BDE8F08FB01D0808D3
:1013F000F0B589B007465DF06DFC10F0FF0232D009
:10140000484C7E1D3946722205E09D4239D1B142D9
:1014100014D014F8012F11F8013BA3F1410EBEF1D5
:10142000190FA2F1410C98BF2033BCF1190F02F142
:101430002005EAD99A4224D1002AE8D13A4A3B4B06
:1014400092F8A61B4FF4C87000FB01221868998817
:1014500002F69C4302F65C521860998006339A4269
:10146000FAD109B0F0BD304991F8A63B4FF4C870ED
:1014700000FB031101F69C41012009B0BDE8F040DA
:1014800054E72B4901AA384662F07CFE4FF0FF3347
:10149000079378B1264E02AD0024F5F769FA01AA48
:1014A00045F8040B31460020013462F06BFE30B188
:1014B000062CF2D11F48FCF7ABFF09B0F0BD042C9D
:1014C000F8DD029B1F2BF5D8039A0F2AF2D8049C53
:1014D000262CEFD8059F07F57A71B1F5FA6FE9D898
:1014E000069EFF2EE6D8079D691C4029E2D80E49CA
:1014F00091F8A60B4FF4C87C0CFB00F04FF0060CE3
:101500000CFB03030B440C4883F89C2C83F89D4C84
:10151000A3F89E7C83F8A06C83F8A15CFFF768FFBA
:101520009FE700BFD8190808B8D9002038830708FA
:10153000E8700808CC190808907808082DE9F04FE1
:10154000A1B0DFF834A1129206461F4688469346A2
:101550004FF000090BE04F450BD009F10109B9F13B
:10156000400F08F114080BF1140B00F081807B1C74
:10157000F1D145460FCD16AC0FC42B68236098F807
:1015800010300E9398F911300F9398F8123098F8A4
:101590000420109398F8133009920D93D8F808207E
:1015A000129B0C9298F80C200A900B92002B48D0BA
:1015B0001A9B9BF804C023F07F4EDBF80030119398
:1015C000DBF8083014939BF80C3013935D469BF8BE
:1015D000133015930FCD1BAC0FC42B68236023F081
:1015E0007F439E452FD000210D9B07930C9B0693B4
:1015F0000B9B05930A9B0493099B0393109B0293F7
:101600000F9B01930E9B009352464B46304611911F
:10161000FEF7E8FB11990D9B07930C9B06930B9B20
:1016200005930A9B0493099B0393109B02930F9BC2
:1016300001930E9B009352464B463046FDF7BCFF8C
:101640008BE71946E7E7099B6345CCD10A9B8342A8
:10165000C9D10B9B139A9342C5D10C9B149A934208
:10166000C1D10D9B159A991AB1FA81F14909BBE7CD
:1016700021B0BDE8F08F00BFC81D08082DE9F0417A
:101680008AB006460C465DF025FB10F0FF0010D135
:10169000524B93F83E2022B1631C3CD10AB0BDE806
:1016A000F0814F494FF0FF3301200AB0BDE8F0410F
:1016B00044E74C4C701D3146722205E09D4232D108
:1016C000814214D014F8012F11F8013BA3F1410E0F
:1016D000BEF1190FA2F1410C98BF2033BCF1190FD4
:1016E00002F12005EAD99A421DD1002AE8D13E48EC
:1016F0003E4A904203D3D1E714309042CED20388C1
:10170000C3F30B03B3F57E7FF6D135490AB0BDE8CC
:10171000F041F5F7E1BD32490246234601200AB007
:10172000BDE8F0410AE732496A46304662F02AFDD8
:1017300078B12F4E6D460024F5F71AF96A4645F840
:10174000040F31460020013462F01CFD38B1092C31
:10175000F2D12848FCF75CFE0AB0BDE8F081092C04
:10176000F7D101993F29F4D8029B012BF1D80398B6
:10177000421C402AEDD8049F342FEAD8DDF814E04B
:10178000BEF1070FE5D8DDF818C01B4C0CF574222C
:1017900002F51072A242DCD8079E072ED9D8089D08
:1017A00005F5742202F51072A242D2D8099CFF2CD2
:1017B000CFD8124A4FF0140808FB012209B2507624
:1017C00013760F48977682F80CE0C2F808C01675B9
:1017D0001561D476FFF752FF60E700BFB8D900204B
:1017E000B8EA0020D8190808748D0808B0920808D3
:1017F000E8700808CC19080880841E00B0EA0020B0
:10180000907808084FF0FF3138E700BF2DE9F04F1E
:10181000A3B0DFF824B1129207468A4691464FF0F2
:101820000008DAF800300B93DAF808300D939AF8D4
:101830000C300C93BAF810300E93BAF812300F93A4
:10184000BAF814301093D446BAF816301193BCE8A5
:101850000F0014AC0FC49CE80700129B9AF80460B8
:101860009AF8185084E80700002B45D0CC46BCE815
:101870000F001BAC0FC49CE8070099F818E0AE45B8
:1018800084E807003AD00021119B0893109B07932E
:101890000F9B06930E9B05930D9B04930C9B039348
:1018A0000B9B0095CDE901635A4643463846139198
:1018B000FEF798FA1399119B0893109B07930F9BBF
:1018C00006930E9B05930D9B04930C9B03930B9B1C
:1018D0000293CDE9005643465A46384608F10108BE
:1018E000FDF76AFEB8F1040F0AF11C0A09F11C09A0
:1018F00097D123B0BDE8F08F1946DCE799F80430A2
:10190000B342C0D1D9F800300B9A9A42BBD199F8B2
:101910000C300C9A9342B6D1D9F808300D9A9A42FD
:10192000B1D1189A8242AED11999209BC91AB1FA45
:1019300081F14909A8E700BFEC1D08082DE9F04333
:101940008DB007465DF0C6F910F0FF0231D0504C63
:101950007E1D3946722205E09D4230D1B14214D03D
:1019600014F8012F11F8013BA3F1410EBEF1190F3C
:10197000A2F1410C98BF2033BCF1190F02F12005F0
:10198000EAD99A421BD1002AE8D14248424A904201
:1019900003D32EE0143090422BD20388C3F30B0301
:1019A000B3F57E7FF6D13D490DB0BDE8F043F5F7C4
:1019B00093BC3A4901200DB0BDE8F04326E7384911
:1019C00001AA384662F0DEFB80B1354E02AD00243C
:1019D000F4F7CEFF034645F8043B01AA3146002048
:1019E00062F0D0FB013438B10A2CF1D12D48FCF75C
:1019F0000FFD0DB0BDE8F0830A2CF7D1029B032B3D
:101A0000F4D8039A012AF1D804980728EED8DDF813
:101A10001480254C08F5742101F51071A142E5D818
:101A2000DDF818E0BEF1070FE0D8DDF81CC00CF5BA
:101A3000742101F51071A142D8D8089FB7F5004F65
:101A4000D4D2099EB6F5004FD0D20A9DB5F5004F0D
:101A5000CCD20B9CB4F5004FC8D214494FF01C09EE
:101A600009FB031383F80C0583F820251048C3F8FD
:101A7000088583F814E5C3F810C5A3F81875A3F812
:101A80001A65A3F81C55A3F81E45FFF757FFB0E7EA
:101A9000D8190808748D0808B0920808B8EF00201B
:101AA000E8700808CC19080880841E00B0EA0020FD
:101AB000907808082DE9F04FDFF88081A1B08346C7
:101AC0008A46002415460AEB44174FEA441C7968FD
:101AD0005AF80C00BA68FB6810AE0FC6386979690D
:101AE000BA69FB690FC6002D65D005EB0C0E55F8E1
:101AF0000C00DEF80410DEF80820DEF80C309DF84B
:101B0000406018AF0FC7DEF81C30DEF81000DEF8BA
:101B10001410DEF818200FC79DF86030BDF8427031
:101B2000B3424AD09DF84430BDF846209DF8489015
:101B3000BDF84A100C919DF84C100D91BDF84E1057
:101B40000B9100210B9807900D9806900C98019727
:101B5000CDE9023214ABCDE90490089300962346F8
:101B6000424658460B91FEF73DF90B99BDF84E20C1
:101B70009DF84C30069314A8CDE907209DF8483015
:101B8000BDF84A20CDE90432BDF846209DF8443026
:101B9000CDE90232BDF842209DF840305846CDE9EB
:101BA0000032234642460134FDF706FD032C8AD15C
:101BB00021B0BDE8F08F2946D8E7BDF86230BB42BE
:101BC0009DF84430B0D19DF864209A42BDF846207B
:101BD000ACD1BDF866109DF848909142A8D19DF80F
:101BE00068104945BDF84A10A4D108460C91BDF8CB
:101BF0006A1081429DF84C1004D00D91BDF84E1032
:101C00000B919EE708460D919DF86C108142BDF83E
